:020000040000FA
:100000000212FC022003FFFFFFFFFF02200BFFFF95
:10001000FFFFFF020E5DFFFFFFFFFF02201BFFFF40
:10002000FFFFFF022023FFFFFFFFFF02202BFFFF48
:10003000FFFFFF022033FFFFFFFFFF020EA0FFFFC5
:10004000FFFFFF022043FFFFFFFFFF02204BFFFFE8
:10005000FFFFFF022053FFFFFFFFFF02205BFFFFB8
:10006000FFFFFF022063FFFFFFFFFF02206BFFFF88
:10007000FFFFFF022073FFFFFFFFFF02207BFFFF58
:10008000FFFFFF022083FFFFFFFFFF02208BFFFF28
:10009000FFFF70DFFFFF040000000002000000C847
:1000A0000300030369A5020269A501000000000026
:1000B00004003273000074F8121043900393E06060
:1000C0001590030274FEF0900304744DF0A37405C0
:1000D000F07A011206747F0102116074F712104366
:1000E00074FF1212687E00801F851882851983E0D4
:1000F00064FE70069003877401F085188285198369
:10010000E0F8900384E068F07C017D00AA18AB1948
:10011000120E188B09EA450970030201E98518825D
:10012000851983E064EF70027E07E0C0E0900387EA
:10013000E0F8900385E0FAE82AF8E434001206C7F4
:10014000D0E0F0900387E060A014600E14602A14E1
:10015000603A14605014606680A0900384E4F085D7
:100160001882851983E0900386F0C39480900387FA
:100170004003E4808474028080851882851983E0BE
:10018000900382F090038774030200F9851882853A
:100190001983E0900383F0900386E0601990038751
:1001A00074040200F9900385E004F0F8900386E0FF
:1001B0006860030200FA90038774050200F9900357
:1001C00085E4F0900387F0900384E0F88518828539
:1001D0001983E06860030200FA900382E0644D60D6
:1001E000030200FA12031E8002EEF97401121234A7
:1001F0007F0202116074F712104374FB121268EA56
:10020000FEEBFF75080475090078081212CC740221
:100210001212E57A907B007904120EC17402121258
:1002200034120666121336E0687003A3E069701298
:10023000851882851983E0F47003A3E0F46003025B
:1002400002FE74041212DD1206D38A088B09A80874
:10025000A9097402121336E8F0A3E9F0740412132A
:1002600036E0600879011200B6020317851882850E
:100270001983E0687003A3E0697076851882851998
:1002800083E0F47003A3E0F470197402121336745F
:1002900010F0A37420F08518828519837410F0A3E0
:1002A0007420F075080175090078081212CC7402E8
:1002B0001212E57A247B08120F467402121234756A
:1002C000080478081212CC74021212E57A907B00AE
:1002D0007904120EC1740212123412066612133619
:1002E000E0687003A3E069700479028006790480F5
:1002F0000279031200B68E828F83741E80058E826F
:100300008F83E4F0120666121336E0687003A3E0F0
:1003100069700479018002790074050201ED74EDC1
:1003200012104374F8121268900307E0FA90030663
:10033000E0FB8B08EAF8E4C8F9EB28FEE93408FF93
:10034000751001880C750D068F0974027808121259
:1003500093C39508F8E49509F9740228F50E74031F
:1003600039F50F8E088F09740978081212EDE50827
:10037000F511EE2410F508E43FF509EEF50AEF5407
:1003800001F50B900383E0146054147003020453CE
:100390001470030204CE14601024FE700302058959
:1003A000147003020639020649750D03794E120CCA
:1003B0005890030712065C7402F0A3744012065AA8
:1003C000740812065AF0A3F0751012AA10A90C12A4
:1003D0000674A90D74081212347F0C021160750D99
:1003E00004794E120C58EE450B7005A911120FAC92
:1003F000C3EE9425EF9408503CC3E5089424E50926
:1004000094084031E50E2496F8E50F3420F98882EF
:100410008983E0701BA3AA82AB83E07013900388EA
:100420007401F08882898374A5F08A828B838004AA
:10043000900388E4F075081075090078081212CC52
:100440007C087D03EEFAEFFB120F467402121234A1
:100450000203CB750D05E511C394794006750C01B7
:100460000203CB75124075130078121212CC7C096E
:100470007D037402780A121293AA0AAB0BA9111217
:100480000EC17402121234900307E0A3F090030629
:10049000E0A3F0751043C3EE9425EF9408400302E7
:1004A00003CBC3E5089424E509940850030203CB69
:1004B000900388E070030203CBE50E2497F8E50F64
:1004C0003420F988828983E4F0A3F00203CB750815
:1004D0000475090078081212CC74021212E57A90A1
:1004E0007B007904120EC1740212123474021213CA
:1004F00036E0F8A3E0F9851882851983E068700377
:10050000A3E069851882851983700BE0F47003A35A
:10051000E0F470578009E0F47003A3E0F4700D85F7
:1005200018828519837410F0A37420F012066612E5
:100530001336E8F0A3E9F075080178081212CC74BC
:10054000021212E57A247B08120F4674021212344A
:1005500075080478081212CC74021212E57A907BA6
:10056000007904120EC174021212341206661213BC
:1005700036E0687003A3E0697006750D010203CBD5
:10058000750D02750C070203CB900391E0600764C0
:100590000260030203CBEAFF7A017900120674E0DD
:1005A000600302062D8003120D19120D23E970F766
:1005B000740412133612064E74041213367808129D
:1005C000131A85080C85090D850A0E850B0F9005F9
:1005D000A2780C1212B97404121336780C12130B91
:1005E000E5084509450A450B70CE8EC2E5C554E0C5
:1005F0004FF5C5740412133612064E7404121336E6
:10060000780812131A85080C85090D850A0E850BCA
:100610000F9005A2780C1212B97404121336780CDC
:1006200012130BE5084509450A450B70CE7A01798E
:100630000012067479080203D4EB900393F0700360
:100640000203CB750D090203CB79060203D4E4F053
:10065000A37426F0A3E4F0A3F022F0A3E4F0A3F047
:10066000A3F0A3F0A322851882851983E0F8A3E004
:10067000F974022274F6121043EAFE900305E0D2E8
:10068000E7F0E9A3F0EE900303F08E0A74042AFE6B
:100690007A028004E0620A0AEAF83395E01206C79B
:1006A0008E08C3E89508E99400A2D265D03340E4EF
:1006B000E50AF0740128FC3395E0FD7A027B031211
:1006C0000E487F03021160F9740228F58274033921
:1006D000F5832274E91210437582007583FE1211AE
:1006E000FB8A168B177514007515008A828B83E4BC
:1006F000F0900391E07006D2AAD2AF800464027039
:100700000579001200B6750C00750D20750E007588
:100710000F00900391E0600464027015120D19122D
:1007200000DBE9F87409686003020803790012002D
:10073000B675080075090278081212CC74021212FC
:10074000E5850C08850D09AA08E5095407FB850E07
:100750000A850F0B740B780812124FA908120EC1EC
:1007600074021212347E007F009005AAC0828E109F
:10077000EFF5113395E0F512F513850C08850D0999
:10078000850E0A850F0B780879101212A69005A61F
:1007900078081212B9758305D08278081211DC50DE
:1007A0001D851882851983E5822EF582E5833FF544
:1007B00083E0F9AA14AB151208328A148B150EEED9
:1007C00070010FC3EF940240A09005AE780C121296
:1007D000B99005B2780C1211DC40030207127900BF
:1007E000AA14AB1512083279001208328B15900347
:1007F00091E07004C2AFC2AAEA451570277AA57BC2
:10080000A58021E8700302073174066870030207AF
:100810003174076870030207318516828517837467
:1008200001F080BA7582007583021211FB7F1002FD
:100830001160C008C0097C088A088B09740F780809
:100840001212EDEA25E0FAEB33FBE9A2E75004745B
:10085000014AFAE508A2E0500874216AFA74106BA4
:10086000FBE9C333F91CEC70CFD009D0082274F730
:1008700012104378007900802374942508F582E4EF
:100880003403F583E08A828B83F09004141209F319
:100890004005900414E4F008E87001099004141273
:1008A000095D6007C3E89CE99D40CEE8FAE9FB7F5B
:1008B0000202116074F5121043900498E0FEA3E068
:1008C000FF8F08EEC39508F895E0F9EFC39EE85056
:1008D0000B120ADA701178007900801B247F500116
:1008E00009C39CE99D50EF7A007B008041E004F051
:1008F000D2E908E8700109C3E89CE99D502C8A827E
:100900008B83E0C0E0900499E0FE74182EF582E439
:100910003404F583D0E0120ACA90049AE4F09004FB
:1009200099E0C3947F40C6E480C5E8FAE9FB7F0400
:1009300002116074F7121043C2E990049812095D25
:10094000601874182508F582E43404F583E0F5C1D5
:10095000900498120AF14002E4F00208AFE0F508B2
:10096000A3E065082274F71210437800790090051F
:100970001DE07063A3E0705F75F900C28FC284A2AE
:100980008340FCA28F4004A28350F8E5F9C28FA2F5
:10099000835004D2848040C0E0E0FE749D2EF58236
:1009A000E43404F583D0E0F090051E120AF140D340
:1009B000E4F080CF749D2508F582E43404F583E0EB
:1009C0008A828B83F090051D1209F3400590051D66
:1009D000E4F008E870010990051D12095D6007C385
:1009E000E89CE99D40CEE8497006E4F090051DF0D2
:1009F0000208ABE004120ACEC394802274F81210ED
:100A0000439005A0E0FF8F82A88290059FE0FEEF53
:100A1000C39EE0500DC398F895E0F9120AD97018FA
:100A20008012C398F895E0F9E8247F500109C39C2F
:100A3000E99D4004EC4D70077A007B00020AC58AEC
:100A4000828B83E0F5F9A3AA82AB837801790080D9
:100A500008E004F008E8700109C3E89CE99D50270C
:100A60008A828B83E0C0E09005A0E0FE741F2EF523
:100A700082E43405F583D0E0120ACA9005A0E0C3F1
:100A8000947F40CDE480CCC28FA28340FCC284A27C
:100A90008F4004A28350F890059F120AE4E0F5F914
:100AA000C28F90059FE0FAA3E06A90059F7005123F
:100AB0000AE48005120AF14002E4F0A28350D0D289
:100AC00084E8FAE9FB7F01021160120ACE22F08A63
:100AD000828B83A3AA82AB8322E824FF18E934FF28
:100AE000F9E84922E0FA741F2AF582E43405F58317
:100AF00022E004F0C394802274FB1212687E0090FE
:100B000005CA780812131A9005CA7401F0A3F0A35D
:100B10007469F0A374A5F09005B6780812127E707F
:100B2000030E80159005BA780812127E6008E59DC4
:100B3000541864107003022000120C7EEEA2E050E4
:100B400003020BFBAA18AB191201F5E97003020BA3
:100B5000FB851882851983E0C3943C500CE0F8743F
:100B60003CC398FA95E0FB80047A007B00120D3CB0
:100B7000E97003020BFB900391E06401700C75F8BF
:100B800000C2AB539AF7D2EA805E79071200B680B2
:100B900003120D19120D23E970F77401121336E4D4
:100BA000F0A37426F0A3E4F0A3F0740112133678D6
:100BB0000812131A85080C85090D850A0E850B0F7E
:100BC0009005A2780C1212B97401121336780C1227
:100BD000130BE5084509450A450B70CE758600C222
:100BE000AAC28B539AFBC2E990000174CDF0022097
:100BF00000C2AF75C9AB75C95B80FE750800750989
:100C000000750A00750B00900391E0701BD2AAD208
:100C1000AF79051200B6E07003120D191200DBE97E
:100C2000F8740968700980E9794E120C5880ED74E7
:100C3000016870E2E07017120D199005BE78081275
:100C400012B99005C278081211DC50EBC2AAC2AFEB
:100C500075C9AB75C95B80FEC082C08378109005F2
:100C6000A1E0C399501575B60FE5B4A2E750FAE5B7
:100C7000BBC39940F118E870EDE9F0020D37C0826E
:100C8000C08353BEFBE59DA2E650FA0078F87901D7
:100C900000120AD970FA75C6807480659E70FA4396
:100CA000BE049062707408F0794A120C58900001EA
:100CB00074F5F07403F5D575D489A2A0E4339003DC
:100CC00091F0A2E05029D28453F3F753F3EF53FD90
:100CD000F743FD10538FF753F7DF43FC2043F10236
:100CE00053F5DF75F82043F4F0D2FED2AB802853E1
:100CF000FF3F85FFFF53F1FE43F30C53F2F375867C
:100D00008075C48090049BE4F0A3F075C2D875C5CB
:100D10000B75C402438640801E8003120933A2E98A
:100D200040F922C082C083900498E0F8A3E0686094
:100D300004790180027900D083D0822274F11210EC
:100D40004374FF1212687E00900391E06401706B9F
:100D5000C2849003927401F07508388E098E0A8E51
:100D60000B7C017D00AA18AB19120E188B0DEA45F9
:100D70000D6018851882851983E06410602CE0648A
:100D8000EF70088E088E098E0A8E0B85080C850977
:100D90000D850A0E850B0F9005A278081212B9E591
:100DA0000C450D450E450F70330E900391E0640124
:100DB0007056D284900392E4F08051D2AAD2AF8AC6
:100DC000088B09E4F50AF50B9005C6780C12131A86
:100DD0007808790C120FC379061200B6900391E0DF
:100DE0006003020D61120D191200DBE9F874096845
:100DF000700779061200B680927407686085E86013
:100E00008A74066870A48083C2AFC2AAEEF9740126
:100E10001212347F08021160C082C083900391E0F7
:100E2000700512086E801E900392E06015A28F502C
:100E30000BE5F98A828B83F07A0180027A007B00CD
:100E40008003120965020D37C082C083900391E0D0
:100E500070051208B480031209FC020D37C0E0745B
:100E6000F21210A9900001E064CD700512201380E9
:100E70002AE064F57024E5C1C28BC0E0900415E05F
:100E8000F8749428F582E43403F583D0E0F09004FC
:100E900015120AF14005E4F08001007F01021108FB
:100EA000C0E074F21210A9900001E064CD70051248
:100EB000203B800BE064F57005120933800100804F
:100EC000DA74F51210438908740F5508F50A750B8A
:100ED00000740B780A121293EA2400F8EB3480F9BC
:100EE000E82400E9350BF9E5C7F509A2AFE433F5CD
:100EF0000AC2AFE508C4540FFAE5C754F84AF5C76B
:100F0000740B121336E0FAA3E0FB801C88828983FD
:100F1000E08C828D83F088828983A3A882A9838C48
:100F2000828D83A3AC82AD83EAFEEBFFEE24FF1A31
:100F3000EF34FFFBEE4F70D48509C7E50AA2E092BB
:100F4000AF7F0402116074F7121043ED900389F033
:100F5000ECA3F0A37462F0A37473F0A3E0541FF049
:100F60007409121336E0F508A3E0F509E5083333F8
:100F700054FC90038EF0740678081212EDE5089088
:100F8000038DF090038F7412F0A37442F075D1FEBC
:100F900075D601EA906271F0EBA3F0906270E0D236
:100FA000E1F0E0A2E740FB7F02021160C082C08353
:100FB000E9C333906272F0906270E0D2E0F0D083C7
:100FC000D08222080808EAC0E0EBC0E086F0E7A47F
:100FD000FA180986F0E7A42AFA180986F0E7A42A85
:100FE000FA180986F0E7A42AFA1986F0E7A4FBE5C7
:100FF000F02AFA190886F0E7A42BFBE5F03AFA1973
:101000000886F0E7A42BFBE5F03AFA18180986F0F9
:10101000E7A4C5F02BFBE43AFA1908E7C5F0C6A42B
:1010200026F6E5F03BFBE43AFA1886F0E7A4F6E58D
:10103000F00826F6E43B08F6E43A08F6D0E0FBD0E8
:10104000E0FA222518C582C0E0E51934FFC583C047
:10105000E0E518C3958224F910AF088583198582CD
:10106000188008858319858218D2AFCEF0A3E520B9
:10107000F0A37808E608F0A3DEFAEFF0A3E58124F8
:10108000FBF8E608F0A3E608F0A30808E608F0A3DA
:10109000E608F0A315811581D0E0FED0E0F81581B7
:1010A0001581E8C0E0EEC0E022C0D02518C582C09E
:1010B000E0E51934FFC583C0E0E518C3958224F349
:1010C00010AF088583198582188008858319858269
:1010D00018D2AFC8F0A3E9F0A3EAF0A3EBF0A3792C
:1010E00008E709F0A3D8FAECF0A3EDF0A3EEF0A323
:1010F000EFF0A3D0E0F0A3D0E0F0A3D0E0F0A3E5C0
:1011000020F0A3E5F0F0A322851983851882E0C0C2
:10111000E0A3E0F9A3E0FAA3E0FBA37808E0F60877
:10112000A3DFFAE0FCA3E0FDA3E0FEA3E0FFA3E061
:10113000C0E0A3E0C0E0A3E0F5D0A3E0F520A3E089
:10114000A3F5F010AF088583198582188008858380
:1011500019858218D2AFD082D083D0E0F8D0E032A7
:10116000851983851882E0A3FEE0A3F5207808E0C6
:10117000A3F608DFFAE0A3FFE0A3C0E0E0A3C0E02D
:10118000E0A3C0E0E0A3C0E010AF0885821885832B
:10119000198008858218858319D2AFD083D0822226
:1011A000E490030278A179038002F0A3D8FCD9FA75
:1011B0007AA27B0590008E782979018015E493A3AB
:1011C000AD82AE838A828B83F0A3AA82AB838D82A9
:1011D0008E83D8E9D9E7120AF8121340C008C3E099
:1011E00096F50808A3E096420808A3E0964208088E
:1011F000A3E09645087001D3D00822C5822518C502
:1012000082C583351910AF07F5198582188007F557
:1012100019858218D2AFC583222518F58210AF0830
:10122000F518400C15198008F51840021519D2AFB1
:101230008519832200C0D0251810AF08F518500C6E
:1012400005198008F51850020519D2AFD0D02260D8
:1012500016080808C6C313C618C613C618C613C690
:1012600018C613C6D5E0EA22251810AF08F51840B5
:101270000C15198008F51840021519D2AF22E06646
:10128000701008A3E066700A08A3E066700408A363
:10129000E06622700422600D18C6C333C608C63348
:1012A000C6D5E0F41822E627F60809E637F608095D
:1012B000E637F60809E637F622E026F608A3E03618
:1012C000F608A3E036F608A3E036F62274028000A2
:1012D000C0E0F404121219D0E0121329222518FAE2
:1012E000E43519FB222518FCE43519FD22600C08B1
:1012F000C6C313C618C613C6D5E0F42275D0007550
:10130000813F7518027519030211A0E6F008A3E6E3
:10131000F008A3E6F008A3E6F022E0F608A3E0F662
:1013200008A3E0F608A3E0F622CAC0E0E6F0A308AE
:10133000DAFAD0E0FA222518F582E43519F583228D
:1013400000000080FBFFFFFFFFFFFFFFFFFFFFFF2D
:10135000FFFFFFFFFFFFFFFFFFFFFFFFFFFFFFFF9D
:10136000FFFFFFFFFFFFFFFFFFFFFFFFFFFFFFFF8D
:10137000FFFFFFFFFFFFFFFFFFFFFFFFFFFFFFFF7D
:10138000FFFFFFFFFFFFFFFFFFFFFFFFFFFFFFFF6D
:0A1FF600CA05094338860000000008
:020000040003F7
:01FFF000F020
:020000040000FA
:10200000022C2A0221E7FFFFFFFFFFFFFFFFFFFF78
:10201000FFFFFFFFFFFFFFFFFFFFFFFFFFFFFFFFD0
:10202000FFFFFFFFFFFFFFFFFFFFFF022918FFFF7A
:10203000FFFFFFFFFFFFFFFFFFFFFFFFFFFFFFFFB0
:10204000FFFFFF022745FFFFFFFFFFFFFFFFFFFF2F
:10205000FFFFFF022123FFFFFFFFFFFFFFFFFFFF47
:10206000FFFFFFFFFFFFFFFFFFFFFF0228F0FFFF63
:10207000FFFFFFFFFFFFFFFFFFFFFFFFFFFFFFFF70
:10208000FFFFFF02218301FFFFFFFFFFFFFFFFFFB5
:102090001020102001FF01010503010F10FEFF4475
:1020A0004B00000000DC4A00000000FF000000FFC1
:1020B00000010000D1380000000023380F3A6B38CF
:1020C00085390000593800000000000000000000C1
:1020D0000000000000000000000000000000FF0100
:1020E0000100A507000000FFFF1E08E8036400646C
:1020F00000B80102020008000005020701051E02E7
:10210000051E020A0A0103B80B02803E0102FEFF0F
:10211000E8030A050001FFFF0A01E09651180002DA
:1021200006FFFFC0E074F2122564A2AFE433FED2D2
:10213000AFE5A7FFE5A1F5085F5410600612429DC8
:1021400075A1EFE5085F540860081242A375A1F776
:102150008024E508A2E092F0EFA2E082F050179010
:102160006198E0F8900D4BE0C398A2D265D033504F
:1021700002E8F075A1FE751A00EEA2E092AF7F01B1
:102180000225C3C0E074F2122564A2AFE433FED28C
:10219000AF9061A4E0F8759B00E591585408600881
:1021A0007591F71242EB8023E59158541060087541
:1021B00091EF1242F18014E591A2E092F0E8A2E0E2
:1021C00082F05007E0C2E0F01244479061A3E0F8CB
:1021D000E5E9585404600E12441D75E9FB906193C3
:1021E000E0A2E640F2808FC0E074F2122564A2AF54
:1021F000E433FED2AF9061A5E0F8E5BF5854046027
:102200000675BFFB12445F022176C3E498F8E49997
:10221000F912224B8026C3E49AFAE49BFBE920E7FB
:10222000E912224BE498F8E499F922C3E498F8E41F
:1022300099F912224BE498F8E499F9C3E49AFAE484
:102240009BFB22EB20E7CFE920E7E0B90010BB00C1
:1022500008E88AF084F8AAF022E4FBC8FA22EB70BE
:10226000227B10C833C8C933C9335007C39AC3DBB4
:10227000F280069A50012ADBEAC833F4C8C933F465
:10228000C9FA2275F008E4C833C8C933C933C99AFA
:10229000C99B5004C92AC93BD5F0ECFBC833F4C82C
:1022A000E4C9FA2274F51224FE74FA122AC47508DD
:1022B000047509007808122A027404122A8E7AF82A
:1022C0007B0779031241777402122A309080AC7830
:1022D00008122C587402122CAF7808122AEF704999
:1022E0007508027509007808122A027402122A8EF3
:1022F0007AF67B0779031241777402122A30851827
:1023000082851983E0F47003A3E0F4601C851882D1
:10231000851983E0F8A3E0F9888289837402F0A329
:10232000F0A37469F0A374A5F0C2AF75D69F020044
:10233000007406122A307F04022788080808EAC0C1
:10234000E0EBC0E086F0E7A4FA180986F0E7A42ADB
:10235000FA180986F0E7A42AFA180986F0E7A42AF1
:10236000FA1986F0E7A4FBE5F02AFA190886F0E7E7
:10237000A42BFBE5F03AFA190886F0E7A42BFBE55D
:10238000F03AFA18180986F0E7A4C5F02BFBE43AF6
:10239000FA1908E7C5F0C6A426F6E5F03BFBE43AD7
:1023A000FA1886F0E7A4F6E5F00826F6E43B08F60E
:1023B000E43A08F6D0E0FBD0E0FA22E4CFC0E0E453
:1023C000CEC0E0E4CDC0E0E4CCC0E075F020E6266D
:1023D000F608E633F608E633F608E633F61818187A
:1023E000EC33FCED33FDEE33FEEF33FFC3EC970926
:1023F000ED9709EE9709EF97191919400FFFEC9720
:10240000FC09ED97FD09EE97FE191906D5F0BFEC12
:10241000F709EDF709EEF709EFF7191919D0E0FC04
:10242000D0E0FDD0E0FED0E0FF222518C582C0E05C
:10243000E51934FFC583C0E0E518C3958224F81080
:10244000AF088583198582188008858319858218CD
:10245000D2AFCEF0A3E520F0A37808E608F0A3DE23
:10246000FAEFF0A3E58124FAF8E608F0A3E608F015
:10247000A3E608F0A30808E608F0A3E608F0A31511
:10248000811581D0E0FED0E0F8158115811581E835
:10249000C0E0EEC0E022122CA4B900030224E8E45C
:1024A0009004D1780379118002F0A3D8FCD9FA788E
:1024B0001A9020867A01BA00028007E493A3F608F6
:1024C000DAF97AD37B14902094789079018015E41E
:1024D00093A3AD82AE838A828B83F0A3AA82AB835F
:1024E0008D828E83D8E9D9E77582CA7583E3740536
:1024F0001229DC75826D75834874001229DC251859
:10250000C582C0E0E51934FFC583C0E0E518C39576
:102510008224F910AF088583198582188008858385
:1025200019858218D2AFCEF0A3E520F0A37808E693
:1025300008F0A3DEFAEFF0A3E58124FBF8E608F04B
:10254000A3E608F0A30808E608F0A3E608F0A31540
:10255000811581D0E0FED0E0F815811581E8C0E05A
:10256000EEC0E022C0D02518C582C0E0E51934FFD6
:10257000C583C0E0E518C3958224F310AF088583B6
:10258000198582188008858319858218D2AFC8F012
:10259000A3E9F0A3EAF0A3EBF0A37908E709F0A31D
:1025A000D8FAECF0A3EDF0A3EEF0A3EFF0A3D0E0A7
:1025B000F0A3D0E0F0A3D0E0F0A3E520F0A3E5F095
:1025C000F0A322851983851882E0C0E0A3E0F9A377
:1025D000E0FAA3E0FBA37808E0F608A3DFFAE0FC4A
:1025E000A3E0FDA3E0FEA3E0FFA3E0C0E0A3E0C002
:1025F000E0A3E0F5D0A3E0F520A3E0A3F5F010AF51
:10260000088583198582188008858319858218D2E8
:10261000AFD082D083D0E0F8D0E0320975F0108ED0
:10262000218F22858226858325851882851983E05E
:10263000CEA3E0CF852682852583EBC9EAC8EDCB02
:10264000ECCAC3E833C8E933C9EA33CAEB33CBC3B6
:10265000EA9EF524EB9FF523B35004AB23AA24ECA8
:1026600033CCED33CDD5F0DAAE21AF2222D083D0FA
:1026700082ECC0E0EDC0E0E493A3FCE493A3FDEDA5
:102680004C600D1227C8EC24FFFCED34FFFD80EFF9
:10269000E493A3FCE493A3FDED4C600D12289BECA6
:1026A00024FFFCED34FFFD80EFD0E0FDD0E0FCE442
:1026B00093A3C0E0E493C0E022851983851882E0EB
:1026C000A3FEE0A3F5207808E0A3F608DFFAE0A374
:1026D000FFE0A3C0E0E0A3C0E0E0A3C0E0E0A3C04F
:1026E000E0E0A3C0E010AF08858218858319800858
:1026F000858218858319D2AFD083D0820229E2D097
:1027000083D082E9C0E0E493A3C386F0C5F095F0DE
:10271000F908E493A386F0C5F095F0700BE493A359
:10272000C3994005E9048002A3E475F002A4258260
:10273000F582E5F03583F583D0E0F9E493A3C0E0BA
:10274000E493C0E022C0E074F2122564A2AFE43347
:10275000FED2AFC2C09013CBE0700BE5D1A2E45023
:102760001D1241FB8018E5D1A2E3500675D1F71286
:1027700041D1E5D1A2E4500675D1EF1241D7EEA2C6
:10278000E092AF7F010225C3851983851882E0A3FB
:10279000FEE0A3F5207808E0A3F608DFFAE0A3FF47
:1027A000E0A3C0E0E0A3C0E0E0A3C0E0E0A3C0E09D
:1027B00010AF088582188583198008858218858363
:1027C00019D2AFD083D08222C0E0C3E493960874BC
:1027D00001939618400FE49366700808740193669D
:1027E0001870007019A3A3C3E4939608740193961C
:1027F00018A3A3400DD0E0D0E0D0E00226A9A3A307
:10280000A3A3A3A3D0E022D083D082C5F0E493A3F6
:10281000C5F0C395F0F5F0E493A3C395F04005E54A
:10282000F0048001E475F002A42582F582E5F0351C
:1028300083F583E493A3C0E0E493C0E022740480B2
:102840000474028000CCC0E0EDC0E0E518C39CCC6D
:10285000AD1950011D10AF068C188D1980068C180B
:102860008D19D2AF12295ED0E0FDD0E0FC227402B7
:102870008000CCC0E0EDC0E0E518C39CCCAD1950A1
:10288000011D10AF068C188D1980068C188D19D279
:10289000AF12293CD0E0FDD0E0FC22C0E0C0F088BF
:1028A000F0E4936670080874019366187000A8F04D
:1028B000A3A3700BD0F0D0E0D0E0D0E00226A9A313
:1028C000A3D0F0D0E022D083D082CCC0E0E493A3A8
:1028D000600612297F1470FAE493A36006122AAEF0
:1028E0001470FAD0E0FCE493A3C0E0E493C0E022CB
:1028F000C0E074F2122564758900C2C59013CBE064
:10290000700E7A007B10900719E0F9123BA180034A
:102910001246DB7F010225C3C0E0C0D0E8C0E0E979
:10292000C0E0E5A8D2AFC2C7751A00A2E7A2E7923D
:10293000AFD0E0F9D0E0F8D0D0D0E032CAC0E0E4C7
:1029400093A3C582CCC582C583CDC583F0A3C582C0
:10295000CCC582C583CDC583DAE5D0E0CA22CAC022
:10296000E0E0A3C582CCC582C583CDC583F0A3C5F5
:1029700082CCC582C583CDC583DAE6D0E0CA22C049
:10298000E0E493A3D39C5010E493A3C39C400AD0EB
:10299000E0D0E0D0E00228E3A3A3A3D0E022C00867
:1029A000C3E096F50808A3E096420808A3E0964223
:1029B0000808A3E09645087001D3D00822700908E2
:1029C0000808226016181818C6C333C608C633C6CE
:1029D00008C633C608C633C6D5E0EA22C09FF59FB5
:1029E000E473D09F22D083D082C09FE493C0E07470
:1029F0000193C0E0740293F59F227404800A74036B
:102A00008006740280027401C0E0F404122A15D01A
:102A1000E0122C67222518F58210AF08F518400C3B
:102A200015198008F51840021519D2AF85198322AF
:102A300000C0D0251810AF08F518500C05198008F3
:102A4000F51850020519D2AFD0D022BB0102E722FF
:102A5000C082C08389828A83BB0003E08002E49342
:102A6000D083D082226016080808C6C313C618C6D1
:102A700013C618C613C618C613C6D5E0EA22251811
:102A8000F8E43519F9222518FAE43519FB2225183E
:102A9000FCE43519FD22C3E0C696F608A3E0C6960D
:102AA000F608A3E0C696F608A3E0C696F622C0E0B4
:102AB000E493A36C7009D0E0D0E0D0E00228E3A357
:102AC000A3D0E022251810AF08F518400C15198086
:102AD00008F51840021519D2AF22C3E09608A3E00A
:102AE0009608A3E09608A3E096A2D265D03322E030
:102AF00066701008A3E066700A08A3E06670040818
:102B0000A3E06622E76670100809E766700A080904
:102B1000E76670040809E76622C3E697F60809E647
:102B200097F60809E697F60809E697F622C3E096B5
:102B3000F008A3E096F008A3E096F008A3E096F072
:102B400022E657F60809E657F60809E657F6080997
:102B5000E657F622E056F608A3E056F608A3E0563C
:102B6000F608A3E056F622E026F008A3E036F008C7
:102B7000A3E036F008A3E036F022E026F608A3E052
:102B800036F608A3E036F608A3E036F622E627F686
:102B90000809E637F60809E637F60809E637F622A7
:102BA000E647F60809E647F60809E647F60809E6A3
:102BB00047F622E056F008A3E056F008A3E056F0EE
:102BC00008A3E056F022700422600D18C6C333C675
:102BD00008C633C6D5E0F41822E4C396F608E49696
:102BE000F608E496F608E496F622C3E7960809E7A5
:102BF000960809E7960809E79622C6F4C608C6F4BF
:102C0000C608C6F4C608C6F4C622600D08C6A2E708
:102C100013C618C613C6D5E0F322C3E09608A3E096
:102C20009608A3E09608A3E0962275D00075813F30
:102C30007518D175190400022496600C08C6C313D8
:102C4000C618C613C6D5E0F422E6F008A3E6F008DD
:102C5000A3E6F008A3E6F022E0F608A3E0F608A356
:102C6000E0F608A3E0F622CAC0E0E6F0A308DAFA2C
:102C7000D0E0FA22EAF0A3EBF0A3ECF0A3EDF0220F
:102C8000E0FAA3E0FBA3E0FCA3E0FD22E0F8A3E070
:102C9000F9A3E0FAA3E0FB22E8F0A3E9F0A3EAF04D
:102CA000A3EBF022E5C754F84401F5C779012225CA
:102CB00018F582E43519F583221229E55EB2031274
:102CC00029E5D4B2031229E540B3031229E55CB328
:102CD000031229E58DB3031229E5CCB3031229E5CC
:102CE000CDB4031229E57CB5031229E509B8031216
:102CF00029E562B9031229E5F5B9031229E5CABA33
:102D0000031229E540BB031229E5A8BC031229E5FB
:102D1000C6BC031229E50080021229E55A8002127E
:102D200029E5C480021229E54D81021229E50982B4
:102D3000021229E55182021229E58C82021229E54C
:102D4000E282021229E54A83021229E5CE830212A9
:102D500029E5E783021229E50C84021229E54A8459
:102D6000021229E59984021229E5C284021229E59A
:102D70001185021229E5BD85021229E58586021218
:102D800029E5EA86021229E5B787021229E5FD87BF
:102D9000021229E51988021229E54B88021229E559
:102DA000F389021229E5CA8A021229E5F68A02127B
:102DB00029E52C8B021229E54D8B021229E55C8B4B
:102DC000021229E5678B021229E51B8C021229E504
:102DD0008E8C021229E5008D021229E5088D02125F
:102DE00029E5838D021229E5DC8D021229E51F8E6B
:102DF000021229E5B190021229E5F791021229E5A4
:102E00008794021229E56F95021229E5A295021214
:102E100029E56496021229E51397021229E55B97CA
:102E2000021229E5BD97021229E5E297021229E56F
:102E3000F397021229E56B98021229E5F398021222
:102E400029E55799021229E53C9A021229E5619A6F
:102E5000021229E5829B021229E5A09B021229E5B4
:102E6000B39B021229E5269C021229E5359C021229
:102E700029E5BD9C021229E50B9D021229E5149D4E
:102E8000021229E5149F021229E568A0021229E521
:102E900078A0021229E594A1021229E50DA20212DE
:102EA00029E543A3021229E585A3021229E5C1A35E
:102EB000021229E595A5021229E5FAA7021229E5D1
:102EC0000EA8021229E518A8021229E522A802126A
:102ED00029E52CA8021229E536A8021229E54FA8F7
:102EE000021229E559A8021229E563A8021229E570
:102EF0006DA8021229E59CA8021229E5C4A80212B5
:102F000029E5CFA8021229E519A9021229E523A96A
:102F1000021229E52EA9021229E552A9021229E579
:102F200076A9021229E5D7A9021229E522AA0212DE
:102F300029E53EAA021229E5A8AA021229E5F4AA67
:102F4000021229E53CAB021229E5B7AB021229E5D2
:102F500051AC021229E515AE021229E583AE021228
:102F600029E5B5AF021229E5DBAF021229E54BB125
:102F7000021229E5FFB4021229E5FFB6021229E583
:102F8000D7B8021229E570B9021229E582BB0212F4
:102F900029E544BC021229E590BC021229E5F6BCE1
:102FA000021229E508BD021229E558BF021229E5DF
:102FB00047C0021229E586C1021229E5D8C10212D2
:102FC00029E57DC2021229E538C4021229E569C546
:102FD000021229E587C5021229E5DCC5021229E59E
:102FE000DAC6021229E502C7021229E565C70212F4
:102FF00029E566C8021229E5D9C8021229E507CADF
:10300000021229E572CA021229E562CB021229E5F1
:10301000C8CD021229E5F6CD021229E5F1CE021241
:1030200029E58FD0021229E5DFD0021229E597D1D8
:10303000021229E54CD2021229E5B0D2021229E58A
:1030400069D3021229E509D4021229E56DD40212CE
:1030500029E5B7D4021229E5F4D4021229E55CD699
:10306000021229E50181011229E54381011229E5B6
:103070003E84011229E59184011229E5D7840112C9
:1030800029E51886011229E57D86011229E5BD860C
:10309000011229E50088011229E5428B011229E578
:1030A0006B8C011229E5AC97011229E54C980112AD
:1030B00029E53F9B011229E5769C011229E5EC9C4C
:1030C000011229E5169E011229E5669F011229E5E4
:1030D0004DA0011229E5B6A2011229E5C4A40112EE
:1030E00029E555A5011229E529A6011229E5B5A66C
:1030F000011229E5BFA6011229E5E7A6011229E57B
:1031000094A7011229E57FA8011229E552A901120D
:1031100029E5DFA9011229E5F5A9011229E559AA36
:10312000011229E582AA011229E5AFAA011229E5B7
:10313000F4AC011229E5CFAD011229E513AE01125D
:1031400029E584AE011229E53DAF011229E56FAFF3
:10315000011229E5B6AF011229E5E9AF011229E50F
:103160004EB0011229E59DB0011229E5A2B001126D
:1031700029E5F6B0011229E540B1011229E53CB27A
:10318000011229E5A1B2011229E5FFB2011229E5D8
:1031900049B6011229E51DB7011229E5AAB80112A5
:1031A00029E584BB011229E537BC011229E55EBE81
:1031B000011229E503BF011229E541BF011229E5EA
:1031C00011C1011229E524C1011229E52DC1011205
:1031D00029E536C1011229E54BC1011229E56AC171
:1031E000011229E59FC3011229E5F2C3011229E565
:1031F000FCC3011229E506C4011229E561C40112CC
:1032000029E5BDC4011229E5D5C5011229E536C657
:10321000011229E585C7011229E5CEC7011229E56A
:10322000A6C8011229E5D1C9011229E587CA0112F0
:1032300029E589CB011229E58BCC011229E570CD56
:10324000011229E587CD011229E5C4CD011229E536
:10325000CECD011229E5D8CD011229E5E3CD011229
:1032600029E501CE011229E543CE011229E5A1CEBF
:10327000011229E5C6CE011229E5E0CE011229E5A9
:103280006DCF011229E5A6CF011229E5F6D0011272
:1032900029E54DD1011229E567D2011229E59DD218
:1032A000011229E539D3011229E5B5D3011229E527
:1032B00025D5011229E540D6011229E506D70112CC
:1032C00029E5B0D7011229E535D8011229E59DD8A5
:1032D000011229E552D9011229E5A4D9011229E5E3
:1032E00019DA011229E5E2DA011229E505DB0112FA
:1032F00029E5C9DB011229E5EDDB011229E50FDC27
:10330000011229E570DC011229E5BBDE011229E575
:1033100096DF011229E540E0011229E581E2011260
:1033200029E5CFE2011229E512E3011229E56AE35A
:10333000011229E5C8E3011229E5F2E3011229E5AA
:1033400016E4011229E547E4011229E571E40112AE
:1033500029E5B8E4011229E516E5011229E572E52F
:10336000011229E573E6011229E5DDE7011229E5DD
:103370001BE8011229E544E8011229E5D5E801120C
:1033800029E51FE9011229E543E9011229E599E937
:10339000011229E5B4E9011229E56FEA011229E5D4
:1033A00099EA011229E5EFEA011229E5F4ED01128B
:1033B00029E527EE011229E5E4EE011229E5BFEF28
:1033C000011229E54FF0011229E590F0011229E5DB
:1033D00083F3051229E5C2F3051229E544BD031262
:1033E00029E5EDBD031229E5CCBE031229E5E7BFAF
:1033F000031229E507C0031229E529C1031229E5B3
:10340000C6C2031229E533C3031229E509C4031216
:1034100029E50FC5031229E574C5031229E5B0C5D6
:10342000031229E509C6031229E542C6031229E55C
:103430008BC6031229E51DC7031229E5BAC703127B
:1034400029E58FC8031229E55CC9031229E5E9C9FA
:10345000031229E50FCA031229E53CCA031229E524
:103460006DCA031229E542CB031229E552CB0312A0
:1034700029E5A5CB031229E5B2CB031229E5BFCB81
:10348000031229E5C8CB031229E52CCC031229E548
:103490008ACC031229E5D5CC031229E5F0CC03121E
:1034A00029E517CD031229E534CD031229E540CDD6
:1034B000031229E5E4CE031229E5FDCE031229E526
:1034C00079CF031229E58CCF031229E59CCF031293
:1034D00029E542D0031229E5B2D1031229E5C5D26C
:1034E000031229E565D3031229E56FD3031229E5F9
:1034F000DDD3031229E5EED3031229E52DD40312FF
:1035000029E55BD4031229E528D5031229E57FD5E7
:10351000031229E5C4D5031229E51AD6031229E5B9
:1035200038D6031229E586D6031229E554D70312AB
:1035300029E5A2D7031229E5E4D7031229E567D8C4
:10354000031229E591D8031229E5C7D8031229E50A
:10355000D6D8031229E534D9031229E5ACD90312D0
:1035600029E5EDD9031229E53CDA031229E567DAEA
:10357000031229E581DA031229E59BDA031229E512
:1035800070DB031229E57ADB031229E5B5DB0312B0
:1035900029E5C5DB031229E5CEDB031229E51FDC93
:1035A000031229E533DC031229E551DD031229E575
:1035B00064DD031229E57BDD031229E590DD0312AA
:1035C00029E52ADE031229E5A9DE031229E54CDFED
:1035D000031229E557DF031229E5A4E0031229E5C8
:1035E000C0E0031229E518E1031229E586E1031280
:1035F00029E5D2E1031229E5ECE1031229E54CE2C9
:10360000031229E5EAE2031229E535E3031229E56D
:1036100098E5031229E530E6031229E5A7E603122F
:1036200029E5EDE8031229E505E9031229E508E992
:10363000031229E514E9031229E528E9031229E513
:1036400030E9031229E567E9031229E55BEA031271
:1036500029E5E5EA031229E567EB031229E5DCEB2E
:10366000031229E5B4EC031229E5D6EC031229E58F
:103670006DED031229E579ED031229E5D6ED03126C
:1036800029E5D9ED031229E506EE031229E51BEE23
:10369000031229E58AEE031229E5D6EF031229E584
:1036A000E9F0031229E574F1031229E587F2031208
:1036B00029E551F3031229E582F3031229E5A8F362
:1036C000031229E5B1F3031229E5E0F3031229E51A
:1036D00090F4031229E540F5031229E5B3F503122E
:1036E00029E565F6031229E5D8F6031229E517F74F
:1036F000031229E560F7031229E595F7031229E57E
:103700003DF0041229E5A8F0041229E5EFF00412B7
:1037100029E565F1041229E5B5F1041229E539F22C
:10372000041229E57DF4041229E5A8F6041229E51E
:1037300085FA041229E502FB041229E53DFB041277
:1037400029E55BFB041229E5BBFB041229E5E3FB39
:10375000041229E513FC041229E544FC041229E5AE
:1037600071FC041229E5CAFC041229E515FD0412B6
:1037700029E5E8D5041229E564D6041229E58AD69C
:10378000041229E5C1D6041229E51AD8041229E544
:1037900036D8041229E57BD8041229E50BD9041286
:1037A00029E563D9041229E538DA041229E516DB84
:1037B000041229E560DB041229E5C1DB041229E5C6
:1037C00045DC041229E56EDC041229E5AFDC0412A5
:1037D00029E55DDE041229E52DDF041229E5F4DF79
:1037E000041229E5C7E0041229E501E1041229E5E4
:1037F00059E1041229E57BE1041229E50FE20412E4
:1038000029E5C2E2041229E546C6051229E5ABC640
:10381000051229E552C7051229E58AC7051229E5CF
:10382000D9C7041229E584C8041229E521CA041263
:1038300029E59DCA041229E5D5CA041229E5C0CD9F
:10384000041229E552CF041229E5BCCF041229E560
:10385000F4D2041229E595D4041229E507EA0512E9
:1038600029E52FEA051229E51BEB051229E5A49E9F
:10387000051229E5279F051229E53E9F051229E536
:10388000B19F051229E517A0051229E540A00512F0
:1038900029E5C5A0051229E567A1051229E5CAA1F8
:1038A000051229E52FA2051229E54FA2051229E5E7
:1038B0007FA2051229E59BA2051229E5CAA20512DD
:1038C00029E5FAA2051229E530A3051229E590A3FE
:1038D000051229E516E3041229E5E6E3041229E5B9
:1038E0000BE4041229E52BE4041229E53FE4041259
:1038F00029E5A7E4041229E5CBE4041229E549E609
:10390000041229E56FE7041229E550E8041229E5BD
:10391000B4E8041229E5E0E8041229E564E9041298
:1039200029E5B5E9041229E5D6E9041229E54EEAAC
:10393000041229E5F2EB041229E555EC041229E5FD
:10394000E5ED041229E5B2EE041229E5EDEE0412CC
:1039500029E512EF041229E532EF041229E558EFA8
:10396000041229E56CEF041229E5D5EF041229E5CC
:1039700029F0041229E536DD051229E540DD05129E
:1039800029E561DD051229E551F1011229E55FF410
:10399000011229E58CF5011229E567F7011229E5E5
:1039A000F1F7011229E5AAF8011229E5D3F801126D
:1039B00029E51DF9011229E5D8F9011229E54BFA8B
:1039C000011229E54EFA011229E551FA011229E501
:1039D0008FA6031229E574FA011229E577FA01127C
:1039E00029E590FA011229E5F4FA011229E5E6FB2E
:1039F000011229E51BFD011229E568FD011229E5E7
:103A00006FFE011229E541FF011229E5CFD602120E
:103A100029E507D7021229E56ADB021229E53CDC19
:103A2000021229E5C3DC021229E5F4DC021229E5C1
:103A300022B2031229E576DD021229E5A4DD021285
:103A400029E5C5DE021229E5F3DE021229E521DFB0
:103A5000021229E557DF021229E504E0021229E5E6
:103A60002AE0021229E589E0021229E503E20212A6
:103A700029E59DE2021229E58EE3021229E56BE4B5
:103A8000021229E5B5E4021229E504E5021229E54E
:103A900070E5021229E5D8E5021229E525E60212B1
:103AA00029E595E6021229E5A6E7021229E59AE83A
:103AB000021229E54BE9021229E580E9021229E503
:103AC000D5E9021229E580EA021229E5AEEA0212DE
:103AD00029E533EC021229E5B8EC021229E5F8ECED
:103AE000021229E537ED021229E550ED021229E50F
:103AF000FFED021229E5B7EE021229E55EEF021290
:103B000029E5F2EF021229E598F0021229E502F107
:103B1000021229E58DF1021229E520F2021229E5AF
:103B20003EF2021229E511F3021229E5CFF3021247
:103B300029E585F4021229E523F5021229E5BB9255
:103B4000051229E5FC92051229E56593051229E580
:103B50008693051229E59F93051229E559940512CC
:103B600029E56294051229E5B394051229E5DC9450
:103B7000051229E5F394051229E55795051229E563
:103B8000E995051229E51A96051229E5769605129A
:103B900029E5DC96051229E51097051229E583979A
:103BA000051229E5C597051229E50598051229E5AD
:103BB0003D98051229E54F98051229E561980512EF
:103BC00029E59298051229E5D298051229E5F2AE69
:103BD000051229E535B0051229E55BB0051229E586
:103BE0006CB0051229E584B2051229E5A3B20512CD
:103BF00029E583DF051229E5B9DF051229E504E08F
:103C0000051229E550E1051229E5ADB3041229E5B5
:103C1000EBB4041229E527B5041229E5ECB6041229
:103C200029E516B7041229E59CB9041229E5DCB987
:103C3000041229E571BB041229E506BC041229E52A
:103C400064BC041229E5F5BC041229E52DBD04125B
:103C500029E56FBD041229E5E9BE041229E572C009
:103C6000041229E5A8C2041229E5D6C2041229E5E6
:103C700002C3041229E50BC3041229E561C304122F
:103C800029E5F1C3041229E5F8C6041229E57CC729
:103C9000041229E586F2051229E59CF2051229E5B0
:103CA000A6F2051229E5F6F2051229E5CABD0512AC
:103CB00029E5E3BD051229E588BE051229E5C8BE40
:103CC000051229E5E1BE051229E515BF051229E512
:103CD00062BF051229E596BF051229E5D8BF051276
:103CE00029E5AEC1051229E519C2051229E584ECC2
:103CF000051229E5D9EC051229E532ED051229E571
:103D000037F1051229E58AF1051229E5CCF10512F2
:103D100029E5DCF1051229E5069A041229E55E9AE7
:103D2000041229E5729B041229E53F9C041229E53F
:103D3000549C041229E59E9C041229E50C9D041252
:103D400029E51F9D041229E5639D041229E5D29DF2
:103D5000041229E52EA0041229E534A1041229E554
:103D60008FA1041229E580A3041229E501A40412FD
:103D700029E53AA4041229E585A4041229E59BA4A7
:103D8000041229E5A8A4041229E5E1A4041229E5F6
:103D9000F3A4041229E5D1A5041229E5DCA5041237
:103DA00029E561A6041229E5B9A6041229E505A7AB
:103DB000041229E53EA8041229E566A8041229E5A3
:103DC000DEAA041229E506AB041229E51FAC041291
:103DD00029E54EAC041229E5C0AC041229E5CCACAF
:103DE000041229E500AD041229E570AD041229E59D
:103DF0004DAE041229E586AE041229E590AE0412F8
:103E000029E593AE041229E59DAE041229E5B9AE69
:103E1000041229E535AF041229E56EAF041229E535
:103E20008AAF041229E5B6AF041229E5F1AF0412F6
:103E300029E50CB0041229E516B0041229E545B0B5
:103E4000041229E55BB0041229E577B0041229E5D4
:103E5000A6B0041229E5C6B0041229E50FB1041278
:103E600029E558B1041229E562B2041229E5037F5D
:103E7000001229E5147F001229E59D7F001229E533
:103E8000FDF7031229E54CF8031229E50AFA03129B
:103E900029E5DDFB031229E51BFC031229E5F1FCF2
:103EA000031229E5F6FD031229E518FE031229E5A0
:103EB00074FE031229E5F5FE031229E5054E0012F2
:103EC00029E5274E001229E5794F001229E5C24F56
:103ED000001229E53B50001229E5B650001229E5F1
:103EE0001F51001229E56651001229E5D851001230
:103EF00029E57952001229E5F852001229E53453D8
:103F0000001229E58857001229E59659001229E583
:103F1000C959001229E50E5A001229E5185B001252
:103F200029E5015E001229E5975E001229E563602C
:103F3000001229E59661001229E5AC62001229E51C
:103F40002063001229E5EC63001229E56064001289
:103F500029E56364001229E51A65001229E55F6608
:103F6000001229E5A368001229E53D6B001229E53E
:103F70001B6C001229E5586D001229E59D70001296
:103F800029E5AD70001229E5E471001229E595726A
:103F9000001229E5E173001229E54F74001229E5AA
:103FA0008275001229E5D775001229E500800412F8
:103FB00029E5A780041229E51981041229E5298140
:103FC000041229E5AB81041229E50282041229E5D5
:103FD000F782041229E51E83041229E5C383041223
:103FE00029E51284041229E57084041229E5CB84A2
:103FF000041229E5A687041229E55F88041229E541
:10400000C488041229E5578A041229E5F78A0412A4
:1040100029E5908B041229E5ED8B041229E5638CC8
:10402000041229E55F8D041229E5528E041229E558
:10403000AB8E041229E5C18E041229E5E28E04122A
:1040400029E5218F041229E5B18F041229E5F490A6
:10405000041229E5B192041229E5FB93041229E523
:104060003595041229E54096041229E5E0960412DC
:1040700029E54F97041229E56C98041229E5008080
:10408000051229E56B80051229E5B380051229E5A3
:104090001A81051229E57681051229E5B1810512FB
:1040A00029E54D82051229E5A782051229E5138429
:1040B000051229E59A84051229E5D384051229E51C
:1040C0000285051229E57C85051229E5C4850512BE
:1040D00029E5EA85051229E54187051229E5468784
:1040E000051229E5BD87051229E52988051229E56C
:1040F0002489051229E5118A051229E5CCA90512A2
:1041000029E509AA051229E5A2AA051229E5ADAB00
:10411000051229E5F5AD051229E571AE051229E56F
:10412000CBD4051229E57CD5051229E544D6051224
:1041300029E599D6051229E51CD7051229E53CE4A5
:10414000051229E525FF031229E536FF031229E5AB
:10415000D6FF031229E5EFFF011229E5EAFF02125B
:1041600029E5BDEF051229E5CDEF051229E5E2EFBE
:10417000051229E573F0051229E5B9EE051229E5C6
:104180003EEF051229E5A4EF051229E5F9FF01121A
:1041900029E521F4051229E531F4051229E534F465
:1041A000051229E537F4051229E5F87F001229E503
:1041B000B3E1051229E5D5E1051229E543E305122E
:1041C00029E5C7E3051229E5F8F3051229E501F40D
:1041D000051229E50AF4051229E518F4051229E566
:1041E000FB98051229E56799051229E52F9A051212
:1041F00029E5289B051229E5159D051229E56F9DE6
:10420000051229E5C29D051229E5D39D051229E570
:10421000E59D051229E5519E051229E5659E0512C9
:1042200029E5709E051229E57E9E051229E5909EDE
:10423000051229E544A4051229E570A4051229E513
:1042400017A7051229E56CA7051229E5A8A70512ED
:1042500029E5BCA7051229E5D5A7051229E5C8A8B7
:10426000051229E5A4A9051229E5B8A9051229E531
:1042700037E7051229E55BE7051229E574E7051222
:1042800029E5B3E7051229E5E6E7051229E516E871
:10429000051229E520E8051229E588E8051229E537
:1042A0008BE8051229E595E8051229E5A2E8051233
:1042B00029E556FD041229E57EFD041229E5BFFD1E
:1042C000041229E5DDFD041229E5F8FD041229E5B3
:1042D00060FE041229E56CFE041229E5CBFE0412EF
:1042E00029E5EFFE041229E5B0FF041229E5BDFF20
:1042F000041229E5CEFF041229E56BFF021229E51D
:1043000083FF021229E5A9FF021229E53BB4051239
:1043100029E584B5051229E58AB5051229E5A1B577
:10432000051229E5C2B5051229E5D8B5051229E51A
:10433000ECB5051229E56BB6051229E5D0B60512D4
:1043400029E558B7051229E5D1B7051229E5AAB81C
:10435000051229E5BAB8051229E5C9B8051229E5FB
:10436000EDF1051229E511F2051229E539F20512E0
:1043700029E561F2051229E579DA051229E5E5DA80
:10438000051229E504DB051229E56ADB051229E59A
:10439000B0D7051229E5C9D7051229E5E0D70512DE
:1043A00029E5E9D7051229E507D8051229E511D82D
:1043B000051229E51BD8051229E52ED8051229E595
:1043C000BBD8051229E52AD9051229E558D90512C5
:1043D00029E5A9D9051229E5F5D9051229E510DA4B
:1043E000051229E51ADA051229E52BDA051229E565
:1043F0006EDA051229E52CF3051229E577F305128B
:1044000029E5E8F5021229E514F6021229E532F64B
:10441000021229E545F6021229E560F6021229E5A5
:10442000BFF6021229E5EDF6021229E5F9FA0212A9
:1044300029E53BFC021229E56DFC021229E5D8FCB6
:10444000021229E55CFE021229E584FE021229E52A
:1044500099FE021229E5A9FE021229E5E9FE0212DF
:1044600029E52BFF021229E53BFF021229E54CEB5F
:10447000051229E55CEB051229E57AEB051229E521
:1044800095EB051229E5BCEB051229E5DDEB0512DC
:1044900029E5F7EB051229E52FEC051229E552EC89
:1044A000051229E583F0051229E5C9F0051229E571
:1044B0000CCE051229E51CCE051229E53ACF0512CE
:1044C00029E56CCF051229E58ECF051229E5B6CF77
:1044D000051229E5CFCF051229E50BD0051229E5F4
:1044E00074D0051229E5B0D0051229E5F7D00512E0
:1044F00029E524D1051229E550D1051229E5AAE5BF
:10450000051229E5E1E5051229E507E7051229E588
:104510000AE7051229E5A6ED051229E518EE0512B0
:1045200029E556EE051229E597EE051229E5B28A2E
:10453000051229E5B88A051229E5FF8A051229E541
:104540000B8D051229E53B8D051229E5A58D051278
:1045500029E5608E051229E5A78E051229E5DA8E78
:10456000051229E5648F051229E57B8F051229E5DF
:10457000888F051229E5928F051229E532910512DF
:1045800029E52492051229E58292051229E586760D
:10459000001229E59C76001229E54E77001229E5E4
:1045A0007878001229E56D79001229E5047A001265
:1045B00029E53F7A001229E5B17A001229E50F7B3F
:1045C000001229E51F7B001229E5467B001229E530
:1045D000987B001229E5077D001229E50C7D001269
:1045E00029E52E7D001229E526C2051229E544C2DF
:1045F000051229E588C2051229E5AEC2051229E592
:10460000D0C2051229E5E8C2051229E500C305124A
:1046100029E518C3051229E5BEC3051229E500C422
:10462000051229E50AC4051229E51FC4051229E56A
:1046300026C5051229E541C5051229E54AC5051219
:1046400029E553C5051229E55CC5051229E566C5AE
:10465000051229E5E3C5051229E5FAB8051229E591
:104660003FBD051229E55BBD051229E560BD0512B8
:1046700029E544CA051229E55ACA051229E5F8CBED
:10468000051229E543CC051229E5ADCC051229E533
:10469000ACCD051229E5DBCD051229E5EDCD0512DE
:1046A00029E5ACE8051229E5A4D1051229E500D2D7
:1046B000051229E540D2051229E542D3051229E564
:1046C0005AD3051229E56FD3051229E59BD30512AC
:1046D00029E5D2D3051229E5E2D3051229E5F8D35D
:1046E000051229E51DD4051229E5A8D4051229E5EE
:1046F000CCF3051229E550A4031229E5EFA3031218
:1047000029E596A3031229E51DA3031229E5F3A2C7
:10471000031229E5E8A0031229E5B8A0031229E550
:104720007CA0031229E568A0031229E5D49F031297
:1047300029E5F29E031229E5249E031229E5D39B65
:10474000031229E5A89B031229E5499B031229E5D9
:10475000BA99031229E54899031229E545990312EC
:1047600029E58D97031229E54497031229E51E9741
:10477000031229E55A96031229E5A494031229E5A8
:10478000D9B1031229E592B1031229E5DCB0031275
:1047900029E550B0031229E541B0031229E52EADF9
:1047A000031229E57BAA031229E54494031229E5A3
:1047B0001594031229E51294031229E5FD930312BF
:1047C00029E542A9031229E5BD93031229E5A49323
:1047D000031229E5AE92031229E56D92031229E531
:1047E00022DD021229E5FA91031229E563A80312DA
:1047F00029E5C791031229E56C91031229E53B9144
:10480000031229E5048E031229E5168D031229E50A
:10481000D08B031229E57E8B031229E5728B0312DC
:1048200029E5D98A031229E5A789031229E5F88623
:10483000031229E59B84031229E54F84031229E51D
:104840003483031229E5C982031229E5F381031297
:1048500029E5AF81031229E50080031229E56B8069
:10486000031229E53280031229E554FA0100000001
:1048700080FBE4738F000100030987000100020937
:10488000240002002A15250002002C152600020033
:104890002E152700020030152800010032152900CE
:1048A000010033158400040034158600010038151A
:1048B0002A00010039152B0001003A152C000100D7
:1048C0003D152D000800EA082E0001003E152F00BE
:1048D00001003F1530000100401531000100411575
:1048E00032000100F20833000100F3083400010037
:1048F000421536000100F408380001004315390064
:1049000001003C1583000200551563000100FF08FB
:1049100064000100E108650001003B156D00010025
:10492000000971000800E208660001005415430008
:1049300001004515440002004615450001004815D8
:1049400046000200491547000800F708480001002A
:104950004B154B0001004C15040001005715A10038
:10496000010059153700010058158800010004099D
:104970003C000100F5083D0001004415490002001B
:104980004D156700010001094D0002004F154E0052
:10499000010051154F00020052153E000100F608BB
:1049A0000000000000000001363601010001020194
:1049B00000010301000104010606050200000701D1
:1049C00000340801000F090401010D0100FF0E0869
:1049D000000017020000190100FF1A0100011B016D
:1049E00000FE1C0100081D0200001F010001200143
:1049F0000001210200002301000F24020000260113
:104A0000000127010008280200FF2A0100072B01EE
:104A100002402C0100002D0100012E0100012F0198
:104A200000FF30010B1C310800003A0100083B0177
:104A3000000F3C0100013D0100FF3E040000420464
:104A40000000460400004A0400004E040000520426
:104A50000000560400005A0400005E20FFFF3600EC
:104A60000100060000000F00000000000000000030
:104A70000000000003FFFF00000403FFFF0000FF31
:104A8000FF0FF4010005C4040320000100000B0027
:104A90000000000000000003010F00000000000003
:104AA0000000000000000000000000000000000006
:104AB00000000000000000000000000000000000F6
:104AC00000000000000000000000000000000000E6
:104AD000000000000000000000000000010371035E
:104AE0000103010301030103010322030203010384
:104AF000100300030003000300030003000300038E
:104B0000420300032403060300030003040312030B
:104B100025032303250323030403040300030003E5
:104B20000003440300030003230300036503210083
:104B300035038103000305030003000300030003A2
:104B40002503230303007100300160001100700091
:104B500031022003500480001000610000001400A6
:104B6000630073007200620043000000130006003F
:104B7000000000000400120000000000000000001F
:104B800004000400370037003C024400000000002D
:104B900000000000650000003500810000000500F5
:104BA00000008300000001017101010101011101F8
:104BB00001013101010101018001100161013B008E
:104BC00014006301730172016201430100011301CA
:104BD00006013D0135000401120100010001000140
:104BE000000104010401330133013C01440132019D
:104BF000360000010001650100013500810100015E
:104C0000050182018301000103027102300160028B
:104C1000110270020102020202028002100261020D
:104C20003A00410063027302720262024302000210
:104C30001302380000020002040212020002000205
:104C40000002000204020402370037003C02440262
:104C500000023900000200026502000235028102F2
:104C600000020502820283020002030471040204AE
:104C7000600411047004020402040104020410041C
:104C800061040004140463047304720462044304A2
:104C900000041304060400040004040412040004C5
:104CA0000004000400045104640000040004000433
:104CB00044040004000400040004650400043504F6
:104CC0008104640005040004830400040000EB3F39
:104CD00013005B3F0100EB3F0200DD3E0300E33EBB
:104CE0000400E93E0500EF3E0600FB3E30001F3F9A
:104CF0003100193F32002B3F3300313F3500373F41
:104D000034003D3F3600433F11004F3F1400553FF4
:104D100015000D3F1F00133FFFFF000001A93006E3
:104D2000DF3008D9300BF7301013300A093102AFE9
:104D30003005CD3007B5300C91300D9D30641B2E01
:104D4000FF000007ECFDFDFDECDCDCCCBCACAC9C5A
:104D50009C8C7C7C6C6C5C5C5C4C4C3C3C2C2C1CC3
:104D60001C03EAF5E5D5D5C5B5A595958585757579
:104D70006565555545453535252515150500160F2D
:104D800000000B150B020002220F3300000E0C0E68
:104D9000020B040B0A0708000F000119161816165B
:104DA0001823030000034A49434E181A2505023010
:104DB0003017181921301B1D1F30303016181920DC
:104DC000231A1C1E3000393D3F373C3C362C442D05
:104DD00002040201010101090200BE040A3C003C78
:104DE000007F00E803000000000E00280C08100CF3
:104DF000030303080900040001FF1E1E0C0505083B
:104E0000040415100AC082C083900816E4F0A3F0D1
:104E10007CD57D047A897B07124525122E21124804
:104E200055122E27026BBE74F312242A74F5122A2F
:104E3000C489098A088B0AE9705F74026508703EAC
:104E40009007A87408F0750C00780C122A06ECF58F
:104E50000C780C122A06EBF50C780C122A06901529
:104E60003412283D901538E0F97CF77D08901555EF
:104E7000126BCF122E4B7407122A30024F39740175
:104E800065086003024F3C9007A87408F07B00AAF5
:104E90000AA90A122E87024F397401650960097444
:104EA0000265096003024F3CEA60067403650870FE
:104EB000409007A87402124F5D122C80122E399078
:104EC00007AEE0A2E34010E9700D90081AE004F08C
:104ED00064047003124F6774036508705C90081BCC
:104EE000E0F8740128F0E8C39405404D124F678044
:104EF00048740165087045740165099007A8702E13
:104F0000740AF07401122CAFE4F07402122CAF7426
:104F100003F004122CAFE4F0A3F0A3F0A3F07408A4
:104F2000122CAFE4F0AA18AB191230BB8025740A1A
:104F3000124F5D122C80122E6FE960179080A01224
:104F4000283D7A017B009007A5E0F9123CC174046A
:104F5000122A30740B122A307F050226B9F0901500
:104F600038E0F990153422901534E4F0A374F8F089
:104F7000A374FFF0A37407F02274F612242AE9FF49
:104F8000EAFE7AD1F9123B7D8A828B83E5824583E2
:104F9000702A7A027B00123B5FEA4B700E7A107B1C
:104FA000009007A5E0F9123BA180148A828B8374DC
:104FB000D1F0EFA3F0EEF9123B6B8003EFA3F00208
:104FC00051D374F712242A8908900702127289FFBC
:104FD000901526E0F47003A3E0F47036900719E012
:104FE000901526F0A3E4F080298E828F83A3A3126C
:104FF000645260168E828F83A3A3A3E0F583888218
:10500000A3126452FAA908123EC58E828F831275CC
:10501000B6FFEE4F70D3901526E0F47003A3E0F4D2
:10502000600A901526E0FAA908123EC51231C39015
:1050300007731257391231BD0273C574F112242A55
:10504000890A8C08750900750B00740F122CAF12B9
:1050500060507411122CAF1257608049AE0E12517D
:1050600007F50CA3E0F50DAE0BEE2EFEE433FFEAE0
:105070002EF582EB126445650C7004A3E0650D709B
:1050800019AE09EE2EFEE433FFEC2EF582ED3FF56E
:1050900083E50CF0A3E50DF00509050EE50EC395BB
:1050A0000840B9050BE50BC3950A5005750E008045
:1050B000EBA909026AE474F412242A890B7D0074B6
:1050C0000C122CAF12605080010DEDC3950B5032C5
:1050D000750A008002050AE50AC39C50ECED25E044
:1050E000FEE433FFEA2EF582EB3F125117F509AECD
:1050F0000A12510765087004A3E0650970D77901A9
:105100008002790002688BEE2EFEE433FFE82EF574
:1051100082E93FF583E022F583E0F508A3E02274FD
:10512000F612242A1251BA7003A3E06D70177508A5
:10513000AC7509077808122A02EEFA123FF17402E0
:10514000122A30801F7508027509807808122A0219
:105150008C088D097808122A021251AD124015747C
:1051600004122A30806D74F612242A1251BA700388
:10517000A3E06D70177508B97509077808122A023F
:10518000EEFA123FF77402122A30801F7508037579
:1051900009807808122A028C088D097808122A02E0
:1051A0001251AD1240157404122A308026125B048D
:1051B000F583E0FD7C801264FE22EAFEEBFF1273B1
:1051C000CA1275C7FCE439FD900773E06C227402C3
:1051D000122A307F020226B974F612242A74FE12B3
:1051E0002AC4EAFEEBFF851882851983E4F0A31236
:1051F0005990126648FBECFA88828983A3A3E0F9F0
:10520000750900750800600574FF697005750882EE
:10521000803D900773E06A7003A3E06B701AAA18D0
:10522000AB1912373FE9F509851882851983126891
:1052300096701C7508838017900902E06004640171
:1052400070057508818008E0640270037508808528
:105250001882851983125760A908EEFAEFFB123FF6
:10526000FDE509601185188285198312689660062C
:10527000126BC9123C010251CE74F212242AEAFECA
:10528000EBFF750A00750B001252EB1231C3EA6591
:10529000087003EB65097012123751E914F50A79A9
:1052A000017AE27B071237578003750B8012643F47
:1052B000F50C780C122A06750CE2750D07780C12A5
:1052C0002A02780A122A067808122A02E50BF50843
:1052D0007808122A06126315126442F97A057B8057
:1052E0001240037407122A3002605E1273CA1275EC
:1052F000C7F508E439F5092274F612242AE9FE7F7D
:105300000080298A828B83125119F8E4C8F9E508D4
:1053100028E439F509EF25E0F8E433F9EC28F582C3
:10532000ED125B0DEA2402FA50010B0FEFC39E4011
:10533000D20251D374E812242A74FB122AC48A16AA
:105340008B17851882851983E4F07403122CAFE45F
:10535000F0A3F004122CAFE4F0A3F0125E86351730
:10536000125962F50B850A82F5831275C3FEE43982
:10537000FF850A82850B83A3A3E0FA850A82850B49
:1053800083A3A3A3E0F9EAF508E439F509E50A24C3
:1053900004F50A5002050BEEFAEFFB12325FE964E6
:1053A000016016EEFAEFFB12325FE9703D90077371
:1053B000E06E7003A3E06F6031126650122A06E4BB
:1053C000F508F5097808122A027808122A069007CB
:1053D000731228417508807808122A0612573F1266
:1053E00040037407122A3002572F12576688106044
:1053F0002B1271C8123BFB7403122CAF1257397475
:1054000003122CAF12689660137403122CAF12575C
:1054100058A910123EF58A0A8B0B800375100012F2
:105420005766880F60271271C8123BFB7401122C5B
:10543000AF1257397401122CAF126896600F7401C5
:10544000122CAF125758A90F123EF58003750F00AA
:10545000900702805D850A82850B83A3A3A3A3A383
:10546000A3A3A3E4F0A3F0AA0AAB0B8514828515CD
:1054700083A3A3125776126452F9123B6B851282F2
:10548000851383E0C0E0851882851983E0F874E213
:1054900028F582E43407F583D0E012689A04F0E539
:1054A00011A2E05007AA12AB13123C0185148285A9
:1054B0001583E0F514A3E0F515E514451570030216
:1054C000569C851482851583A3A312645260DD85E2
:1054D0001482851583A3A3A3A3A3A3A3A3E0A2E09F
:1054E00050CA851482851583A3A3A3A31268968549
:1054F0001482851583A3A3601F126452FA79018573
:105500001482851583A3A3A3A31264571248728A39
:10551000128B13751101800F125776A3A3E0F512B9
:10552000A3E0F513751100E5124513700302549FB3
:10553000851282851383A3E065087004A3E06509E2
:10554000600F74FF6508700474FF650960030254FE
:105550009F851282851383A3A3A3A3A3A3A31228C9
:1055600041851282851383A3A3A3A3A3A3E0FC74A4
:1055700005122CAF126BCFA910123ED77402122A5B
:1055800030E9703C851282851383A3A3A3A3A3A350
:10559000A3A3A3A3122841851282851383A3A3A3E7
:1055A000A3A3A3A3A3A3E0FC7403122CAF126BCF9D
:1055B000A90F123ED77402122A30E9700302549FD9
:1055C000E50F2510C333240AFA7B00123B5F8A0AD9
:1055D0008B0BEA450B700302547D8A828B8374D255
:1055E000F0851682851783A3A31260508A828B836D
:1055F000A3A3E8F0A3E91274CDA3E5101275CFE5DB
:105600000FF0E510603CEA2405FAE4350BFBE50AEF
:10561000240AF8E4350BF98A828B83125E8B7403BB
:10562000122CAF12577B1229FEAC10EC2CFCE43389
:10563000FD8A828B83126BCF123B3B7403122A309C
:10564000800D8A828B83A3A3A3A3A3E4F0A3F0E538
:105650000F7003025455A810E828F8E433F9E50A5E
:1056600028F8E50B39F9E8240AFAE439FB850A82BF
:10567000850B83A3A3A3A3A3A3A3A31257397401E8
:10568000122CAF12577B1229FEAC0FEC2CFCE4332A
:10569000FD123B3B7403122A300254678518828541
:1056A0001983E06027126650122A067508E2750910
:1056B000077808122A027403122CAF126659122AB4
:1056C000069007731228417508008029EEFAEFFB57
:1056D00012325FE9702F126650122A067508E275C1
:1056E00009077808122A027508007808122A06901D
:1056F00007731228417808122A0612573F124003F6
:105700007407122A307403122CAF126896600B745F
:1057100003122CAF126BCF123C017401122CAF128A
:105720006896600B7401122CAF126BCF123C01749F
:1057300005122A307F100226B9EAF0A3EBF022E529
:10574000162402FCE43517FDE5161262A63517F59E
:1057500083E0F97A067B8022125760AA0AAB0B22FB
:10576000E0FCA3E0FD22850A82850B83E0F8A38597
:10577000820A85830B22126457A322E0F50CA3E072
:10578000F50D750E00780C2274F112242A74F412AF
:105790002AC48A088B09ECFEEDFF740B122CAF743F
:1057A00003F0122A861245251231BDEAFCEBFD7486
:1057B00003122A8612451FE9600FEE241312644279
:1057C00064036010E06401600B851882851983749E
:1057D0008402591A8E828F83A3A3A3A3A3A3A3A396
:1057E000E06018F46015EE2413126442640370162E
:1057F000EE24141264426003F4700B85188285193C
:1058000083748202591A127375E064217002A3E056
:1058100060030258F1851882851983748C1259909F
:10582000640360030258DB7401122A8E12602A128C
:1058300047D7E960030258DB123E598A0A8B0BEA0C
:10584000450B700302591B8E0C8F0D750E00780CE2
:105850001229FE7C157D00123B3B7403122A308511
:105860000882850983A3A3E50A2415FCE4350BFD12
:10587000740912295E126FD6C0E0E50A241EF58273
:10588000E4350BF583D0E0125E91C0E0E50A241FF9
:10589000F582E4350BF583D0E0F0E50A2420F582AB
:1058A000E4350BF5837405F0EE240BFE50010FFA7E
:1058B000EFFB1237F97D007C007900EEFAEFFB1266
:1058C0003FBB9080A012283D7A007B109007A5E096
:1058D000F9123CC17404122A308078125958122AE5
:1058E0000612596A1247F57401122A30E9702C80A9
:1058F00014125958122A0612596A1247EF740112EB
:105900002A30E9700D851882851983E4F0123E294A
:1059100080098518828519837488F0126FD6F50A7C
:10592000780A122A067401122A7E880A890B780ADC
:10593000122A02E508240CF582E435091259624462
:1059400080F50B780A122A021263D7123FAF740552
:10595000122A30740C026AE1EE12603DE0F50A781A
:105960000A22F583E0F50AA3E022EE240BFCE43FD3
:10597000FD8E828F83A3A3A3A3A3A3A3A3A3126CCF
:105980000C8E828F83A3A3A3A3A3A3A3A3E0F922D6
:10599000F0127510E022C082C08374F3122AC4850D
:1059A0001882851983E4F004122CAF12573974035E
:1059B000122CAFAA82AB83122D49AA18AB19122D53
:1059C0007F740D122A30026BBE74F612242AEAFE8E
:1059D000EBFF12604A8882898312737DF89007B4C6
:1059E000E058F508A3E059F509E5084509601C7879
:1059F00008122A0290077312284112643FFD7C00AE
:105A00001264FA12400F7404122A300251D374F453
:105A100012242A74FF122AC4EAFEEBFF851882853D
:105A20001983E4F09008F6E06021EE240B12644242
:105A3000640160178E828F83A3A3126050EE241539
:105A4000126442687003A3E0696003025AFF1260A7
:105A50004AE8FAE9FB88828983A3A3A3A3A3A3A3AB
:105A6000A3E0FC88828983A3A3A3A3A3A3A3A31277
:105A70007568EC28F508E439F509EC45096010EC87
:105A80009471E994085008900902E06402700A8554
:105A9000188285198374808038122DBB8A0A8B0B7B
:105AA000A80AA90BE849602188828983A3A3A3A33C
:105AB000E06016C394035011E82412125B0AE82434
:105AC00014125B0A123E2980098518828519837495
:105AD00081F0125B04126657122A067401122A7EA4
:105AE000880889097808122A0275081F75098078C4
:105AF00008122A0212630B123FAF7405122A307487
:105B000001026888EE1273A03F22F582E439F58322
:105B1000E508F0A3E509F02274EA12242A74DB12E6
:105B20002AC48A148B1575120075130012644AF585
:105B30000EAC18AD197A007B00799C122E997A046C
:105B40007900122D91EAF50C851882851983E02AD7
:105B5000F0F8E50EC3984003025D37E0C3950EF5FB
:105B600009C394044003750903E50975F01AA4FA02
:105B7000ABF0123BFB8A128B13EA45137003025DF4
:105B80003A750D00AE12AF13850E08807E125DA22D
:105B9000123B47850A82850B83A3A3A3A3E0702D44
:105BA000850A82850B83126896700C126D19F0EECF
:105BB0002418126D1C8010125DB0F0900564E01482
:105BC000C0E0125D8AD0E0125DDBE48034900564B1
:105BD000E004C0E0125D8AD0E0125DD3C39403EE0E
:105BE0004003025C9E1260397402125DD36401703E
:105BF00003025CABEE2415125DB3F0EE2416125DC9
:105C0000B3F0EE241AFE50010F050DE50DC3950902
:105C10004003025CD6E508C3950C4003025CB485E2
:105C2000080AAA0A7B00122E038A0A8B0B05089029
:105C30000551125DBC124525850A82850B831260D1
:105C400050125D98E8F0A3E9125DED850A82850B9C
:105C500083A3A3A3A3A3A3A3A3A3A3E0C0E0125D74
:105C600080D0E0F07401122CAFE4F0850A82850B3D
:105C7000831260507402122CAF125E8B7401122AD0
:105C800086122D6DE964016003025B8D7404122C91
:105C9000AFAC82AD83125DA8124525025B93125D05
:105CA000B1125DD364036003025BF4EE2415126D40
:105CB0001C025BFAE50CC3950E4005750800801DBB
:105CC000E50EC3950CF5088014125DB0F0EE241AB1
:105CD000FE50010F050DE50DC39509505D740E12C0
:105CE0002A8E85080AAA0A7B007987122E99050850
:105CF0007418122CAF125DBC124525125DA2123B26
:105D000047EE2412F8E43FF9740E122CAF126BCF59
:105D100088828983EAF0A3EB125DDB7403125DEDE8
:105D2000741D122CAFE0C0E0125D80D0E0126B3623
:105D30007097126D198095750900750A00780A121E
:105D40002A067812122A027809122A06E50EF509A7
:105D50007809122A067405122CAFE0FD7C0012624D
:105D60009212404B7405122A30E51245136007AABF
:105D700012AB13123C017425122A307F0E0226B991
:105D8000EE2419F582E43FF58322125D8E22EE2483
:105D900018F582E43FF58322EE2412F582E43FF504
:105DA00083227C087D0079FFEE240AFAE43FFB227F
:105DB000EE2414F582E43FF5837401221260548EC0
:105DC000828F83E8F0A3E9F07C657D05EE1265150E
:105DD0003FFB22127523A3A3A3E022F0EE126D1065
:105DE0007402F0EE2416F582E43FF58322F0EE24EF
:105DF00017F582E43FF5837402F0125D8E74FFF0B4
:105E00002274F612242A74F9122AC48A088B091201
:105E10005E863509127650123B53EAF8EBF9ECFA3C
:105E2000EDFB851882851983122C98EE2404FE5010
:105E3000010F8E828F83E0C0E07404122CAFD0E09B
:105E4000126B0DFA7405122CAF7401F07406122C4B
:105E5000AF7401F090077DF09007860412753AA3A5
:105E600012605090077E125E8BEA900787125E9157
:105E700090077CF0AA18AB19122E3FE96003122E8E
:105E80004574070251D0EA12727C22E8F0A3E9F0CF
:105E900022F01274A7E02274F212242A74FF122A4C
:105EA000C47508007E007F001230EB8A0A8B0B124B
:105EB00030EB8A0C8B0DA80CA90D80080508126028
:105EC0003212604EE84970F4900902E06007640104
:105ED0006003025FA71230EB8A0C8B0DA80CA90D92
:105EE000800612603212604EE849603588828983EC
:105EF000126BCF900551E06A7003A3E06B600C1247
:105F00006032F583126BCFEA4B70D7888289831297
:105F10006050900551E0687003A3E0697003025F70
:105F2000A77A167B00123BFB8A0C8B0DAE0CAF0DD3
:105F3000EE4F60739005511260508E828F83125E17
:105F40008B900546E08E828F83A3A3F0123247E93F
:105F50008E828F83A3A3A3A3A3F090153912751784
:105F6000F07C657D0512602A124525AA18AB1979C7
:105F7000411245F1851882851983E0600890077306
:105F8000126050800478FE79FF8E828F83A3A3A3D2
:105F9000A3A3A3A3125E8B126038E50AF0A3E50B5E
:105FA000F08E0A8F0B0508900787E0F8E508C39884
:105FB00050047A008022E508C398FAC39406400290
:105FC0007A057900800DE50A126044350B1259629A
:105FD000F50B09E9C39840EE7509007809122A0605
:105FE000780A122A02EAF5097809122A0690078728
:105FF000E0F5097809122A06AD087C007A7E7B0755
:1060000090077CE0F91240457405122A309009028D
:10601000E060046401700BEE4F6007EEFAEFFB12D4
:106020003C01122E4574010252E5EE240BFAE43FC6
:10603000FB22E81260443922EE12603D22126044D5
:106040003FF583222414F582E42212727B3FF5830C
:1060500012605422E0F8A3E0F922EEFAEFFB7F068B
:106060000226B974EC12242A74FF122AC48A0A8BFD
:106070000B7E008E0E8E0F125E86350B126450FF63
:10608000AC18AD197A007B00799D122E9985188283
:10609000851983E0F8EFC398400302613EE0C39F97
:1060A000FEC3940B40027E0AEE75F007A4FAABF033
:1060B000123BFB8A088B098A0E8B0FEA450F607C26
:1060C000750C00801A850882850983A3A3A3A3A366
:1060D0007403F0E5082407F50850020509050CE5EE
:1060E0000CC39E5059AC08AD09850C10E5102FFA71
:1060F000E43400FB798B122E99850882850983A3ED
:10610000A3A3A3A3E014600814601314601F80B558
:10611000850882850983A3A3A3A3A3E480B485088B
:1061200082850983A3A3A3A3A3740180A585088204
:10613000850983A3A3A3A3A3740280967E00750898
:10614000007808122A06780E122A02EEF50878085E
:10615000122A06EFF5087808122A067405122CAFE9
:10616000E0FD7C00E50A126515350BFBE50A1262BD
:10617000A6350BF583E0F91240517405122A30E57B
:106180000E450F6007AA0EAB0F123C017401122AD4
:10619000307F0C0226B974EA12242A74FE122AC433
:1061A0008A148B15750A00750B0012644AF508AC49
:1061B00018AD197A007B0079A31247E385080C8596
:1061C0001882851983126050C3E50C98E499507DBC
:1061D000851882851983E0C3950CFEA3E09400FF27
:1061E000C3EE9404EF940040067E037F008004EE2B
:1061F0004F605AEEFAEFFBEA75F015A4FAA8F075B5
:10620000F015EBA428FB123BFB8A0C8B0D8A0A8B42
:106210000BEA450B6037750900750E00850E10C33B
:10622000E5109EE49F502BAC0CAD0D850E12850839
:1062300010E5122510FAE43400FB79A21247E3E5D9
:106240000C2415F50C5002050D050E80CF75098B39
:106250007E00750C00780C122A06780A122A02EECB
:10626000F50C780C122A067808122A067405122CEE
:10627000AFE0FDAC091262921240577405122A3049
:10628000E50A450B6007AA0AAB0B123C0174020237
:106290005D78E5141265153515FBE5141262A63517
:1062A00015F583E0F922240FF582E42274F6122416
:1062B0002A74FF122AC41263021273BDA3A3A3A3FC
:1062C000A3A3A3A3E0F9122E63E98518828519839D
:1062D000F07508007808122A067401122A7E8808D0
:1062E00089097808122A027508357509807808121C
:1062F0002A0212630B123FAF7405122A3074010296
:1063000051D0EAFEEBFF12727B3F22790112631536
:10631000FAE43FFB22EE2402FCE43FFDEE240F22D0
:1063200074F412242A74FA122AC48A088B09EA1215
:106330007274127289FFEEFAEFFB122D4FE96013AF
:106340001231BDEAFCEBFDEEFAEFFB12451FE964EA
:1063500001700A7401122CAFE4F0A38009740112D9
:106360002CAFEEF0A3EF127556A3A3A3A3A3E0F8FE
:10637000A2E650087403122CAF7401F0E8A2E750B3
:10638000087404122CAF7401F07405122CAFE4F001
:1063900004122A86122E8DE9851882851983F07AD7
:1063A000007B001231E1750A00780A122A06740196
:1063B000122A7E880A890B780A122A02750A347515
:1063C0000B80780A122A021263D7123FAF740512AB
:1063D0002A3074060268887901E5082402FCE43555
:1063E00009FDE508240FFAE43509FB2274F61224AE
:1063F0002A74FF122AC4126302126450F9122E5139
:10640000E9851882851983F0EE240B126442702C02
:106410007508007808122A067401122A7E880889F5
:10642000097808122A027508367509807808122A38
:106430000212630B123FAF7405122A300262FDEEA6
:10644000240EF582E43FF583E022EA12727C3515D2
:10645000F583126457E022E0F8A3E0F583888222F6
:106460000229E274F412242A74EF122AC4EAFEEB21
:10647000FF1252EB900773E065087004A3E0650912
:106480007052A818A919880A890B780A122A02756D
:106490000A11750B00780A122A027C007D007A81AD
:1064A0007B00123C857404122A30E97027750A00BB
:1064B000780A122A067401122A7E880A890B780A41
:1064C000122A02AC08AD091264FA124009740312D0
:1064D0002A308021750A11750B80780A122A0278F9
:1064E00008122A0212643FFD7C841264FA124015DD
:1064F0007404122A3074110268881264FE22EE12AB
:1065000065153FFBEE240FF582E43FF583E0F922A9
:10651000FCEFFDE5082402FAE42274F112242A7447
:10652000EB122AC4EAFEEBFFEE2413126442126659
:1065300048FAE4CAFBEC2AF508E43BF50990077336
:10654000E065087004A3E0650960030265F08882D5
:106550008983A3A3E09410500F88828983A3A3E0CA
:10656000851882851983800885188285198374109F
:10657000F0E0C0E07404122CAFD0E01273AEA3A31D
:10658000A982AA83890C8A0D750E00780C1229FE47
:106590007407122CAFE0FC7D007408122CAFAA82A5
:1065A000AB83123B3B7403122A307404122A7E8898
:1065B0000A890B780A122A02750A11750B00780AEB
:1065C000122A027C007D007A817B00123C7F7404D9
:1065D000122A307404122CAFE09007AC6005E0D2B0
:1065E000E48003E0C2E4F0851882851983E4800822
:1065F0008518828519837484F0E0C0E07401122C40
:10660000AFD0E0F07402122CAFE508F07403122C46
:10661000AFE508F0125B04126657122A06740212E4
:106620002A7E880889097808122A027508147509D3
:10663000807808122A02790312630D123FAF7405A5
:10664000122A307415026AE11273D1E0FCA3E02231
:10665000E5161273A03517F583E0F5087808227463
:10666000F412242A74E0122AC48A088B09AC18ADEB
:1066700019123F9D900902E0640270337402122CDB
:10668000AFAE82AF831231BDEEFCEFFD12451FE9C4
:10669000601D1231C38A0A8B0BA80AA90B851882C8
:1066A000851983E0687003A3E069700302688612AD
:1066B00033797402122CAF126BC512328FE9640168
:1066C00070030268867418122A861231CF7402127F
:1066D0002CAFAC82AD837418122A8612451FE96074
:1066E000321231C98A0A8B0BA80AA90B8518828538
:1066F0001983E0687003A3E0696018851882851922
:1067000083126050900547125E8B7A477B05794B68
:106710001245F7900902E06007640160030267C454
:1067200012719AC082C0831231C38A088B09D08348
:10673000D082E065087004A3E06509605C74021211
:106740002CAFAA82AB83122DBB8A088B09A808A99B
:1067500009E849602688828983A3A3A3A3E0640192
:10676000600D88828983A3A3A3A3E06402700C74E4
:1067700002122CAFAA82AB83122DC79005E51268D6
:106780009660169008F6E06401700E126BC99005D1
:10679000E6E0F58388821248721231C38A088B09B9
:1067A000A808A909851882851983E0687003A3E009
:1067B0006960117402122CAF126BC5122D9DE96035
:1067C00003123E297402122CAF126BC51233677983
:1067D00000126BC9122FDD740B122CAFE412689AF1
:1067E000F8A3E0F9740C122CAF125E8B740B122A12
:1067F00086122D6DE9603F7C087D007900741812C7
:106800002A86123B47740E122CAFAC82AD837418EB
:10681000122A8612451FE9601D7402122CAFAC8249
:10682000AD83740E122CAFAA82AB83122D49740B68
:10683000122A86122D7F7402122CAFAC82AD8374A3
:106840000E122CAFAA82AB83122D49740B122A862A
:10685000122D73E96030740C122CAF126050851841
:1068600082851983E0687003A3E069601985188246
:10687000851983126050740C122CAF125E8B740B4E
:10688000122A86122D7F7420122A307F040226B924
:10689000F582E438F583126D5022F085188285194F
:1068A00083E02274F112242A74F6122AC4EAFEEB61
:1068B000FF75080090081812689670507A377B00B0
:1068C000123BFB900818EAF0A3EB12708560197C6C
:1068D000377D007900123B47EEFCEFFD900818125F
:1068E0006BCF123F6DE9700B851882851983748810
:1068F000026A4A127381126AE97401F07C797D3F61
:106900009004D3126BCF12484F026ADFE0C8126ABC
:10691000E97402F0EEFCEFFD126FDB123F6DE970DF
:106920000C8518828519837488F0750801750AE250
:10693000750B07780A122A02126BDF1228411273B4
:10694000812428126FCEFC126C121273812414124F
:106950006FCEF9123ED17404122A30126AF6126B0D
:10696000132431126FCE604312706FFAE433FB12BE
:106970003BFB900818E02432126B286022750CE271
:10698000750D07750E00780C1229FE12706FFCE46D
:1069900033FD126BFD123B3B7403122A30800C85D1
:1069A00018828519837488F0750801780A122A0202
:1069B000126BD31228411273812411126FCEFC1274
:1069C0006BF4127381242B126FCEF9123ED1740432
:1069D000122A301273812434126B132434126FCEB6
:1069E0006035127066FAE433FB123BFB900818E046
:1069F0002435126B286042750CE2750D07750E0088
:106A0000780C1229FE127066FCE433FD126BEB1257
:106A10003B3B7403122A30E508A2E04025126AF6D7
:106A2000126FCE700890081812703260157B007AD1
:106A3000007900123F73026ADF851882851983741A
:106A400088F08518828519837486F07409122CAF3A
:106A500074021271DE126B05122CAFE8F0A3E9127A
:106A60006B0DF5087808122A067401122A7E880830
:106A700089097808122A0275082075098078081299
:106A80002A0279017406122A8EEEFAEFFB123FAF4A
:106A90007405122A3012702170427409122CAF74DE
:106AA00002F0126AFF122CAF12708C122A067401C7
:106AB000122A7E880889097808122A02750820752A
:106AC00009807808122A0279017406122A8E900829
:106AD00018126BCF123FAF7405122A30123F677441
:106AE0000A122A307F070226B9126AED22242EF5F7
:106AF00082E438F58322900818126FF7243122902F
:106B00000818126457A3A31260547401221271DE94
:106B1000A3E022F582E438F583126B1EC822E9F067
:106B2000900818E0F8A3E022F8A3E03400F9888286
:106B30008983EAF0A3EB1273B7126D5022C082C0B2
:106B4000839008181268966075E0C8243512689022
:106B50006006126BEB123C011273812432126890B2
:106B60006006126BFD123C011273812412126890B0
:106B70006009126BD3126BCF123C01127381241582
:106B80001268906006126C12123C01127381242963
:106B90001268906009126BDF126BCF123C01127306
:106BA00081242C1268906006126BF4123C0190084C
:106BB00018126BCF123C01900818E4F0A3F0D083B8
:106BC000D0820229E2AC82AD8385188285198312B6
:106BD0006C0C22126FF42412F582E438F583221231
:106BE0006FF42429F582E438F58322126FF42435FA
:106BF000126C0622126FF4242C126C0622126FF40F
:106C00002432126C0622F582E438F583E0FAA3E020
:106C1000FB22126FF42415126C062274F112242A3E
:106C2000EAFEEBFF8C088D09750A018C0C8D0D7541
:106C30000E00780C1229FE7C177D00123B3B74037A
:106C4000122A30EE2412126D1CF0A3F0EE2415125D
:106C50006D1CF0A3F012719AE0603AEE2412F8E491
:106C60003FF9880C890D1271C3123BFB126D3D6018
:106C700021E5082412126D301229FEE508241112B4
:106C80006D24125D99126BCF123B3B7403122A30B4
:106C90008003750A00E5081271A86035EE2415F826
:106CA000E43FF9880C890D1271C3123BFB126D3D54
:106CB0006055E5082415126D301229FEE5082414EC
:106CC000126D24126D0C126BCF123B3B7403122A0F
:106CD00030E50AA2E0402BEE2412F582E43F126870
:106CE000946009125D98126BCF123C01EE2415F5E9
:106CF00082E43F126894600AEE126D0C126BCF12A0
:106D00003C01A90A026AE4750A0080CB126D1022C8
:106D10002415F582E43FF58322EE2414F582E43F46
:106D2000F583E42212736DE025E0FCE433FDEE22EE
:106D300012736DE0F50CA3E0F50D780C22850C8242
:106D4000850D83125739850C82850D83126D502273
:106D5000E0F8A3E0F9E8492274EE12242A74ED1257
:106D60002AC4890A8A0E8B0F750C00750D00750BED
:106D7000FF7510FF7511FF750800750900851882F1
:106D8000851983E412708560177403650A600674C0
:106D900002650A7010E0C82430126FCE650F6005DE
:106DA0007900026FC47C797D3F7A007B0012484FE6
:106DB0007401650A700A8518828519837485803D7F
:106DC000E50A60067403650A7019900818127001CC
:106DD000F07403650A7029E50E602985188285190B
:106DE00083801A7402650A701BE50E9008187005FE
:106DF00012700180081273841270187402F08004FB
:106E0000E50A601E127007701912702B6005126A75
:106E1000F9800A127032600A1273812434126FCE24
:106E200014F012702B6022125119F50912706FF8CC
:106E3000E433F9900818E0FAA3E0CA243212704350
:106E4000241D126FE82425802E127032602E9008C7
:106E500018E02417F508A3E03400F509127066F86D
:106E6000E433F9900818E0FAA3E0CA24351270431D
:106E70002406126FE8240E126FCEF50B7409122C43
:106E8000AF740212689A6003026F32E50845097018
:106E900003026F3212700770047E2280027E218509
:106EA0000882850983126B05122CAF125E8B900845
:106EB0001CE0C0E01273812430F582E438F583D001
:106EC000E0F07412122CAF7403F0AC0CAD0D740A28
:106ED000122A86124525850882850983A3E0F50CD0
:106EE000780C122A06780B122A06740C122A7E8855
:106EF0000C890D780C122A027810122A02E5082457
:106F000006F50CE43509F50D780C122A02126FD63D
:106F1000F97409122A8EEEFA7B00124021740812CD
:106F20002A307C797D3F9004D3126BCF12484F02F8
:106F30006FC2126AFF122CAF12708C122A067401F3
:106F4000122A7E880889097808122A027508207595
:106F500009807808122A0279017406122A8E900894
:106F600018126BCF123FAF7405122A3012702170C5
:106F70004E1273812419F582E438F583126B0712DF
:106F80002CAFE8F0A3126B192418F582E4381266CE
:106F900057122A067401122A7E8808890978081275
:106FA0002A027508207509807808122A027901746E
:106FB00006122A8E126FDB123FAF7405122A3012AE
:106FC0003F6779017413122A307F0A0226B9F582CD
:106FD000E438F583E0221274B7E022900818E02428
:106FE00017FAA3E03400FB22F50CA3E03400F50D02
:106FF000126FF422900818126FFB22E0F8A3E0C889
:1070000022127011740122900818127011E06401AC
:1070100022126FFB12701822242FF582E438F583B8
:1070200022126FF4126AEDE0640222127075900869
:10703000182212703622126FFB2434F582E438F5E0
:1070400083E022F582E43AF583E028F8A3E039F9F9
:10705000E824FEF582E934FFF583E0F510A3E0F5BE
:1070600011900818E02290081812703625E02212BC
:10707000707525E022900818126FFB2431F582E428
:1070800038F583E022126B1FF9E84922E8F0A312D9
:107090006B1EF5838882A3E0F508780822C082C0C1
:1070A000837B007A857901123F73026BBE74F41200
:1070B000242A8C088D09EA240F12755C1274C112FF
:1070C00060508C828D83A3A3125E8BEA240E12750E
:1070D0005CA3F01272801271CF12739350010FFCF7
:1070E000EFFDE5082406FAE43509FB124525EE24F8
:1070F00008FE50010F8E828F83E0C0E01274B3D07F
:10710000E012728EF81274A3E812739750010FE523
:107110000824121271A2A3F0E50824151271A2121C
:1071200071D8A30EAF83C0E012719AD0E0F060284E
:10713000E50824121271BA123BFB12756F6019E553
:107140000824121271AD12719CE0F9123EF58A0A00
:107150008B0BAE0AAF0B8007E50824111271A28ECB
:10716000828F83E0A3AE82AF83C0E0127266D0E06C
:10717000F0601FE50824151271BA123BFB12756FFF
:107180006010E50824151271AD1271A8F9123EF5D0
:107190008005127266E4F002688BE5082411127310
:1071A0006D2212736DE4F02212726CE02212736D84
:1071B000125760EEFAEFFBE50822F8E43509F9888A
:1071C0000A890BE01271C82225E0FAE433FB22FFA2
:1071D0001274938C828D8322A31271DEE022F08ED2
:1071E000828F832274F612242A8C088D09127280F1
:1071F000FFEEFCEFFDAA08AB09124525EE2408FEC0
:1072000050010F8E828F831275BD12728E85088297
:10721000850983A3A3A3A3A312739350010F8E82A6
:107220008F83E0F8E508127274E8127388740368BB
:107230007026EEFCEFFDE508240BFAE43509FB129D
:1072400045258E828F83A3A3A3A3A3A3A3A3E0C0FA
:10725000E0127266D0E0800A12748C127367E8F054
:10726000A3E9F00251D3E50812726C221260443592
:1072700009F5832212727C12737022EE1273DB22E4
:1072800012753412728722F583E0FEA3E022127495
:10729000E21274972274F212242AEAFEEBFF750AB6
:1072A00000EE2410126442C3940C400D12750C12AF
:1072B0007384240B126FCEF50AA80AE828F8E43389
:1072C000F9E8240DFAE439FB123BFB8A088B09EA42
:1072D0004509700302735E1263061274FB8A828B87
:1072E000831274DE7078EEFCEFFDEA2403FAE435D5
:1072F00009FB124525EE2408FE50010F8E828F8374
:1073000012737D85088285098312739650010F12CE
:107310007365E4F0E50A6046E508240DF8E43509F4
:10732000F98E828F83E0C0E0127365D0E012749E04
:10733000C0E0127375D0E0127388850A0B8E828FBD
:1073400083E0FCA3E0FBEC888289831273A65001E2
:1073500009EE2402FE50010F150BE50B70DFAA08A1
:10736000AB0902605EE508240B12736D22F582E41E
:107370003509F58322E508240C12736D22127497E7
:1073800022900818126FF72212738C221274EA0EE0
:10739000AF8322A3A3A3A3F0A3E9F0EE2402FE226D
:1073A000240EF582E42212573AE82402F8221273DE
:1073B000B2221273B7A322F08882898322126C0A48
:1073C0008A828B83227F010226B91273DA3FF5830A
:1073D000E0F8A3E0F98882898322EE2413F582E4A1
:1073E0002274F212242A127530125117850882F580
:1073F00083E0F50DA3858208858309A3A3E0F50C3E
:107400001274F63400FB123BFB8A0A8B0BAE0AAFF8
:107410000BEE4F60378E828F83E50DF085088285F5
:107420000983E0FA127543850882850983A3A3A323
:10743000A982AA8389088A09880A78081229FE1273
:1074400074F13FFB123B3B7403122A3002605A7402
:10745000F712242AEA2413F8E43BF988828983E0AE
:10746000FAA3E0F5838A821275621274871273D1CF
:10747000A3E0FA88828983A3A3E0F9EA8C828D8352
:10748000A3125E8C0273C51273B7E022127497F8D0
:10749000E508228E828F83E0FAA3E0F9EA221273D4
:1074A0008CE0221274A722E508240FF582E4350946
:1074B000F583221274B722E5081273A03509F5830B
:1074C000221274C6A322F08A828B83A3221274D163
:1074D00022F08A828B83A3A3A322A3A3A3A3127463
:1074E000E2221274EAAE82AF8322F08E828F83A3EF
:1074F00022AC0C7D00EE2404FAE4221274FF22F583
:1075000083E0FEA3E0FF8E828F83E02212751022BB
:107510001273DA3FF58322E08E828F83A3A3A3A3A5
:10752000A3A322F0850A82850B83A3228C088D09F0
:1075300012753422EA1273DB3B22F085088285093A
:1075400083A322127568EA8E828F83A3F0A3E912C7
:107550007556E50CF0221274EAA3A322F582E43BEF
:10756000F583E08C828D8322A3E0F8E4C8F92285BC
:107570000A82850B83125739850A82850B83126D27
:10758000502274F612242A12752CF5831275B61245
:1075900071CF12739750010F1265103509FB124518
:1075A000258E828F83A3A3A3A3A3A3A3A31275BD38
:1075B000A3A3F00251D3126054E8FEE922127663CD
:1075C000A3A3221275C722E0FA127568EA282212D4
:1075D00074D1A3A3A3A32274F612242A12752C1229
:1075E0007650123B53EAF8EBF9ECFAEDFB85088292
:1075F000850983122C98EE2404FE50010F8E828F91
:1076000083E08508828509831274DAC394065005E5
:107610001276688037850882850983A3A3A3A3E037
:1076200064FE600E850882850983A3A3A3A3E0F40A
:10763000701B12765B127388850882850983A3A369
:10764000A3A3E0F47007127675F0A3E9F00251D31A
:10765000127287FF7904EEFAEFFB228E828F83127B
:10766000766322127668A322E0850882850983A3C7
:10767000A3A3A3A322127493850882850983A3A3DD
:10768000A3A3A3A3A322C082C083E9901560F090B6
:1076900013C774C7F0A37445F0027B3F74F412243F
:1076A0002A74FF122AC48A088B09EB54807056EAA8
:1076B000A2E0507C9013BDE0F91245A9E9FE6010EC
:1076C00012773E1245F7790012310F9013BEE4F0A5
:1076D0007A027B00123B5FEA4B60128A828B8374D2
:1076E00033F0EEA3F0901561E0F9123B6BE508640E
:1076F00001FAAB09803EE0640D70031245DFEEFA3B
:10770000EFFB123B65901560E0F9123B778A0A8B1C
:107710000BAE0AAF0BEE4F600E8E828F83E0640CCF
:1077200070D41245D980D7AA08E5096480FB80048B
:107730007A007B007401122A307F040226B9851872
:10774000828519837401F0AA18AB1979522274F654
:1077500012242A8A088B09ECFEEDFF7C177D007944
:1077600000EEFAEFFB123B4712784DC0E0EE24101A
:10777000F582E43FF583D0E0F0E508241DF582E4CE
:107780003509127EFBE508240DF582E43509F58301
:10779000E0FAA3E0FB8E828F83A3A3A3A3A3A3A3FA
:1077A000A3A3A3EAF0A3EBF088828983E0FA8E8298
:1077B0008F83F088828983A3A882A98374035A6483
:1077C00003703C8E828F83E0540CFA74086A700850
:1077D0001278437401F08013127843E4F0740C6A59
:1077E000700912785A12786B50010912785A12787F
:1077F0006950010912785AA3A3127869500109EE61
:10780000240EF582E43FF583E8F0A3E9F0EE2410BE
:10781000FAE43FFBE508241DF582E43509F583E031
:10782000FC8A828B83E0C3982CF8F012784DC398C1
:10783000C0E0EE240DF582E43FF583D0E0F07F0256
:107840000226B9EE240CF582E43FF58322E50824F4
:1078500017F582E43509F583E02288828983E0FC0C
:10786000A3E0FBEC8E828F8322A3A3A3A3A3A3F0A8
:10787000A3EBF0E82402F82274F712242AEAF8EBCA
:10788000F9ECFAEDFB740B122CAF1279EBEC24152A
:10789000F582E43DF583E0540D700F8C828D83A357
:1078A000A3A3A3A3A3A3A3E0700579B60279578885
:1078B0008289837403F0EC2408FEE43DFF8E828FFE
:1078C00083E08A828B83A3A3A3A3A3A3A3A3F08EA5
:1078D000828F83E0640F701088828983E0D2E31284
:1078E000795C8C828D8380158C828D83A3A3A3A366
:1078F000A3A3A3A3E064028C828D837009127EFD92
:107900008A828B83804AA3A3A3A3A3A3A3A3E06437
:10791000037005124525803D8C828D83A3A3A3A30C
:10792000A3A3A3A3E06401702C88828983E0440CA4
:1079300012795C8A828B8374FFF0A3F08C828D8332
:10794000127EFD7409122CAFE0FAA3E0F5838A825F
:10795000E8F0A3E9F079007F010226B9F08A828B72
:1079600083A3A3A3A3A3A3A3A37402F02274F51279
:10797000242AE9FE8A828B83F0A3AA82AB83740C4B
:107980005E640C700AECF0A3EDF0A30A0AAB8374FA
:107990000B122CAF1279EBEC240D1279DBAA8212B8
:1079A00079F1240F1279DB0A1279F12413F582E4BC
:1079B0003DF583E0F508A3E0F509750A00780812A3
:1079C00029FEEC2411F582E43DF5831279EB123B9C
:1079D0003B7403122A307F030226B9F8E43DF9888C
:1079E000828983E08A828B83F0A322E0FCA3E0FDFE
:1079F00022AB8388828983A3E08A828B83F0A30AE7
:107A0000AB83EC22C082C08374FE122AC4740112BC
:107A10002CAFE9F07902123145E9701E124651E9A6
:107A200060187401122A8679E11245F712773E1226
:107A300045F79013BEE4F0F980027901027B3A74B5
:107A4000F712242A74FE122AC4E9FE9013BEE060E5
:107A500004790180547401122A8679E11245F17487
:107A600001122CAFE06E601F9013BE7401F0F9128A
:107A7000310F851882851983E41277461245F7EE97
:107A8000F91245A9E970047900801EEE9013BDF04B
:107A90009080B012283D7A017B00901560E0F912C9
:107AA0003CC17404122A3079BA7402122A30027965
:107AB00057C082C08374FE122AC49013BEE06004D3
:107AC000790180497401122A8679E11245F1740125
:107AD000122CAFE0F8900546E06870047900802D24
:107AE0009013BE7401F0851882851983E4127746DD
:107AF0001245F77A467B0579E11245F712773E1277
:107B000045F7790012310F9013BEE4F0F9802BE9AC
:107B1000F874FE6870047901800279000229E2C0DD
:107B200082C0838A828B83127B8EE0901561F08AFB
:107B3000828B83E09013BFF080057402122A30D04C
:107B400083D0820229E2C082C0838A828B83E0F8DC
:107B5000740D68600A740C687030A3A3127B8EA346
:107B6000A3127EFD88828983E5824583601CE054F0
:107B70000364037015A3A3E054036403700C901511
:107B800060E0F9123B6B79018002790080B1A3E0DB
:107B9000F8A3E0F58388822274F212242A74DC129E
:107BA0002AC48A0A8B0B7401122CAFE4F0A3F09064
:107BB00013BEE070138A828B83A3A3A3A3A3A3A302
:107BC000A3A3A3E064FE60057901027CFD7C217D16
:107BD0000079007403122A86123B47780A122A029F
:107BE0007403122A7E880889097808122A02740709
:107BF000122A8E7404122A8612459D7404122A30A9
:107C0000E9FE6003027CFB7A01851882851983E016
:107C1000540C640C70020A0AE50A2411F582E4355A
:107C20000BF583E02A2406F5087421122CAFE50831
:107C3000F0FA7B00123BFB8A088B09EA45097003C6
:107C4000027CF97422122CAFEAF0A3EBF0780A124E
:107C50002A027403122CAF1279EB7402122CAFE0DB
:107C6000F9EA2402FAE43509FB1245A37402122A48
:107C700030AE08AF09123247E9F50C750D007402F9
:107C8000780C122BC6E50C44038E828F83F0A3E59B
:107C90000DF0E50A240BF582E4350B127EFB740C23
:107CA000122CAFE8F0A3E9F0740E122CAF7403F0BD
:107CB000E50A2417F582E4350BF583E0C0E0740F84
:107CC000122CAFD0E0F0851882851983E0540C7037
:107CD0000C7410122CAF7401F0A3E480087410121D
:107CE0002CAFE4F0A3F07403122A8612462DE9FEAD
:107CF000AA08AB09123C0180027E10EEF97424122E
:107D00002A307F060226B9795D0229E2C082C0834B
:107D1000EAF8EBF988828983A3E0FB88828983A350
:107D2000A3E0FA9013BFE0F912370F027B3F74F51E
:107D300012242A74BC122AC4EAFEEBFF8E828F83BF
:107D4000A3A3A3A3E0F50A8E828F83A3A3127EFDD3
:107D5000880889097C217D0079007403122A861223
:107D60003B477403122CAFE50AF07403122A8E8588
:107D70000882850983E0FAA3E0F8E4C8F9EA28E478
:107D800039FB1231AB7404122CAF7402F0E50824F5
:107D900002F8E43509F97420122CAFE8F0A3E9F0F9
:107DA0007403122CAFE024FEC0E0741A122CAFD082
:107DB000E0F0EE241CF582E43F127EFB7410122CDE
:107DC000AFE8F0A3E9F0EE2413FCE43FFD743B12AE
:107DD0002A861245197405122CAFE0640360030271
:107DE0007EF6123247E9F87406122CAFE0686003A1
:107DF000027EF67407122CAFE070287408122CAFC4
:107E0000E070207409122CAFE07018741B122CAFB4
:107E1000E07010740A122CAFE07008740B122CAFD3
:107E2000E06003027EF67424122A8E7403122A86FE
:107E30001245977424122CAFE054036403600302CC
:107E40007EF6E0540C64047003027EF6E0A2E55076
:107E500003027EF6A2E75003027EF69013BFE0C055
:107E6000E07426122CAFD0E0F07427122CAF74FE11
:107E7000F0EE242FF582E43FF583E0851882851922
:107E800083F0EE2430F582E43FF583E0C0E0740136
:107E9000122CAFD0E0F0EE2431F582E43FF583E020
:107EA000C0E07402122CAFD0E0F075080078081220
:107EB0002A06EE2425F582E43FF58312283D780852
:107EC000122A067406122A7E880889097808122A5E
:107ED00002EE242BF582E43FF583122841741F1231
:107EE0002CAFE0F97445122A8E742E122A8612479E
:107EF00011740A122A3074440279D3F583E0F8A38E
:107F0000E0F922C082C083123E71123E77D083D046
:107F1000820229E2C082C083900902E070089007C3
:107F2000ACE054F8801B6401700A9007ACE054F890
:107F30004401800DE0640270099007ACE054F844FD
:107F400002F09007ACE05407F0A37440F0900902EF
:107F5000E06004640170139007AE748EF090090223
:107F6000E070129007AE748F800AE0640270069091
:107F700007AE7480F09007AFE4F0A3F0A37450F064
:107F8000A374A0F0A3E4F09007B674A0F0A3E4F00B
:107F90009007B4F0A3F09007B8F0027F0DC082C044
:107FA00083900902E060046401700B9007B97410BB
:107FB000F0A374C18033E06402702F90152AE0F8BA
:107FC000A3E0F9E8499007B96007127FED4401800A
:107FD00005127FED44029007B9F0A3E9F09007B9CC
:107FE000E0540F4420F0A37482F0027F0DE054F0BF
:107FF000F8A3E0F9E822FFFF851A87000229E2FFD3
:108000007546D13567305B488F471B3D833E9145B0
:1080100073456B41000000000000000000000000FC
:108020000000000000000000000000000000000050
:108030000000000000000000000000000000000040
:108040000000FFFFFFFFFFFFFFFF0008000400022A
:108050000001FFFFFFFFFFFFFFFF00000000000027
:108060000000020502000801740000000000008208
:10807000003A003B0000000000000002000206027F
:10808000FA0000000400000019E0FCFFF8FF000007
:10809000E71F0300805101003C000000100E0000AB
:1080A000E8030000300000000000000009433886AB
:1080B00064000000000000FF3200000000F8FF072D
:1080C00060EA000000000000010000000A0000005B
:1080D00002000000FEFFFFFF1F000000080000007C
:1080E000975118006AAEE7FF965118009F020000F2
:1080F000E9FFFFFF0000FF00BC02000000000000DD
:108100000A74F712242AE990059EF0900553E4F0D2
:108110001244FB9005B2E4F0A3F090059FF0A3F0A9
:1081200012331F900902E0600464017006122D8B67
:10813000122F47124501900514E4F0A3F0124633C4
:1081400002B13B74F012242AEAFEEBFF548060680F
:1081500090059EE0F9123B778A088B09EA45096091
:108160004F7C0080010CEC75F003A4F8A9F0741C9E
:1081700028F582744D39F583E493F4602CE493F888
:108180008508828B83E06870DCAA08EC75F003A494
:10819000F8741D28F582744D39F583E493C0E074BA
:1081A0000193F583D082124872AA08AB09123B658D
:1081B000EEFAEF6480028434EF5420601E123181A5
:1081C0008A088B09EA4509600A12309DAA08AB09A2
:1081D000123B65EEFAEF6420028434900902E064F9
:1081E000027024EEA2E0501F900558E0640F701159
:1081F000790012306DE9600990152A12D31F1230F0
:1082000085EE640102833AEE5420700302830B75FD
:108210000C007A207B0090059EE0F9123CD3EA4BDB
:108220004C4D70179080D012283D7A207B0090052D
:108230009EE0F9123CC77404122A307C0079047A5B
:10824000007B0012314B8A088B09801885088285D3
:108250000983A3A3A3A3A3A3A3A3A37401F0850AE3
:1082600008850B09E508450960777C007904AA08B0
:10827000AB0912314B8A0A8B0B750C01E5082404FB
:10828000F8E43509F98882898312EECD12EA657027
:10829000CD850882850983A3A3A3A3A3A3A3A3A336
:1082A000A3E0640170A6850882850983A3A3A3A324
:1082B000A3A3E054047095850882850983A3A3A332
:1082C000A3A3A3A3A3A37406128B36700374B7F001
:1082D000E0FA85088285098312861212307F0282B5
:1082E0005E12311B7C0079017A007B0012314B8BCE
:1082F00009EA45097010E50C700C7A207B009005A6
:108300009EE0F9123CCDEE6420802FE0600764010E
:10831000600302840AEE54106008122F83EE64108A
:108320008018EE54406008122FFBEE6440800BEE84
:108330005480600B122E57EE6480FAEF028434EF03
:10834000540160169005D112CB65600612C5CF129C
:108350004872EEFAEF6401028434EF540860471269
:108360002F539008F2E0640170349008F3E0602E1F
:10837000F508E4F509F50AF50B9080A0780C122CAD
:10838000587808790C12233B78081229FA7A007B76
:108390000890059EE0F9123CC77404122A30EEFAE8
:1083A000EF6408028434EF541060129005B0E0606E
:1083B00005E4F0122F53EEFAEF64108077EF54408B
:1083C00060489005DB12CB6560399005E112CB6502
:1083D00060319008F6E0640170299005DB12C5CC8D
:1083E0001248729005E112C5CC1248729080C012FA
:1083F000283D7A007B4090059EE0F9123CC774044A
:10840000122A30EEFAEF6440802AEF5402600A121A
:1084100032E9EEFAEF6402801BEF5404601912CACD
:108420006F12C881790190055112D31F122ECFEE21
:10843000FAEF6404FB80047A007B0002C10CC08266
:10844000C08374EA122AC47C167D007900AA18AB96
:1084500019123B477408122CAF7402F090054712B2
:10846000975C12847D7409122CAF12C881741312A8
:108470002CAFE412C9CB1246217416800EE8F0A38B
:10848000E9F090055112D0E0227408122A3002C19E
:108490004474F712242A74DF122AC4EAFEEBFFEEBA
:1084A0004F602DAC18AD191231A57406122CAFE037
:1084B000601E7417122CAFE0FD7401122CAFE0FCAB
:1084C000EEFAEFFB7900122D07E9600479A480022F
:1084D0007900742102B13874F412242AEAFEEBFF09
:1084E0008E828F83A3A3A3A3A3A3E054406016129C
:1084F0008B2A12325FE960077AFF7BFF0285D9126F
:10850000C5C80285CC900902E060076401600302DF
:1085100085B290053EE0A2E140030285B28E828FD3
:108520008312860C12C991A3A3A3A3E0FA888289BF
:1085300083A3A312D4F28E828F83A3A3A3A3A3A3A6
:10854000A3E054106004794080027900750AFE753A
:108550000BFF780A122A0212B600122841AC08ADAD
:1085600009128B2A122F597404122A30E5086A70F6
:1085700003E5096B600B12B6056A7003A3E06B702C
:108580004E750A00780A122A0679028E828F8312AB
:10859000B1F0AA08AB091232A17401122A30750891
:1085A000CDAA088E828F8312861212307FE9604C2A
:1085B0008057900902E06402600FE060046401707B
:1085C000DD90053EE0A2E140D590054712D31F742F
:1085D000FE6A700374FF6B60C512C5C812DA13120D
:1085E000325FE98E828F83600512AA26800312AA69
:1085F0003B12AA44124627E9F50870A5EE4F600920
:108600007901EEFAEFFB12312702BED9E0F812B27F
:10861000322212ED98E0F92274F612242AE9FEEAD9
:10862000FF7A0F7B00123B5FEA4B601F8A828B83CD
:10863000740CF0EEA3A3F0EF8A828B8312AE7990D4
:10864000059EE0F9123B6B7900802FEEF912315153
:108650008A088B09A808A909E849601C88828983CF
:10866000A3A3A3A3A3A3A3A3A3740612E655E0F9AF
:1086700012300DEEF912312D791002C4B874F412D3
:10868000242A900558E0640F7030EA4B602C900566
:1086900053E064086005E06404701F8A088B09E4F5
:1086A000F50AF50B78081229FA7A017B0090059EED
:1086B000E0F9123CC17404122A3002984774F21295
:1086C000242AEAFEEBFF8C088D09890A740E122C0D
:1086D000AF129776850C82F583E4F0A312C887E089
:1086E000F912323BE9602612D31212325FE96402BA
:1086F000701B8E828F83A3A3A3A3A3A3A3A3A31200
:10870000B898850C82850D8312C8818003750A0094
:1087100012B02A14602514603A14605B146063146C
:10872000603F14607D24FE70030287BC1470030256
:1087300087D01470030287E30287F1780C122A02B3
:10874000AC08AD09EEFAEFFB122F6B7402122A305F
:108750000287ECAC08AD09EEFAEFFB122F7102872D
:10876000FB12D31212325FE960030287F1EEFAEFD7
:10877000FB122FBF0287FBA90AEEFAEFFB1232A70A
:10878000806A12BB4064027068E50A700A12DACC93
:108790007003A3E0697064EEFAEFFBA90A12322FAE
:1087A000804A12DACC7003A3E069704512BB4064C2
:1087B00002703EEEFAEFFB123217803F9005D312A3
:1087C000CB656037EEFAEFFB12C5CF124872802BF3
:1087D00012DACC7003A3E0697017EEFAEFFB1232E5
:1087E000B38018EEFAEFFBA90A1232BFE9F50A804E
:1087F0000A750A007AD37B00124105A90A02D0F15A
:1088000074F412242A74DB122AC48A088B098A821F
:108810008B83A3A3E0F91231518A0A8B0BAE0AAF06
:108820000BEE4F7003028931850882850983A3A866
:1088300082A983E0C0E012C84FD0E012E66C64F178
:108840006033850882850983A3E064CD60278508AD
:1088500082850983A3E0641A601B850882850983E9
:10886000A3E064E9600F850882850983A3E064E1E1
:108870006003028A1B900902E06007640160030242
:10888000894A8E828F83A3A3A3A3A3A3A3E0540842
:10889000700302894A8E828F83A3A3A3A3A3A3A3F9
:1088A000A3A37405F0900902E0600464017053858D
:1088B0000882850983A3E064E960479005D712CB5D
:1088C00065600612C5CF1248729005D912CB65605B
:1088D0003190053EE0A2E1502912CD3DA3A3A312A1
:1088E000B0408882898312D31F12334FEA4B601243
:1088F000850882850983A3E0F99005D912C5CC12B9
:1089000048728E828F83A3A3A3A3A3A3A3A3A3E0F0
:10891000640270108E828F83A3A3A3A3A3A3A3A337
:10892000A37406F0850882850983A3A3E0F91231B8
:108930002D12311B900902E06402700990152E126D
:10894000D31F12308574250298447900123127E92B
:108950007003028A1B900902E06007640160030251
:1089600089F090053EE0A2E140030289F012CB605D
:10897000607E8E828F8312D31F7404122A8E12CDD2
:108980005A1231A5850882850983A3E064E9702025
:10899000128B19122A06850882850983A3E0F50A3D
:1089A000780A122A0612D5031231DB7402122A3019
:1089B000740D122CAF12CB5612E99112C8817409B2
:1089C000122CAFE06004794080027900740F122C01
:1089D000AF12B040740D122CAF12D31F122F65E9E5
:1089E000600E8E828F83A3A3A3A3A3A3E04420F0F1
:1089F000EE2404F50AE43FF50B8E828F8312ACD28D
:108A0000E0F9850A82850B8312D31F12450D850A72
:108A100082850B83EAF0A3EB0288A485088285098E
:108A200083A3E0C0E07402122CAFD0E012A4B8EE31
:108A3000F0A3EF128B36C0E07403122CAFD0E0121B
:108A4000E266E0AA18AB19702E122EAB900902E074
:108A50006004640170247402122CAFE0701C128B4D
:108A60002A12325FE970369005D712CB65602E125C
:108A7000C5CF12487280031232357402122CAFE057
:108A800064E97019128B19122A06750AE9780A121C
:108A90002A0612D5031231DB7402122A3090090221
:108AA000E060076401600302890290053EE0A2E1F4
:108AB00040030289028E828F83A3A3A3A3A3A3A34F
:108AC000A3A3E0640270398E828F83A3A3A3A3A320
:108AD000A3E05404602A128B2A12325FE98E828F3F
:108AE00083700F12C5CC74FFF0A312ACED740502B5
:108AF0008923A3A3A3A3A3A3A3A3A37403028923EA
:108B0000850882850983A3E064E96003028902EE97
:108B1000FAEFFB1232C50289028E828F8312D0E0F7
:108B2000E8FAE9FB750A01780A228E828F8312B275
:108B30000BFAA3E0FB22F0E50812ED8E3509F58370
:108B4000E02274F412242AEAFEEBFF75080075098E
:108B5000008E828F83A3A3A3A3A3E0603B750808C4
:108B600012D31279FF1247838B0BEA450B60107505
:108B7000082C8E828F83A3A3A3A3A3E0D2E0F08E60
:108B8000828F83A3A3A3A3A3E05403640160030221
:108B90008C4C430811028C4CEE241812BB436049E4
:108BA000EE241A12BB436003F4701D12DACC70037A
:108BB000A3E0697006750822028C4C900553E064AE
:108BC000046003028C4C801CEE241BF582E43F12EF
:108BD000B628241A12BB43FAEE241912981C122F3D
:108BE000D1E97068750901806312D31212325FE90E
:108BF0006402700375080112DACC7003A3E0697097
:108C000006E508D2E1F508E50860158E828F83A39A
:108C1000A3E07006E508D2E58004E508D2E6F50891
:108C200012D31212325FE964017006E508D2E0F552
:108C3000088E828F83A3A3E0601212B02AF9123249
:108C40003BE964016006E508C2E0F508900902E02E
:108C5000600464017012E508A2E1400CE509A2E09D
:108C60004006E508D2E7F50802BED974EC12242AC2
:108C700074CD122AC4EAFEEBFF851882851983128F
:108C80009B38751000751100750900900902E064A9
:108C900002701C8E828F83A3A3A3A3E060119015A2
:108CA0002C12CB65600990152C12D31F12308574DD
:108CB00005122A8E8E828F83A3A3A312CB5812D3C0
:108CC0001D1231A5E97003028DEE79017407122C93
:108CD000AFE0C394024001197409122CAFE0C394B1
:108CE0000240027900740E122CAFE064F87003A306
:108CF000E0F47003028DEE740E122CAFE064F97094
:108D000003A3E0F47003028DEE740E122CAFE06446
:108D1000FA7003A3E0F47003028DEE740E122CAF10
:108D2000E064FB7003A3E0F47003028DEE7408129C
:108D30002CAFE0F8900541E0686003028DEEE9A2F7
:108D4000E04003028DEE12B88F7424122CAF12C9CA
:108D5000BA241C12B8927412122CAF12C881740B70
:108D6000122CAFE0601D741C122CAFE0FD740612D3
:108D70002CAFE0FC8E828F8312D31D7901122D0758
:108D8000E9703D7405122A86123097E9F508740BD4
:108D9000122CAFE0702E90053BE06028742255083D
:108DA0006422602074425508644270147422122CAC
:108DB000AF129733600E7422122CAF1297396004F1
:108DC0007ACF802CE9A2E6506E900902E06004643C
:108DD00001702590053EE0A2E1501D7422122CAFD7
:108DE00012B0331228C601010A0F8E00EE8D7AD31D
:108DF0007B001241050297177422122CAF12B03378
:108E000024FD600B14600824FD600424FD70DF74F1
:108E100022122CAF12977E700E7422122CAF12C544
:108E2000CEA3E0640D60107405122A8612329BE90D
:108E300064017003029717EE242DF582E43FF58359
:108E4000129E107003A3E069701E750A00780A1262
:108E50002A06780A122A06EE242F12981C12974A24
:108E60001231DB7402122A30740B122CAFE0700343
:108E7000028F1512974A12334F8A0A8B0BEA450B61
:108E80007003028FBE7406122CAFE0F88E828F83BF
:108E9000A3A3E028F8A3E03400F9E8240D129721F9
:108EA000F88A828B83A3A3A3E068600FE88A828B91
:108EB00083A3A3A312DBB0129784F0790474061283
:108EC0002CAF12A2A7E02AF8A3E034008882F58331
:108ED000A3AA82AB83123B538A0C8B0D8C0E8D0F91
:108EE000850A82850B83A3A3A3A3780C12299E4035
:108EF000030297179080C8780C122B7A850A828516
:108F00000B83A3A3A3A3E50CF0A3E50DF0A3E50E4B
:108F1000F0A3E50FF0900902E064026015E060073D
:108F20006401600302905890053EE0A2E150030204
:108F30009052900553E064046008E0640960030205
:108F40009717E508A2E54003028FF9EE242F12BB24
:108F500043C0E07402122CAFD0E01297A4C0E074BA
:108F600003122CAFD0E012979CC0E07404122CAF17
:108F7000D0E0F07416122CAFE06401702674101269
:108F80002CAF12973F7003A3E0697017740E122C78
:108F9000AF12D31F12325FE9640270077416122CED
:108FA000AFE4F012979212283D7406122A8E7409CB
:108FB000122A86122EB17404122A300297179005D5
:108FC00098E064016003028F157422122CAF12978F
:108FD000337009E508A2E65003028F157412122CB3
:108FE000AFE0F47003A3E0F4600CEEFCEFFD740559
:108FF000122A861230A3029717A2E6505274221248
:109000002CAF12CD547016741C122CAFE064027099
:109010003E7405122A86790012322F803274221291
:109020002CAF1297397014741C122CAFE0640470CA
:109030001E7405122A8612322380147422122CAF59
:1090400012977E700A79007405122A861232A702DE
:109050009717900902E06013E0640160030297171C
:1090600090053EE0A2E140030297177416122CAF60
:10907000E0601CEE240212B5EF129CD91412AE6F00
:10908000129CD9C0E07416122CAFD0E0F07006E547
:1090900008C2E7F508E508A2E35061751110A2E2E5
:1090A0005018740A122CAFE054E3F0740A122CAF7B
:1090B000E0131313541FF8E0802CA2E4502A740A22
:1090C000122CAFE01313543F5407F860097407687B
:1090D000600B18E87007C3E508C2E7F508E833330A
:1090E00054FCF8E054E348F0740A122CAFE0C0E0FE
:1090F0008E828F83A3A312ADBFD0E0F0900553E022
:1091000064046008E0640960030291D8740E122CB4
:10911000AF12DAD97003A3E069601F740E122CAF8E
:1091200012D31F12325FE96402600F740A122CAF6F
:10913000E05403640160030297177407122CAFE038
:109140007041EE242F12BB43C0E07402122CAFD04A
:10915000E01297A4C0E07403122CAFD0E012979CE9
:10916000C0E07404122CAFD0E012978D12283D7429
:1091700006122A8E7409122A86122EB17404122A3B
:109180003080527422122CAF12CD547016741C12FF
:109190002CAFE06402703E7405122A867900123208
:1091A0002F80327422122CAF1297397014741C1253
:1091B0002CAFE06404701E7405122A8612322380DC
:1091C000147422122CAF12977E700A790074051263
:1091D0002A861232A702971774615508700302920B
:1091E000DFE508A2E0506D12B0377405122A86122E
:1091F0003001E9705C1231D5E9F5097416122CAF13
:10920000E0700F7410122CAF12973F7003A3E06947
:109210006042A90912B0377405122A86123007E994
:109220006024E508A2E3500C85188285198374FF39
:10923000F0A3800C740E122CAF12975CE8F0A3E937
:10924000F0751004800EE508C2E5F5087509008088
:109250000353089FE508A2E5503FEE242F12BB43BD
:10926000C0E07402122CAFD0E01297A4C0E07403E7
:10927000122CAFD0E012979CC0E07404122CAFD037
:10928000E012978D12283D7406122A8E7409122A54
:1092900086122EB17404122A30E508A2E6400302B9
:1092A00095B2A818A919880A890B780A122A02A966
:1092B0000912972A122A8612308B7402122A30E978
:1092C000F50970030295B27422122CAF12B0336408
:1092D0000160030295B274104510F5100295B27446
:1092E00007122CAFE06401705D7422122CAF12B033
:1092F000336405701EA818A919880889097808120E
:109300002A02129728122A8612308B7402122A30EF
:109310000297177422122CAF12977E7029740E12C6
:109320002CAF12D31F122DA9E9601BA818A9198808
:109330000A890B780A122A02129728122A861230FA
:109340008B7402122A307416122CAFE07025740749
:10935000122CAFE06401700C7422122CAFE0F812F2
:10936000977E600CEEFCEFFD7405122A861230A386
:10937000029717123121E96003029717741D122C0E
:10938000AFE0700302942D7420122CAF12B0407421
:109390001F122CAFE0FA741E122CAFE0F9122FD17D
:1093A000E9607D741F122CAFE0701E740E122CAF9A
:1093B00012975C12BC26FAA3E0FB122DB58B0BEAC8
:1093C000450B60030295AC80517420122CAF12D370
:1093D0001F741F122CAFE0F9122FCB85188285194C
:1093E0008312DA137808740D122CAFE06002781043
:1093F000740C122CAFE06004740828F8740A122C64
:10940000AFE0600108088E828F83A3A3E028FAA34F
:10941000E034008A82F583E014F07510400295ACC8
:109420007508007808122A06790B029565740E12E9
:109430002CAF12C87D7409122CAFE0600302958036
:10944000E508A2E350030295807407122CAFE06494
:1094500001607A790085188285198312D31F123032
:10946000258A0A8B0BA80AA90BE849601C88828907
:1094700083A3A3A3A3A3E06401605288828983A38A
:10948000A3A3A3A3E064026044EE242D12B03A85A6
:10949000188285198312D31F12334F8A828B83E57A
:1094A000824583600FA3A3E0F912336DE96005C321
:1094B000940840197410122CAF12D31F122DA9E971
:1094C000700302955B7409122CAF7404F0E4F50983
:1094D0007809122A06741E122CAFAC82AD83740F69
:1094E000122CAF12D31F740A122CAFE0F9123037CE
:1094F0007401122A30E9600F7510208E828F83A3C9
:10950000A312B033543FF0741D122CAFE0602374EB
:109510000E122CAF12B040741E122CAFAA82AB8375
:1095200012319F85188285198312DA137440451011
:10953000F5107407122CAFE0640160157900741007
:10954000122CAF12B040740E122CAF12D31F122F78
:10955000D7E508A2E35037794080357508007808D0
:10956000122A067902740F122CAF12B04074111235
:109570002CAF12D31F1232A17401122A3002971796
:10958000E508A2E340030294CD74400294CE790032
:109590007410122CAF12B040740E122CAF12D31FE5
:1095A000122F65E9600674204510F5101231D5E9D7
:1095B000F509851882851983E064FE7003A3E0F441
:1095C00070037509009008F5E06401600302966578
:1095D000EE241312BB43F47003A3E0F4700302966D
:1095E00065740E122CAFC3E094F9A3E094FF50759C
:1095F00012B88F7410122CAFE0687003A3E069609A
:10960000647410122CAF12D31F122DB58A0A8B0B63
:10961000A80AA90BE849604D88828983A3A3A3A364
:10962000E06401600D88828983A3A3A3A3E06402A0
:1096300070337426122CAF740112DF89F8A3E0F99D
:109640007431122CAF12C8817426122A86122D7919
:10965000E960127429122CAFAA82AB83122DC7E9DC
:109660006003123E29E508A2E74003029717E509C7
:1096700070030297178E828F83A3A3A3A3E0FA7BC4
:1096800000123BFB8A0A8B0BEA450B70030297170B
:10969000EE2404F512E43FF5138E828F83A3129714
:1096A0006C1229FE851282851383E0FC7D00123B3B
:1096B0003B7403122A307407122CAFE0C0E074022E
:1096C000122CAFD0E0F07403122CAFE4F0A3F074CE
:1096D00002122A7E880C890D780C122A0278101248
:1096E0002A02E509F5087808122A0612CA6112282A
:1096F00041851282851383E0F97407122CAF12B0F2
:1097000040AA0AAB0B1231937407122A30E96007A2
:10971000AA0AAB0B123C017433122A307F0C0226CA
:10972000B9F582E412E7B622790012CA6512B04494
:1097300074072212B20B64062212B21164072212BD
:10974000D0E0EE241312B60C6822EE242BF582E44E
:109750003FF58312B62E241312983722E012976138
:1097600022F8A3E0F985188285198322A31297763F
:10977000750E00780C22E0F50CA3E0F50D2212B274
:1097800011640322A3E4F0A3F0A3F0A322F0129744
:109790009222EE2425F582E43FF58322F0EE243177
:1097A00012B60C22F0EE243012B60C2274F41224FD
:1097B0002AEAFEEBFF8C088D099008F2E0600F1298
:1097C000DACC7003A3E0697005122F53804C790046
:1097D00012D3121230258A828B83E5824583603250
:1097E000A3A3A3A3A3A3E054186027E508241C1295
:1097F000C864122841E508241312C864122841EEF7
:10980000241812981C12982112303D7404122A3028
:1098100080087900129821122F7D802B12B60CF946
:10982000228E828F83A3A3A3A3A3A3A3A3A312B671
:109830002E240B12983722F582E43FF58312E98C2F
:10984000FB227418122A307F040226B974F0122405
:109850002A74EA122AC48A0A8B0BEA2402F50EE45F
:10986000350BF50F0A0AFB122DBB8A088B09AE08CF
:10987000AF09750801850A82850B83A3E0F5097598
:109880000C01AC0EAD0F740B122CAFAA82AB83127D
:1098900045257413122CAF129B387415122CAF741B
:1098A00002F07408122CAFE4F09014D5E0700EEEC4
:1098B0004F700AE50970067508C3029A8C9005532B
:1098C000E0640860067508C2029A88850A82850BE2
:1098D00083A3A3A3A3A3A3A3A3A3A3E0A2E1500EE6
:1098E000A2E35005750C04800C750C038007A2E3FD
:1098F0005003750C02EE4F70030299988E828F838D
:10990000A3A3A3A3E06404600D8E828F83A3A3A30B
:10991000A3E06403700C7404650C602C7403650C84
:1099200060268E828F83A3A3A3A3E06402600D8EC2
:10993000828F83A3A3A3A3E0640170357402650C36
:1099400060067401650C701C8E828F8312D31F1207
:10995000327DE970438E828F8312A623122CAF12C0
:10996000C88180348E828F83A3A3A3A3E0640260A6
:109970000D8E828F83A3A3A3A3E06401700A8E825D
:109980008F8312A78A124872E50A2402FAE4350B83
:10999000FB122DC77E007F007413122CAFE064FE13
:1099A0007003A3E0F4704E122D85E97048E509605C
:1099B00023900590E06402701B9014DC12D31F12F8
:1099C000327DE9700F9014DC12A623122CAFE8F060
:1099D000A3E98020850A82850B83A3A3A3A3A3A365
:1099E000A3A3A3A3E05402F9122F8F7413122CAF78
:1099F000EAF0A3EBF07413122CAFE064FE7003A343
:109A0000E0F470057508C7807FE509F50D780D1243
:109A10002A06850A82850B83A3A3A3A3A3A3A3A3DA
:109A2000A3A3E0F9E50A2402FCE4350BFD7414124B
:109A30002CAF12D31F122ED57401122A30E97048B0
:109A4000A90CE50A2402FCE4350BFD7413122CAFBB
:109A500012D31F122D978A0E8B0FAE0EAF0FEE4F43
:109A6000601E74026509700D8E828F83A3A3A3A369
:109A7000A3E0D2E3F07415122CAFE4F0F5088008EF
:109A80007413122CAF129B38E5097009AA18AB1990
:109A9000124603800AFCA90CAA18AB1912321DE960
:109AA000F8EE4F6053E50960208E828F83A3A3A355
:109AB000A3A3E0D2E6F074026509700D8E828F8355
:109AC000A3A3A3A3A3E0D2E5F0850A82850B83A319
:109AD000A3A3A3A3A3A3A3A3A3E0A2E6500D8E82F6
:109AE0008F83A3A3A3A3A3E0D2E7F08E828F83A3E7
:109AF000A3A3A3A3A3E004F0E5087003E86034FC8B
:109B00007D007A017B10124507EE4F600CE50A24B8
:109B100002FAE4350BFB122DC77413122CAFE0646C
:109B2000FE7003A3E0F4600B7413122CAF12A78A2B
:109B3000124872741602C10974FEF0A304F0227474
:109B4000F712242A74F7122AC4EAFEEBFF90055399
:109B5000E06403600DE064016008E06409600302F2
:109B60009C698E828F83A3E06003029C3F7C007D12
:109B7000007A027B00124507129C6E8A828B831248
:109B8000B89890054412C88179531245F77900902E
:109B9000055112D31F122ECF900553E064096009BE
:109BA00090055112D31F1233498518828519837489
:109BB0000112C9CB79421245F79005537404F07431
:109BC00001122A86794A1245F17401122A8E7A49C5
:109BD0007B05124525900902E060046401701F9026
:109BE0000547E064FE7003A3E0F4602A7900740185
:109BF000122A8E90054712D31F122D978018E06409
:109C000002701390054412B0407A037B001245079E
:109C100012A54A12450790053EE0A2E35004D2F097
:109C20008002C2F012C9C179521245F7900902E0D0
:109C30006402703290152A12D31F12308580278E4D
:109C4000828F83A3AE82AF83FC7D007A037B1012E8
:109C500045078E828F83E0F990055112D31F122E93
:109C6000CF900553E4F01230F1740902B138EE24BC
:109C700002FAE43FFB22C082C08390051412CB6538
:109C8000701F900553E014600924FC600A14600CF6
:109C9000800F90051D8034900519802F90051B8042
:109CA0002AE849600890051512A2B0700C8A828BD0
:109CB00083A3E0F9122EB7801D900514129CD9647D
:109CC0000270051232DD800E9005D512CB6560065C
:109CD00012C5CF12487202C144E0F8129CDF22A3E1
:109CE000E0C82406F582E438F583E02274F41224F7
:109CF0002A74FB122AC48A088B097A0F7B00123B54
:109D00005F8A0A8B0BAE0AAF0BEE4F7003029E0BFD
:109D10008E828F83740212C9CB79501245F1850867
:109D200082850983A3E06003029DEE900551E0F473
:109D30007003A3E0F46044900551E064FE7003A357
:109D4000E0F46037851882851983129E107003A392
:109D5000E0696027850882850983A374EAF07A4464
:109D60007B0579531245F77A477B05794B1245F706
:109D70007A517B0579501245F780738518828519D1
:109D80008312DB9D12C8817A447B0579531245F119
:109D900090054412ACE312C8817A477B05794B12D7
:109DA00045F17A467B0579E11245F1900558E0C30B
:109DB000940F501D900546E0C0E07402122CAFD005
:109DC000E0F07404122CAF7401F004122A861246DB
:109DD0001B750A00780A122A06780A122A069015BC
:109DE0005FE0F912A9D21231DB7402122A30850821
:109DF0008285098312D632A3F09005537403F0EEE6
:109E0000FAEFFB90059EE0F9123B6B740502984453
:109E100012DBA1E0682274F412242A74E8122AC426
:109E2000EAFCEBFD8C828D83A3A3A3A37808122CFC
:109E3000587808122BFA9005547808122BB37F7FBC
:109E40007E7F79009005547808122C58E978081222
:109E50002A65E508A2E05029780090059F801485C6
:109E60000882850983A3A3E069700108E50824142A
:109E700012C86412A6AD70E7E8C39F5004E8FFE97A
:109E8000FE09E9C3941B40BC8C828D83A3A3A3A3CA
:109E9000122C8CE8494A4B607DEC2404F508E43D23
:109EA000F509850882F583122C8C900554122C98A4
:109EB0007C187D007900AA18AB19123B47850882EF
:109EC000850983122C8C851882851983122C98742D
:109ED00004122CAF7401F090055AE0C0E074051232
:109EE0002CAFD0E0F07407122CAFE412C9CB1246AD
:109EF0000F807090055112D31F122F058A0A8B0B09
:109F0000A80AA90B900551E8F0A3E912CB7268707A
:109F100003A3E069602D90059F12A6AD602585081A
:109F200082850983129E107003A3E069700C850876
:109F300082850983A3A3E06E60B9E508241412C8E2
:109F40006480D6EE900546F01230D3E96015900596
:109F500053E4F090051F12CB65600879C412C5CF99
:109F600012487202984274F412242A74E8122AC425
:109F70008A828B83A3A3A3A3A3A3A3A3A312B898AA
:109F8000E8FAE9FB79009005547808122C58E97832
:109F900008122A65E508A2E05031EA29F582E43B7F
:109FA000F583E0F89014DBE0C398501F7508017545
:109FB0000900750A00750B00E978081229BD7808B8
:109FC000122BFA9005547808122BB309E9C3941B9D
:109FD00040B4900554122C8CE8494A4B604E7C18D2
:109FE0007D007900AA18AB19123B47900554122C3A
:109FF0008C851882851983122C987404122CAF74E6
:10A0000001F07407122CAF7401F090055AE0C0E023
:10A010007405122CAFD0E0F07407122CAFE412C913
:10A02000CB12460F9005537406F0801E900553E442
:10A03000F0FCFD7A047B1012450790051F12CB65DA
:10A04000600879C412C5CF12487202984274F512A2
:10A05000242A74D1122AC48A088B098A828B83121B
:10A06000B89C741C122A8E8A828B83A3A3A3A3A3F9
:10A07000A3A312B1E712D31A123103741C122CAF2E
:10A08000E0702C850882850983A3A3A3A3A3A3A3BF
:10A09000A3E0C3940B40188E828F83A3A3A3A3A332
:10A0A000A3A3A3E06402700712C84FE0F4600302A8
:10A0B000A2A2900553E06402700302A184E064064A
:10A0C000700302A18490051412CB65600812A2B03F
:10A0D000700302A1B9900553E064086008E06404CD
:10A0E000600302A2A2741E122CAF12A2A7A3A3A304
:10A0F000A312B89C900514E0F8496007129CDF6435
:10A10000026077900551E06E7003A3E06F60030278
:10A11000A2A274016A60167423122CAFAC82AD83C4
:10A120007A657B0512451FE9600302A2A27A007BD3
:10A130000290059EE0F9123CD3EA4B4C4D600302BD
:10A14000A2A2900554122C8C851882851983122C9A
:10A150009890055AE0C0E07404122CAFD0E0F0747F
:10A1600005122CAF7401F07406122CAF740212C9E0
:10A17000CB122E3FE9600302A29FEEFAEFFB1232F0
:10A18000D702A2A290051412CB65702D7508007835
:10A1900008122A067808122A06EE2410F582E43FF7
:10A1A000F58312CB59A3A3A3A3A3A3A3A3A312AD87
:10A1B000B41231DB7402122A308E828F8312B89867
:10A1C0007407122CAFE8F0A3E912ACED12B8987442
:10A1D00009122CAF12C9BA240D12BB43C0E0740B94
:10A1E000122CAFD0E0F012C84F12ACC6740F780832
:10A1F000122C3A740C122CAFE508F07420122CAF1C
:10A20000E0C0E0740D122CAFD0E0F07422122CAF3D
:10A21000E0C0E0740E122CAFD0E0F0741D122CAF31
:10A22000E0C0E07410122CAFD0E0F0741E122CAF1E
:10A23000E0C0E0740F122CAFD0E0F0EE241012BB9F
:10A2400043C0E07411122CAFD0E0F07421122CAF97
:10A25000E0C0E07412122CAFD0E0F0742E122CAFDC
:10A26000E0C0E07413122CAFD0E0F07423122CAFD6
:10A27000A982AA8389088A09750A0078081229FE2A
:10A280007C087D007417122CAFAA82AB83123B3B73
:10A290007403122A307407122A86122EC980031200
:10A2A0002E45742F02EEDCE0FA8E828F83A3A32268
:10A2B000129CE064012274F612242A74C9122AC482
:10A2C0009005CF12CB65600612C5CF12487290057B
:10A2D00053E06408700302A373900590E064027079
:10A2E00023904E02E493900535F0904E02E4939053
:10A2F0000533F090055C7401F012978404F0A3E438
:10A30000F0A3806C900564E0F874FB28F582E434D7
:10A310000DF583E0FA900535F074FC28F582E434FD
:10A320000DF583E0F9900533F07508FF7509FFEA34
:10A330007808122BC6E508F4FCE509F4FD3395E036
:10A34000FE90055CECF0A3EDF0A3EEF0A3F0750831
:10A35000FF7509FFE9C39A7808122BC6E508F4FCDB
:10A36000E509F4FD3395E0FEA3ECF0A3EDF0A3EED8
:10A37000F0A3F07C237D0079007414122A86123B2E
:10A3800047900564E07009741E122CAF74018006BA
:10A39000741E122CAFE412A4B8740FF09014DA12E9
:10A3A000C9CB79461245F77401122CAFE4F0901531
:10A3B00039E0C0E07402122CAFD0E0F0900541E02B
:10A3C000C0E07403122CAFD0E0F07404122CAFE4A0
:10A3D000F07405122CAFE4F07407122CAFE4F09087
:10A3E0000564E0C3940F500CE0C0E07406122CAF7B
:10A3F000D0E080077406122CAF740FF07C657D05E9
:10A400007408122CAFAA82AB831245257C037D0011
:10A4100079FF7410122CAFAA82AB83123B479005D0
:10A420009DE0C0E07413122CAFD0E012C7C37401DA
:10A43000122A861230FD7AA17B0579451245F71262
:10A44000320B900558E0C0E0741C122CAFD0E0F045
:10A45000900559E0C0E0741D122CAFD0E0F09005DB
:10A4600046E0C0E0741A122CAFD0E0128481741858
:10A47000122CAF12C8817420122CAFE4F090055B4F
:10A48000E0C0E0741F122CAFD0E0F07434122CAF97
:10A49000E4F07429122CAFE4F07A447B057953126E
:10A4A00045F77A477B05794B1245F77414122A86D3
:10A4B000124615743702C4B512A4BC22F085188266
:10A4C00085198322C082C0838A828B83A3E0900592
:10A4D000536004E4F080707408F0900564E0702824
:10A4E00090051F12CB656008790012C5CF12487223
:10A4F00090055112B0407A057B0012450790055136
:10A5000012D31F12334980187900122EC3900544CC
:10A5100012B0407A067B0012450712A54A12450781
:10A520009005DB12CB65601F9008F6E064017017A0
:10A530009080C012283D7A007B4090059EE0F91281
:10A540003CC17404122A3002C14490054712B04441
:10A550007A047B002274F412242A74EA122AC4EAD0
:10A56000FEEBFF129C6E122DBB8A088B09EA45098F
:10A57000700302A61E8A828B83A3A3A3A3E06401B7
:10A5800060278A828B83A3A3A3A3E06402601A8A54
:10A59000828B83A3A3A3A3E06403600D8A828B83D1
:10A5A000A3A3A3A3E064047075EE2402FCE43FFDC2
:10A5B000740B122CAFAA82AB8312452585088285C5
:10A5C000098312A623122CAF12C8817415122CAF66
:10A5D0007401F07408122CAFE412C9CB1246098939
:10A5E0000AAC0A7D007A077B001245078508828540
:10A5F0000983A3A3A3A3A3E0C2E012C0B0A3A374E2
:10A600000112E2755001097A027B00122243E885AB
:10A610000882850983A3A3A3A3A3A3A3A3F074160D
:10A6200002984412D0E074132274F212242A74F8AF
:10A63000122AC4EAFEEBFF8C0A8D0B890C90804233
:10A64000AC18AD19740812295EF50DEEFCEFFDAAE9
:10A6500018AB1912451FE97003750D0190059F8015
:10A660001AEEFCEFFDE508240BFAE43509FB124570
:10A670001FE97023E508241412C86412A6AD6024F3
:10A68000E50DA2E040DB850882850983E0650A705C
:10A6900004A3E0650B70DD850882850983A3A3E030
:10A6A000650C70D0AA08AB09740802D0EE12ACCACF
:10A6B000E508450922C082C08390059F02C141740C
:10A6C000F712242A90059F12E98C800C12D3AB124A
:10A6D000B89F123C01EEFAEFFBEA4B70EF90059F3A
:10A6E000E4F0A3F002B13B74F412242AEAFEEBFF7B
:10A6F000EE241312BB436403700CEE240BFAE43F08
:10A70000FB122DBB800EE06402707C12C84F12D386
:10A710001F122DB58A088B09E508450960698E82EC
:10A720008F83A3E0700F850882850983A3A3A3A369
:10A73000A3A3E4805164F1600A8E828F83A3E06456
:10A74000E17027850882850983A3A3A3A3A3A3E0BF
:10A750006401701685088285098312A78A124872DF
:10A76000EE240BFAE43FFB122DC78508828509838E
:10A77000A3A3A3A3A3A3E0600E850882850983A3F6
:10A78000A3A3A3A3A314F002984712983D90052D0C
:10A7900012C8952274F112242A8A088B09ECFEED66
:10A7A000FF890A12D61FEEF8EFF9A30EAF838A8253
:10A7B0008B83A3A3E0C454F0FA88828983E04A1211
:10A7C000A87512D63312A870E0333354FCF88E8289
:10A7D0008F83E04812A870A3E033333354F8F88E27
:10A7E000828F83E048F0EEF8EFF9A30EAF8385087F
:10A7F000828B83A3A3A3A3A3A3E0A2E0E433131358
:10A80000FA88828983E04AF0E5082407F50CE435EC
:10A8100009F50D750E00780C1229FE7C087D00EEFE
:10A82000FAEFFB123B3B7403122A30EE2408FE5071
:10A83000010FE508240FF50CE43509F50D780C122D
:10A8400029FE7C037D00EEFAEFFB123B3B74031202
:10A850002A30E50AC3940F4012E5082412F582E479
:10A8600012DEA98E828F83A3A3A3F07F070226B9ED
:10A8700012A875A322F08508828B83A3A3A3227458
:10A88000F112242AEAFEEBFF890A8C088D098E82D8
:10A890008F83E08C828D8312B63EAE82AF83E0124E
:10A8A000BEDE12C0CCC412BEDE12A949E054038C35
:10A8B000828D8312C0CAA2E2E4338C828D8312C0DF
:10A8C000C9131313541F12BEDE12C0C8A2E7E4332B
:10A8D0008C828D83A3A3A3A312A9498E0C8F0D751F
:10A8E0000E00780C1229FE7C087D00E5082407FA8A
:10A8F000E43509FB123B3B7403122A30EE2408FEB8
:10A9000050010F8E0C8F0D780C1229FE7C037D00F8
:10A91000E508240FFAE43509FB123B3B7403122AC5
:10A9200030E50AC3940F40158E828F83A3A3A3E062
:10A93000C0E0E508241212C864D0E08008E50824CD
:10A940001212C864E4F002A86BA3A312B6420EAFC1
:10A95000832274F512242A8A088B098A828B83A3A6
:10A96000AE82AF83E0F9122EED8E828F83E064EB2E
:10A970006024850882850983A3E064E16018850866
:10A9800082850983A3E064F1600C850882850983D0
:10A99000A3E0641A7009850882850983A3E4F09016
:10A9A000152A12D31F123085750A01780A122A0659
:10A9B000850882850983A3E0F5087808122A0679BC
:10A9C0000012A9D21231DB7402122A3012311B029A
:10A9D000EEDF90055112B04490054712983D22C019
:10A9E00082C083E99005B17003E480027401806540
:10A9F000E0F902C14474F712242AEAFEEBFF8E82CA
:10AA00008F8312C99312D9F812DA1312325FE98ECA
:10AA1000828F83600512AA26800312AA3B12AA44E1
:10AA200012462702B13B12AA2DE4F0A322E0F8A3BC
:10AA3000E0C8240DF582E438F5832212AA2D7401B2
:10AA4000F0A3E422F07C737D308E828F8312983DD8
:10AA500022EAF0A3EBF002C14474F612242A900516
:10AA6000B1E0701B7C0079017A007B0012314BEA67
:10AA70004B600C8A828B8312CB65600312307902A3
:10AA8000C4B8C082C0837904123145E9F8904DFE04
:10AA9000E493C398401079FF123145E9F8904DFCDA
:10AAA000E493C398500479018002790002C1447490
:10AAB000F012242A8A088B09890B750C008A828B74
:10AAC00083A3A3A3A3A3A3A3A3E0F91231518A0EE6
:10AAD0008B0FAE0EAF0F750A01EE4F600302AB7F16
:10AAE00085088285098312ACD2A3A3A3A3A3A312D2
:10AAF000BC1812D31F1231398A0C8B0DAE0CAF0D5E
:10AB0000EE4F700302ACB88E828F83A3A3A3A3E49D
:10AB1000F0A3F0E508240CFAE43509FB8A828B8364
:10AB2000E0C0E012E26BD0E0F012326BEE240D12C6
:10AB3000DA0DE50812DE9B350912B89612B600123E
:10AB4000C881750C01EE240612BB47547FF0A3E0C8
:10AB500054FC12E66C5404600302ABF6901532E02C
:10AB6000F50875090074077808122BC68E828F834A
:10AB7000A3A3A3A3A3A3E04508F0A3E04509F08E97
:10AB8000828F83A3A3A3A312ACC474077808122CEA
:10AB90003AE5085407F508E50B606B8E828F83A3B6
:10ABA000A3A3A3A3A3A3A3A3740212C0CD12AFAF08
:10ABB000600B90053F12ACE3A3A312C881E50870B7
:10ABC0000302AC84EE240612ED61547FFCA3E05432
:10ABD000FCFDE50824FFF508E434FFF50974077867
:10ABE00008122BC6EC4508F8ED4509F98A828B83DB
:10ABF00012C88102AC848E828F83A3A3A3A3A3A3D4
:10AC0000E0448002AB7EE5087005750A0080758E11
:10AC1000828F83A3A3A3A3A3A3E05420600C123BC1
:10AC200059EA547F7900245F80198E828F83A3A311
:10AC3000A3A3A3A3E05410601A123B59EA540F795E
:10AC400000240A5001098E828F83A3A3A3A3F0A33B
:10AC5000E9800D8E828F83A3A3A3A37401F0A3E4E4
:10AC600012ACED7404F07A207B0090059EE0F9129E
:10AC70003CD3EA4B4C4D700C7A207B0090059EE053
:10AC8000F9123BA1E50CA2E050318E828F83A3A381
:10AC9000A3A312D323F9EEFAEFFB12313FE9601BB5
:10ACA00012B13012CB63600912B21F12D31F123CD3
:10ACB00001EEFAEFFB123C01750A00A90A02C10C71
:10ACC0008E828F83A3A312ACCA22E0F508A3E0F51D
:10ACD0000922A3A3A3A3A3A312B0448508828509D4
:10ACE00083A32212D0E08E828F83A3A32212C87185
:10ACF000A3A3A32274F412242A74F7122AC47E0098
:10AD0000123151EA4B700302ADAD8A828B83A3A34B
:10AD1000A3A3A3A3A3A3A3E06406600302ADAD8A2B
:10AD2000828B83A3A3A3A3A3A3A3E0FF8A828B8325
:10AD300012ADBFE0C0E07408122CAFD0E012B20434
:10AD400012C87E12316FEF54086060851882851931
:10AD50008312B0407A007B001231338B0BEA450B33
:10AD6000704912EED612463F7C007D007A007B00CF
:10AD700080258E828F8312B033F47003A3E0F460D9
:10AD80002A90055112ADB4124639E9641A601C7C50
:10AD9000007D00EEFAEFFB1231338A0A8B0BAE0A0C
:10ADA000AF0BEE4F70CC79001246457E01EEF97480
:10ADB0000902984412B0448E828F8312983D221269
:10ADC000B88A12ADC6222408F582E438F58322C081
:10ADD00082C083EA4B70059005B280068A828B831D
:10ADE000A3A312AFE360258A828B83A3A3A3A3A3AB
:10ADF000A3A3E0540860E5EC4D60158A828B8312B2
:10AE0000B0336C7003A3E06D70D280047A007B00D5
:10AE100002C14474F212242AEAFEEBFF890A8C086C
:10AE20008D097A117B00123BFBEA4B603E8A828BD4
:10AE300083A3A3A3A3A3A3A3A3A3E412B1F8A3E5AD
:10AE40000A12DBB0A3A3A312EFB78A828B83A3A35A
:10AE5000A3A3E4F0A312B21912AE7912DA0012B76A
:10AE60000EE4F012AE6EA3A3F0A3F002D0F1A31291
:10AE7000AE7322F08A828B8322A3F012ED8D3BF514
:10AE800083E4F02274F412242AEAFEEBFF89088C92
:10AE90000A8D0BEE4F700302AF3874016508701213
:10AEA0007901123145E9F8904DFFE493C39850229F
:10AEB00080167404650870147904123145E9F8901D
:10AEC0004DFEE493C398500A7911806E74026508B0
:10AED00070668E828F83A3A3A3A3A3A3A3A3A3E5DA
:10AEE0000812BE4912D6178E828F83A3A3E4F0A363
:10AEF000F09005B212CB6560178003E0F8A312C989
:10AF00009AA3A312AFE388828983A3A370ED800381
:10AF10009005B212DA047A207B0090059EE0F912C7
:10AF20003CD3EA4B4C4D700C7A207B0090059EE0A0
:10AF3000F9123BA17900800279C1029847C082C012
:10AF400083E9F879009005B2801D8A828B83A3A3E0
:10AF5000A3A3A3A3A3A3A3E068600574FF68700183
:10AF6000098A828B83A3A312AFE370DE02C144740B
:10AF7000F712242AEA4B70059005B280068A828B6C
:10AF800083A3A312AFE360208A828B83A3A3A3A32E
:10AF9000A3A3A3A3A3E06970E4EC60108A828B836F
:10AFA000E012AFAF70D780047A007B0002B13B1291
:10AFB000AA2EE0540422C082C0839005B280068A83
:10AFC000828B83A3A312AFE360128A828B83A3A335
:10AFD000A3A3A3A3A3A3E06970E580047A007B0088
:10AFE00002C14412983DEA4B2274F712242AEAFC6B
:10AFF000EBFD9005B280068A828B83A3A312AFE398
:10B0000060218A828B8312B0336C7003A3E06D7071
:10B01000E68A828B8312860E12CA80A2E0E4337025
:10B02000D680047A007B0002B13BEE241DF582E459
:10B030003FF58312B20B22EE2413F582E43FF58331
:10B0400012B0442212B04822E0FCA3E0FD2274F2C8
:10B0500012242A8A0A8B0B8C0C8D0D750800750939
:10B0600000EA450B60309005B280068E828F83A384
:10B07000A312B89FEE4F601EAC0CAD0DEEFAEFFBC5
:10B08000850A82850B83124872E9640170DDEEF84F
:10B09000EFF988088909AA08AB0902D0F179000202
:10B0A00029E274F712242A9005B212B8987C007D28
:10B0B00000800DE8FCE9FD88828983A3A312B8987B
:10B0C000E8496030EA687002EB6970E79005B212F7
:10B0D000D31FE86A7002E96B88828983A3A3700892
:10B0E00012B8989005B2800912B8988C828D83A30B
:10B0F000A312C881804574F712242AEAFEEBFFEE02
:10B100004F602B12316912B225123C018E828F835F
:10B1100012D31F123C0112B13012CB63600912B27C
:10B120001F12D31F123C01EEFAEFFB123C01800B01
:10B13000EE240DF582E43F22122A307F010226B967
:10B1400074F712242A8A828B8312B1F09005B2120E
:10B15000B8987508007E00803388828983A3A3A3F2
:10B16000A3A3A3A3A3A3E0640570180E8882898318
:10B17000E0FFA3E0F5838F82E06C7003A3E06D70C5
:10B1800002050888828983A3A312B898E84970C988
:10B19000904DF012E3C0500890261B12D260400F71
:10B1A0008A828B83A3A3A3A37401F0A3E4800C90F1
:10B1B000053FE0F812B1E7E8F0A3E912B21974050F
:10B1C00012B1F8E0440812B204F47003A3E0F46092
:10B1D0000E90055112D51A124639E9641A70057994
:10B1E0000112464502B13BA312B5E8A3A3A3A322D3
:10B1F00012B20BFCA3E0FD2212B1FC2212DBB8A3B9
:10B20000A3A3A32212AE7312B20B22E0F812B21162
:10B2100022A3E0F5838882E02212B1FCA3A32212CC
:10B22000B130F5832212B22C12983B228E828F838A
:10B23000E0F8A3E0C8241FF582E43822C082C0836E
:10B24000EAFCEBFDEC4D6017EC24FBF582ED34FFDE
:10B2500012CB63700712B296E0F46007123B657977
:10B2600005803090059EE0C0E012B296D0E0F090EC
:10B270004E04E493F97AB47B05123B9BE9640170B8
:10B28000107A007B2090059EE0F9123BA1790080A6
:10B2900002790402C144EC24FFF582ED34FFF5830A
:10B2A0002274F412242AA2AFE433F508C2AF900549
:10B2B000B412B89FEE4F603AEE24FBF582EF34FFF4
:10B2C00012CB637A007B2090059E6007E0F9123B69
:10B2D000A18005E0F9123BA7E4F50AF50B780A1204
:10B2E0002A02EEFCEFFD7AB47B05123B9574021244
:10B2F0002A30E508A2E092AFEEFAEFFB029847741D
:10B30000F012242A74DB122AC4EAFEEBFF750B004C
:10B31000750A007508FE7509FF123121E960030204
:10B32000B5DBEE241512BB43604690154CE0C433E8
:10B3300054E0F8E0333354FC48C0E012D304D0E0CA
:10B3400012B63E12D31E79FF1247838B0DEA450DCC
:10B350006011750B017508FF12B605440412C89EF2
:10B36000D2E0F0900902E0600464017003750A40C5
:10B370008E828F8312D31D12325FE9600312C9716E
:10B38000EE241312BB43700D904DFBE493C0E0120A
:10B39000CA61D0E0F08E828F83E0A2E750045403AC
:10B3A0008019EE241412BB437012900530E0C0E007
:10B3B00012ED3FD0E0F0900530E004F012ED58704F
:10B3C000199008E1E0600D90053BE0700D8E828FD2
:10B3D00083E07006EE241112C974900902E0600443
:10B3E0006401704890053EE0A2E15040E50BA2E008
:10B3F00040218E828F8312D31D12325FE9602D8E21
:10B40000828F83E0600DEE240B12B02DF912323BD7
:10B41000E9601912B614700302B58CEE241312ED14
:10B420005B600302B58C12B60554FBF08E828F83ED
:10B43000E06401700DEE240B12B02D640270031253
:10B44000B62112B614600302B505E50BA2E0500365
:10B4500002B505900902E060076401600302B505CA
:10B4600090053EE0A2E1400302B505E50AF50B7840
:10B470000B122A06EE2406FCE43FFD8E828F831217
:10B48000D31DEE241212981C1230377401122A3088
:10B49000E9600612C97112B61A8E828F83A3A3A324
:10B4A000A3A3A3E0603CEE2402F50CE43FF50D8578
:10B4B0000C8212B6282407FAE43FFB12319F8A0857
:10B4C0008B09850C82850D83E065087004A3E06517
:10B4D00009700C8E828F83A3A3A3A3A3A3E4F0120D
:10B4E000B6218E828F83E064016008A90A12B63308
:10B4F000122FD7A90A8E828F8312B633122F65E9D5
:10B50000600312B61AAC18AD19EEFAEFFB123199BE
:10B510008A0A8B0B74FE6508700474FF650970035A
:10B5200012ACC0EA450B700302B5DF8E828F83E058
:10B53000C0E07401122CAFD0E0F07402122CAF12F4
:10B54000DA047401122A7E880C890D780C122A0202
:10B5500012B600122841EE240E12BB43F50C780CF3
:10B56000122A069005441228417407122CAFE0F904
:10B57000AC08AD091231937407122A30E9FE741039
:10B580006E705EAA0AAB0B123C018055EE241312BA
:10B59000BB43C0E07415122CAFD0E012EDBC740DAB
:10B5A000122CAF12C9BA240412B5EF12B898740F56
:10B5B000122CAF12C9BA241412BB43C0E074161285
:10B5C0002CAFD0E012E26112B5E812B04074041260
:10B5D0002A86123007E9600302B42C791180047EB8
:10B5E00010EEF9742502C109E0F98A828B832212D8
:10B5F000B5F322F8E43FF9E8FAE9FB8A828B83226B
:10B60000EE12C9862212B60922EE240FF582E43F1B
:10B61000F583E02212B60954402212B6094420F004
:10B620002212B6094440F022F58312B62E2212B03F
:10B6300048EE22A3A3A3A312D32F12983D2212B641
:10B640004222F08E828F83A322C082C08374DC12D8
:10B650002AC48A828B83A3A3A3A312B898740E1260
:10B660002CAFE8F0A3E912D0D7740C122CAF12C89B
:10B670008112B70EE0C0E0741A122CAFD0E0F012C5
:10B68000B7183B12B8967420122CAF12C881EA1278
:10B69000D30C3BF583E0C0E07408122CAFD0E0F08F
:10B6A000EA241CF582E43B12B8967412122CAF12F5
:10B6B000C881EA2411F582E43BF583E0C0E0740917
:10B6C000122CAFD0E0F0EA2412F582E43BF583E0DF
:10B6D000C0E07407122CAFD0E012A4B874FFF0746D
:10B6E00001122CAF74FFF07402122CAF74FFF090B3
:10B6F00080C412283D7404122A8E7407122A8612FE
:10B700002EB17404122A307900742402848BEA2446
:10B710000DF582E43BF58322EA12ED8E2274EE12DF
:10B72000242A74EF122AC48A0E8B0F8C088D098983
:10B730000C750A107A217B00123BFB12D137E849C5
:10B74000700302B883750B007C217D007900851899
:10B7500082851983E0FA123B477426122CAF12B887
:10B760009F900902E060046401703EAA08AB0912D0
:10B770002DB58A108B11A810A911E8496023888281
:10B780008983A3A3A3A3E06401600D88828983A3B6
:10B79000A3A3A3E064037009EE5440700474044F43
:10B7A000FFEF54046003750B0190055112D31F8500
:10B7B000188285198312B88A2409F582E43812DACE
:10B7C000117423122CAF12B898740F122CAFE8F03A
:10B7D000A3E912B8A512ED8412B8A512ADC6740281
:10B7E00012BC2212C5CDE508F0A3E50912B8A512D6
:10B7F000ED4FE50CF07425122CAFE0F508851882AA
:10B8000085198312ED94E50812B8A5241FF582E48A
:10B8100038F583E50EF0A3E50FF07406122CAF1295
:10B82000DA047408122CAFE508F07428122CAF1259
:10B83000C5CCC082C083740C122CAFAC82AD83D057
:10B8400083D082740312295EA90BAA18AB19123196
:10B8500027E964017021900902E06004640170121C
:10B86000E50BA2E0500CA908123151EA4B6003121B
:10B870003175750A00800C85188285198312D31FD3
:10B88000123C01A90A741102BE5612D0E5C822EE7C
:10B890002413F582E43FF58312D0E022A3A3A3E0B2
:10B8A000FEA3E0FF2212D146C82274EE12242AEA37
:10B8B000FEEBFF8C088D098E828F83A3740812C95A
:10B8C000ADE060088E828F83A37410F012BB4060DD
:10B8D000098E828F83A3E02408F0EE241512BB4367
:10B8E00060088E828F83A3E004F08E828F83A3A3EF
:10B8F000A3A3A3A3E060198E828F83A3A3A3A3A312
:10B90000A3A3E0C3332402F88E828F83A3E028F040
:10B91000EE241112BB436005750B0E8003750B00FE
:10B920008E828F83A3E0F8EE240D12BB4328250BF3
:10B930008C828D83F0EE241112BB43601190053C84
:10B94000E0F9122D0D850882850983E029F085082C
:10B9500082850983E0C39475400975080075090064
:10B9600002BB39E0FA7B00123BFB8A088B09EA45EF
:10B9700009700302BB398E828F83E0FA9005411271
:10B98000BB517402780C122BC6EA450CFAAB0DEED3
:10B99000241212BB435403F50C750D007406780C89
:10B9A000122BC6EA450CFCEBFDEE241512BB4360DE
:10B9B00004780180027800EE2416FAE43FFBE8F9EF
:10B9C000ED49FDEE241112BB43F50C7409780C12FD
:10B9D0002BC6ED450DFD8A828B8312BB51740B780B
:10B9E0000C122BC6ED450DFD12BE2612BB51740C78
:10B9F000780C122BC6ED450DFD8E828F83A3A3A379
:10BA0000A3A3A312BB51740A780C122BC6ECF8ED59
:10BA1000450DF9E8850882850983F0E9A3F0EE2455
:10BA20000212BB4785088285098312BB75F0EE249C
:10BA300004F8E43FF98882898312C077A312BB75AA
:10BA4000A3A3F0EE241312BB58F0EE241412BB583B
:10BA5000A3F0750A088A828B83E06015EE24181221
:10BA6000B03AE5082408FAE43509FB124525750AC1
:10BA70001012BB40601BEE241A12B03A850A0CE586
:10BA800008250CFAE43509FB1245257408250AF54A
:10BA90000A8E828F83A3A3A3A3A3A3E06058EE24FE
:10BAA00007F510E43FF511851082F583E0C0E01240
:10BAB000C85DD0E012BB65E0C0E012C85DD0E01206
:10BAC000BB6512976C1229FE851082851183E025D3
:10BAD000E0FCE433FD850A0CE508250CFAE43509A1
:10BAE000FB123B3B7403122A30851082851183E0E0
:10BAF000C333250AF50AEE241512BB436008C0E0E3
:10BB000012C85DD0E0F012C84F12976D1229FEEEF8
:10BB1000240D12BB43FC7D00850B0A8E828F83A30C
:10BB2000E0F8E50828F8E43509F9E8250AFAE439E7
:10BB3000FB123B3B7403122A30AA08AB0902BE5920
:10BB4000EE241712B60C22F8E43FF988828983E0CC
:10BB500022E0F50C750D0022F582E43FF58312BB5F
:10BB60007EA3A3A322F0050A8E828F83A3A3A3A39F
:10BB7000A3A3A3A322A3A312DF8F12BB7E2212C012
:10BB80007BA3A32274F412242A74FD122AC48A0807
:10BB90008B09ECFEEDFF7401122A7E880A890B786E
:10BBA0000A122A027402122A8EEEFAEFFB122FB347
:10BBB0007402122A30E97057851882851983E0854E
:10BBC0000882850983F07401122CAFE0F812BC18CA
:10BBD000A3A312BC26602914850882850983A312B9
:10BBE000BC2212D6F87401122CAFE028F8A3E03979
:10BBF000F9E824FEF582E934FFF58312E98C800C24
:10BC0000850882850983A3E4F0EEFAEFFB80047ACD
:10BC1000FE7BFF7403029844A3E0F985088285093E
:10BC2000832212BC2E22E8F0A3E912BC2E2212BC01
:10BC3000322212A4BCE02274EE12242A8A0A8B0B50
:10BC4000ECFEEDFF750F01E9C39408500302BDBE81
:10BC50008E828F83E912AE6F12C0A21231ABE960FF
:10BC600003750F0012C0848E828F8312C0D4EE122F
:10BC7000B7193F12C0BEC0E0EE2411F582E43FF5D3
:10BC800083D0E012C0B6C0E0EE2412F582E43FF5A6
:10BC900083D0E012B63E740812BE49A3A3A3E060AD
:10BCA00018E50A2408F8E4350BF912CA6112C881B4
:10BCB0008E828F83A3E02408F08E828F83A3A3A3B8
:10BCC000A3A3A3A3A3E0601C8E828F83A385820815
:10BCD00085830912C097EE241512E243A3E912CB23
:10BCE000722408F08E828F83A3A3A3A3A3E0600F26
:10BCF00012BE308E828F83A3A3A3A3A312BE50EEE5
:10BD0000241912C974EE241B12C974A3F0EE24186E
:10BD100012BB43700302BDAE12BE30FAEE2419F519
:10BD200082E43FF583EA12BE50F8E50A28F582E482
:10BD300012E23AF812CB76E812BE50E8C39AEE50FF
:10BD400068241912BB43F8904DEFE493C398500553
:10BD500075110C8008EE241912BB43F5118E828FE9
:10BD600083A3E0F8E50A28F50CE4350BF50D750E14
:10BD700000780C1229FEAC11EC2CFCE433FD7A9B0C
:10BD80007B12123B3B7403122A30EE241BF582E433
:10BD90003FF583749BF0A37412F0E511C333F8856B
:10BDA0000882850983E028800412C96DE4F08E8240
:10BDB0008F83A3E0F88E828F83E0C39850047900CC
:10BDC0008062A3E0FAE50A28F8E4350BF9EE241DB9
:10BDD00012E243A3E912C0CDC39AC0E012BE26D03E
:10BDE000E012C86C603CEE2417F8E43FF98808893B
:10BDF000098882F583E024F2F0EE241D12BB47246B
:10BE00000EFAA3E03400FB8882898312DA139005CE
:10BE10003CE0F9122D0DE9F8850882850983E0C31D
:10BE200098F0A90F8033EE2417F582E43FF58322C2
:10BE30008E828F83A3858208858309E0F8E50A282E
:10BE4000F582E4350BF583E02212B642A3A3A322C8
:10BE500012CB8004F022122A307F0A0226B974F431
:10BE600012242A8A088B09EA12BEE5F0EA13135459
:10BE70003F12BEDEA3A3A3F0EAC4131312BEE5A3D0
:10BE8000A3F0EB12BEF012BEF87409780A122C3A35
:10BE900012BEEE12BEF7740A780A122C3AE50A5462
:10BEA00001C0E0EC2418F582E43DF583D0E012BE39
:10BEB000FD740B780A122C3A12BEEEA312BEF77470
:10BEC0000C780A122C3A12BEEEA3A3A3A3A3A3A339
:10BED000A3F0740D7808122C3AA908029847540F61
:10BEE0008C828D832254038C828D83A3A322E50A46
:10BEF00054018C828D8322A3A3A3A3A3A3F08A0A57
:10BF00008B0B22C082C08379008A828B83A3A3A378
:10BF1000A3A3A3E090053B600EE070228A828B838E
:10BF2000A3A3E070198016E060148A828B8312D379
:10BF300016900544E06A7003A3E06B60010902C13A
:10BF40004474F012242A8A0A8B0B890C8C088D0900
:10BF50008A828B8312C0A21231AB12C08485088200
:10BF600085098312C0D4E50812B719350912C0BE7D
:10BF7000C0E0E508241112C864D0E012C0B6C0E0E9
:10BF8000E508241212C864D0E012EDE7740812C06C
:10BF9000B0E0601EE50A2408F8E4350BF9E5082452
:10BFA0001312C86412C881850882850983A3E0241E
:10BFB00008F0850882850983A3A3A3A3A3A3A3A351
:10BFC000E0601B850882850983A312C093E50824DD
:10BFD0001512C864E8F0A3E912C0CD2408F0850862
:10BFE00082850983A3A3A3A3A3E0601985088285A2
:10BFF0000983A3AE82AF8312BE3B85088285098385
:10C0000012C0C804F0AA08AB091231B1E9F50D70ED
:10C0100061850882850983A3A3A3A3A3A312C07784
:10C02000701AE0FAE50A2AF8E4350BF9E508241D50
:10C0300012C86412C881E50CC39A802A12C093E822
:10C04000240EF8500109E508241D12C86412C881A5
:10C0500090053CE0F9122D0D8E828F83E0F8E50CFF
:10C06000C39824F2C399C0E0E508241712C864D02D
:10C07000E0F0A90D02C10C12C07B22E08508828588
:10C080000983A322850A82850B83A3A312C0EAE059
:10C09000F9EA22AE82AF83E0F8E50A28F8E4350B2E
:10C0A000F922E0FAA3E0F8E4C8F9EA28E439FB222F
:10C0B00012EDCAA3A32212C0FDA3A3A3E022F5831D
:10C0C000E812C0F6A3A3E022A3A3A3A3A3F08E8249
:10C0D0008F83E022A3A3A3A3A3A3A3A3A312C0F6C9
:10C0E00012C0EAA3A3E0F9EAF822E0FA850A828501
:10C0F0000B83A3A3A322F0A3E912C0FD22F0850ABB
:10C1000082850B83A3A3A3A322122A307F080226D1
:10C11000B9C082C0837AC27B0579E21245F17AC246
:10C120007B058020C082C0839005448014C082C0FB
:10C1300083900547800BC082C083794A1245F18005
:10C140000312D31FD083D0820229E274F612242A6C
:10C150009005CAE0FE04F0EEF91231518B09EA4570
:10C160000970EDEE60EAF902C4B874EE12242AEA0E
:10C17000FEEBFF8C0E8D0F890A750B00750C0012FB
:10C18000334F8A088B097412122CAFE0F510741328
:10C19000122CAFE0F50DEA45097017E50D600302BA
:10C1A000C28EA90AAC0EAD0FEEFAEFFB123373028A
:10C1B000C39CE50D700302C254900902E060046460
:10C1C00001700E9005D712CB65600612C5CF1248DC
:10C1D00072E510700B850882850983E4F002C2893C
:10C1E000900902E060076401600302C2B190053E5D
:10C1F000E0A2E1400302C2B19005D912CB65600C08
:10C20000A910AA08AB0912C5CF1248728508828509
:10C210000983E0FA12E256500109C3EA98E499A2B0
:10C22000D265D0335009850882850983E004F08502
:10C230000882850983E0F8904DF1E4936870727587
:10C240000B01EEFAEFFB123043850882850983A3C8
:10C25000E4F0805DE5107021EA2402F582E412DE4C
:10C26000A9850A0E250EF8E4340013E813F07009CE
:10C270008A828B83A3A37401F08A828B83A3A3E0B9
:10C28000F890155FE0C3985028750C018023740165
:10C29000650D701DE5106019900902E060046401ED
:10C2A000700F90053EE0A2E15007EEFAEFFB12306E
:10C2B00043900902E06402600FE060046401702AA8
:10C2C00090053EE0A2E140227401650D701CE5106E
:10C2D0009005E96013E004F0901533E0F89005E96B
:10C2E000E0C3984005750B01E4F0E50CA2E092F084
:10C2F000E50BA2E072F0400302C39C900902E060EB
:10C30000046401704190053EE0A2E15039EEFAEF7D
:10C31000FB122DB58A088B09A808A909E8496026EF
:10C32000E50CA2E0500D88828983A3A3A3A3A3E018
:10C33000C2E0F0E50BA2E0506388828983A3A3A347
:10C34000A3A3E0D2E0F0E50BA2E05050900902E098
:10C3500060046401701D90053EE0A2E15015EEFA04
:10C36000EFFB122DA3E9600BEEFAEFFB7900122E22
:10C37000E78029900547E06E7003A3E06F701DEE23
:10C38000FAEFFB7901122EE7900902E06402700CCB
:10C390007A017B0090059EE0F9123CCD02BE5974F3
:10C3A000F412242A74016A4B700E7A017B00900506
:10C3B0009EE0F9123BA1803790152A12DA13EA4B5E
:10C3C00060218A088B09E4F50AF50B78081229FA2E
:10C3D0007A017B0090059EE0F9123CC17404122A98
:10C3E00030800C7A017B0090059EE0F9123CCD0272
:10C3F0009847C082C08390152C02AA51C082C08386
:10C4000090152E02AA5174F612242A750830750967
:10C41000057808122A027C6E7D007A217B00123C8E
:10C42000737402122A30E9F508122D31E94208909E
:10C430000902E0600464017006122DDFE9420890F1
:10C44000070B12CB65600912C5CF124872E942088A
:10C45000122CCBE9FE1240E1E9F8E5084E48F980DC
:10C460005774F612242A12450175083075090578AB
:10C4700008122A0275086E7509007808122A027CD3
:10C48000007D007A217B00123C7F7404122A301256
:10C490002D37900902E0600464017003122DE590CD
:10C4A000070D12CB65600612C5CF124872122CD14F
:10C4B0001240ED8003122A307F020226B974F61270
:10C4C000242A74FF122AC47E007508307509057885
:10C4D00008122A027C6E7D007A217B00123C737464
:10C4E00002122A30E9600302C5A07808122A0275F8
:10C4F000086E8E097808122A027C007D007A217B62
:10C5000000123C857404122A30E9600302C5A09031
:10C510000544E064FE7003A3E0F4700302C5A00EBE
:10C52000900553E064086005E06404706F8518822C
:10C53000851983EE12C9CB79421245F77A5B7B05E8
:10C5400079431245F77A587B0579471245F77A49BE
:10C550007B05794A1245F77A477B05794B1245F7F7
:10C560007A517B0579501245F77A447B057953124D
:10C5700045F77A597B0579541245F77A467B057958
:10C58000E11245F790053EE0A2E35004D2F08002AC
:10C59000C2F012C9C179521245F780041245011E3A
:10C5A000122D3D900902E0600464017003122DF722
:10C5B00090070F12CB65600612C5CF124872122C7D
:10C5C000DDEEF9740102C4B58E828F83E0F8A3E03A
:10C5D000F58388822274F612242AE9FEA2E050260E
:10C5E0007508307509057808122A0275086E7509F4
:10C5F000007808122A027C007D007A217B00123C20
:10C600007F7404122A30EEA2E35003122D439009E6
:10C6100002E0600464017008EEA2E15003122DFDF7
:10C62000EEA2E2500E90071112CB65600612C5CF44
:10C6300012487202C4B874F612242A74EC122AC486
:10C640007401122A8E9014DAE0F97AA17B05123176
:10C6500003900590E06402707C7405122CAFE4F046
:10C660007407122CAFE4F07A04F9122D918A089025
:10C670004E02E493FAC3E5089AEB9400400302C724
:10C680000B122D85E9600302C70B904DE712C767B7
:10C6900060157A047903122D91904E02E493FC9078
:10C6A0004DE712C77150087405122CAF7401F09059
:10C6B0004DE512C76760157A027901122D91904EEF
:10C6C00002E493FC904DE512C771503F7407122CA1
:10C6D000AF7401803590055C122C8CE8494A4B60A0
:10C6E0000474018001E4C0E07405122CAFD0E0F0C6
:10C6F000900560122C8CE8494A4B6004740180015B
:10C70000E4C0E07407122CAFD0E0F09014DAE0F946
:10C710007CA17D057401122A861230FD7AA17B0569
:10C7200079451245F77407122CAFE07011740512A9
:10C730002CAFE07009851882851983E4800885187C
:10C74000828519837401F09014D6E0F89014D5E036
:10C7500058F8851882851983E05812C9CB7941129F
:10C7600045F7741402C4B5E493F8740193F9E849E9
:10C7700022E493F8740193F9ECC398F8E499F9C3AF
:10C78000EA98EB992274F712242A74ED122AC4E96C
:10C79000FE90059DF0AC18AD199014DAE0F97AA17D
:10C7A0007B051231037412122CAFEE12C7C3AA1804
:10C7B000AB191230FD7AA17B0579451245F7741348
:10C7C00002B138F09014DAE0F97CA17D052274F40E
:10C7D00012242AEAFEEBFF9014DCE064FE7003A34F
:10C7E000E0F470687A167B00123B5F8A088B09EAD6
:10C7F000450960588A828B83740112C86C8A828BC7
:10C8000083A3600474028002740112C887A3E08AC3
:10C81000828B83A3A3A3A3A3A3A3A3A312C89DFC5A
:10C82000A3E0FDEA2402FAE43509FB124525E508F8
:10C83000241312C864E4F0AA08AB0990059EE0F93D
:10C84000123B6B12C84F12D0D012C8810298471207
:10C85000C85322EE240BF582E43FF58322850A0CAF
:10C86000E508250CF582E43509F5832212C871E04C
:10C8700022F08E828F83A3A3A3A3A3A322E0129707
:10C8800061E8F0A3E9F022F0EE241DF582E43FF523
:10C890008312C8952212D0E5F583888222A3F0EE98
:10C8A000241512B60C2274F212242A74FD122AC422
:10C8B0008A088B09890A8C0B7401122CAF7404123C
:10C8C000C9CB1232418A0C8B0DAE0CAF0DEE4F70FE
:10C8D0000302C962EE12B7193F12C9917407F0A39F
:10C8E000A882A983E5082413FAE43509FB8A828B20
:10C8F0008312C9A28A828B8312C9A1E50812D30CC4
:10C9000012DEA98882898312C9AD7401F0E508247A
:10C910000BF8E43509F9EE12C96D12C9BA12ED67C8
:10C920001231BD12DA0AEE241312ED697403650A9E
:10C9300060067401650A700712C97D7404800412D0
:10C94000C97DE4F09014DC12ACE312C88174016577
:10C950000B7006EE241112C974EEFAEFFB122E2DA5
:10C96000800279109014DC129B3802D0EC12EDB3E7
:10C9700022EE2412F582E43FF583E4F02212C98509
:10C980007440F0A322EE12DE9B3FF5832212ED8D60
:10C990003BF58312C99722E0F8A3E0F988828983E6
:10C9A00022A3E088828983F0A308A98322F0EE24E1
:10C9B00016F582E43FF58322A3A3E8F0A3E9F0EEA5
:10C9C00022A2F0E433851882851983F0AA18AB19E6
:10C9D0002274F412242AEAFEEBFF7A007B0490050D
:10C9E0009EE0F9123CCD12CA6F12C88190055374B3
:10C9F00009F01231BD8A088B09AC08AD0912CA6171
:10CA000012D31F12451FE9640170537A0F7B001285
:10CA10003B5F8A088B09EA450960438A828B8374ED
:10CA200002F012CA79FC88828983A3A3E0FBEC8A16
:10CA300082850983A3A312DA1488828983A3A3A31E
:10CA4000E08A8285098312C89DFAA3E0FB794A1225
:10CA500045F7AA08AB0990059EE0F9123B6B0298D6
:10CA60004712CA6522EE2413F582E43FF583229033
:10CA7000051612D0E090152E22EE241DF582E43F1B
:10CA8000F58312CD4AE02274F412242A74FD122A8E
:10CA9000C48A088B097401122CAF740212C9CB121C
:10CAA00032418A0A8B0BAE0AAF0BEE4F700302CBFA
:10CAB0005112EDD2700888828983A37420F0850812
:10CAC00082850983A3A3A3A3A3E0640170098882DC
:10CAD0008983A3E0D2E6F0850882850983A3A3A316
:10CAE000A3A3A3E06401700A88828983A3E0D2E74C
:10CAF000800312ED4912EDC3701985088285098300
:10CB0000A3A312CB656006EE241612ED6912EDA503
:10CB100012C881850882850983A3A3A3A3A3A3A325
:10CB2000E06401700312ED7A85088285098312D3CF
:10CB30001F12325FE9600312ED7312ED661231BD10
:10CB400012CB6B12CB5712C9B8FAEFFB122E2D8005
:10CB500002791002BC13E0F8A3E0F98E828F8322E1
:10CB600012B22CF58312D0E0E8492212CB76EAF01B
:10CB7000A3EB12CB8022EE241AF582E43FF5832248
:10CB8000F0850882850983E02274F512242A74F363
:10CB9000122AC4890AEAFEEBFF7508007509007CB9
:10CBA0000D7D007900AA18AB19123B47EE12D70091
:10CBB0003FF58312CD36741F58600C7AD37B001278
:10CBC0004105790002CC88E8A2E55008740C122CCB
:10CBD000AF7401F0E8A2E75008740B122CAF740197
:10CBE000F0E8A2E6740A5008122CAF7401F0800835
:10CBF000122CAFE0640170138E828F83A3A3A3A3D2
:10CC0000A3A3A3E06032EE241380128E828F83A34D
:10CC1000A3A3A3A3A3A3A3E0601EEE2415F582E4BF
:10CC20003FF58312A6AD6010AC08AD097402122C5A
:10CC3000AFAA82AB8312452512C84F12C87D740A71
:10CC4000122CAFE06401703712D31212325FE97018
:10CC500035EE240B12B892900547E0687003A3E00C
:10CC6000697023E508450960161231BDEAFCEBFD49
:10CC70007402122CAFAA82AB8312451FE96007AA87
:10CC800018AB19122EE1A90A02EEDA74F712242A5F
:10CC900074D2122AC4EAFEEBFF8E828F83129CD9D3
:10CCA000A2E0400302CD3112CD3DE054FE12E66415
:10CCB000740D122A8E12CD5A1231B7E97073742A8C
:10CCC000122CAF12CD5470697C0D7D007900AA182A
:10CCD000AB19123B477416122CAF12C87D742A127E
:10CCE0002CAF12CD36A2E55008740B122CAF740194
:10CCF000F0E8A2E75008740A122CAF7401F0E8A221
:10CD0000E65004742080027422122CAF12B04074DA
:10CD100002122CAFAA82AB831245258E828F83A389
:10CD2000A3E0C0E0740C122CAFD0E012C9CB122EDD
:10CD3000DB742E02B13812C895A3E0F8228E828FE0
:10CD40008312CD4AA3A3A3A3A32212D0E5F988821C
:10CD50008983A32212B20B640422EA241EF582E422
:10CD60003BF583E0F9EA241FF582E43B12983B226D
:10CD7000E9F87900740468600A740A68600574034D
:10CD8000687001090229E274F612242A8A828B83D0
:10CD90007420F0A3A37401F0122E338A088B09AE1D
:10CDA00008AF09EE4F60168E828F837401F09005F4
:10CDB00091E0700912ED661231BD12DA0AEEFAEF57
:10CDC000FB02C4B8C082C08390054102A9F0C082B2
:10CDD000C0839014DB02A9F0C082C083E99014DB09
:10CDE00002AA55C082C0839005B67401F0E9A2E39F
:10CDF00050037403F0E9A2E15004E0D2E2F002C172
:10CE00004474F612242A79007C008A088B09780879
:10CE10001226FFF8FF0732CE30CE30CE30CE30CEE5
:10CE200028CE2CCE32CE2DCE7C0480060C0C800277
:10CE30007C089005B6E05C6003098003EC600109A2
:10CE400002C4B874F412242AEAFEEBFF8908122DFA
:10CE5000BB8A0A8B0BA80AA90BE849604188828922
:10CE600083A3A3A3A3E06036C39405503174016586
:10CE700008601A88828983A3A3A3A3E06401600DDC
:10CE800088828983A3A3A3A3E06402700A888289AD
:10CE90008312A78A124872EEFAEFFB122DC702988E
:10CEA0004774F612242A8A828B83E07012A312CB75
:10CEB00065600C8A828B8312D31E1247D180047A5C
:10CEC000007B0002C4B8C082C083900590E0640279
:10CED000700B900553E06408700312328302C14462
:10CEE000C082C0837C00EC12CF937003A3E06B7010
:10CEF00011904DF6E493C0E012CF62D0E0F079C516
:10CF000080510CECC3940340DD7C00EC75F003A46D
:10CF1000F8A9F074BA28F582740512972464FE709B
:10CF200003A3E0F4600F0CECC3940340DE7C00EC40
:10CF300012CF567015EC12E2FD12DA13904DF6E4A2
:10CF40009388828983F0790080090CECC3940340B4
:10CF5000DE79C702C14475F003A4F8A9F012CF62CC
:10CF6000E02274B928F582740539F58322C082C0A5
:10CF7000837D00ED12CF937003A3E06B700912CF95
:10CF80005D6004790180090DEDC3940340E57900EB
:10CF900002C14475F003A4F8A9F074BA28F58274AC
:10CFA0000512E7B66A2274F212242A74DD122AC42A
:10CFB000EAFEEBFF750A00900902E0600764016079
:10CFC0000302D0CA900544E06E7003A3E06F701EA8
:10CFD000EE4F700302D0BE9005CB12CB65700302FA
:10CFE000D0BE750A0112C5CF12487202D0CA122DE6
:10CFF000B58A088B09EA4509700302D0BE8A828B84
:10D0000083A3A3A3A3E0640160108A828B83A3A3FC
:10D01000A3A3E06402600302D0BE85188285198351
:10D02000E412D0D7740B122CAFE8F0A3E912C9CBED
:10D03000122D79E9700302D0BE850882850983121A
:10D04000D0D012C8817900122F8F8508828509837C
:10D0500012DA137403122CAFAC82AD837418122C45
:10D06000AFAA82AB8312452585088285098312B851
:10D07000987420122CAF12C8817422122CAFE4F0E5
:10D080007C02850882850983A3A3A3A3E0F9740D1C
:10D09000122A8612321D85088285098312B8987477
:10D0A00001122CAFE8F0A3E912C9CB122D7F750A4B
:10D0B00001E508240C12C864129785F0800C9005D5
:10D0C0005112B62AFAEFFB123337A90A7423801ED5
:10D0D00012D0E09014DC2212AE7312D0DE22A3A391
:10D0E00012D0E5F922E0F8A3E022A90A7403122A7B
:10D0F000307F060226B9C082C08374FE122AC49013
:10D100000902E0600464017029790190052912C5C3
:10D11000CC12487212D137900544E8F0A3E912C945
:10D12000CB79531245F785188285198312D31F12C4
:10D130003DCF740202848B851882851983EAF0A39F
:10D14000EB12D146F92212BC32F8A3E02274F51298
:10D15000242A74F3122AC48A088B09ECFEEDFF75A9
:10D160000A12EA45097005790002D25A900544E096
:10D1700065087004A3E0650970191231BDEAFCEB83
:10D18000FDEEFAEFFB12451FE97005750A018003F9
:10D19000750A00851882851983E4F004122CAFE526
:10D1A00008F0A3E50912C9CB122D6DE960297403BB
:10D1B000122CAFAA82AB83122D4FE964017018754F
:10D1C0000A017403122CAFAC82AD83EEFAEFFB12AE
:10D1D000451FE9701E801F7412650A701990059032
:10D1E000E064027011EEFCEFFDAA08AB09122D9D60
:10D1F000E96003750A00EEFCEFFDAA08AB091233E3
:10D2000055E9F8740A687005750A01804274A068CF
:10D210007037EEFCEFFDAA08AB091233677E008081
:10D2200023EE75F017A4F8A9F012E7CC7004A3E080
:10D230006509700F12E908122D4FE9700612E4A774
:10D240001233430E12D25D40D87401650A70097919
:10D2500000AA08AB09123295A90A02EEDA904DEE47
:10D26000E493F8EEC3982274F612242AEAFEEBFF48
:10D270008908900902E060046401701E123283E59F
:10D2800008F5097809122A06790DEEFCEFFD7AFC03
:10D290007BFF1232A17401122A3002C4B874F71253
:10D2A000242AEAFEEBFF8E828F83A3A3A3A3A3A36A
:10D2B000A3A3E0601312D30412982E12328FE964F4
:10D2C00001700512C84F802D8E828F83A3A3A3A364
:10D2D000A3A3A3E0602912CA6112D323FAA3E0FB3F
:10D2E00012328FE9640170178E828F83A3A3A3A3E8
:10D2F000A3A3A3A3A312D31F1232777901800279CB
:10D300000002B13BEE12D30C3FF583222415F582C7
:10D31000E4228E828F83A3A3A3A3A3A3A3A3A31218
:10D32000983D2212D32FA3A3A3A3A3A3A3E0221269
:10D33000B0488E828F83A3A32274F212242A74FD34
:10D34000122AC48A088B09ECFEEDFF890B750A01CD
:10D350007401122CAF740412C9CB123241EA4B6033
:10D36000477411122CAFE0601AEA2417F582E43BEF
:10D37000F583E412DBBF8A828B83E0D2E7F012D31D
:10D38000ABE4F012C98D740312D619EE888289833A
:10D39000A3A3F0EF88828983A3A312AE6EA3A31286
:10D3A000EFB7122E2DE9F50A02D0EAEA2414F5822D
:10D3B000E43BF5832274F012242AEAFEEBFF890A8B
:10D3C000750B0112CA79F50C88828983A3A3E0FA50
:10D3D0008882898312D4F212BB406404600A7AD333
:10D3E0007B0012410502D4EDE50C1228C6020002B2
:10D3F00002D4030BA2D4030C89D40D61D40EA2D4A1
:10D40000A0D4900902E060076401600302D4A290F6
:10D41000053EE0A2E1400302D4A27900AB0912303C
:10D4200025EA4B60318A828B83A3A3A3A3A3A3E045
:10D430005418602212C84F1228418A828B83A3A3FA
:10D4400012284179008E828F8312D51112303D74DB
:10D4500004122A30802E7901AA08AB09122EF3801B
:10D4600041900902E060046401703790053EE0A23B
:10D47000E1502FAB09123271AA08AB09123277E9D9
:10D4800064C5701E750B008019900902E060046489
:10D4900001700F90053EE0A2E15007123DF38002BB
:10D4A000880AEE2409F50EE43FF50FAC08AD09A992
:10D4B0000C850E82F58312D31F122F0B850E8285E9
:10D4C0000F8312D31F12325FE96022EE241112BBC8
:10D4D00043C39402401712C84F12DAD97003A3E075
:10D4E00069600AE50BA2E05004A90A8002790002F3
:10D4F000C10CA3A3A3E0F8E4C8F9EA28F508E439CD
:10D50000F50922E508240CF582E43509F58312B506
:10D51000E8A3A3A3A3A3A3A3A3A312B0448A828BCB
:10D520008312983D2274EE12242A74F5122AC48ABA
:10D530000A8B0B890C8C0E8D0F7E01EE122CAF74B2
:10D540000AF0741D122CAFE0F50DE9700FE50DC364
:10D5500033240AC0E0EE122CAFD0E0F0AA18AB19C9
:10D560001232418A088B09EA4509700302D60E126D
:10D57000B718350912D79B740912D7A7450D12D6D3
:10D5800039AC0EAD0FEEFAEFFB124525EE2408FE86
:10D5900050010FE50C70247C00741E122CAF12B8E1
:10D5A000988012EC12DAC5E82AFAE93BFB12D61F82
:10D5B000A30EAF830CECC3950D40E8E508241712C9
:10D5C000C8647401F01231BDE508241AF582E4350F
:10D5D0000912DA117403122A8EAA0AAB0B122D5506
:10D5E000E96019E508241612C8647401F074031286
:10D5F0002A7EE508241812C86412C881850882852D
:10D60000098312D615AA08AB09122E2DE9FEEEF9F0
:10D61000740B02BE56A3A3E50AF0A3E50BF0228A21
:10D62000828B8312D63312D6398A828B8312D632FA
:10D63000F022A3E08E828F8322F0A3AE82AF8322FA
:10D6400074F012242A74F8122AC48A088B0912D69C
:10D65000FF350912D820F50B880AA3AE82AF83EEFE
:10D66000FCEFFDAA18AB19124525EE2408FE500167
:10D670000FAC18AD197A657B0512451FE96074740B
:10D68000E0550A7067AA0BEA2AFA7B00123BFB8A74
:10D690000C8B0DEA450D605B7C00801E8E828F83B3
:10D6A00012C0A2EC12D6F8E50C28F582E50D39126D
:10D6B000DA11EE2402FE50010F0CECC3950B40DC96
:10D6C000780C122A02780B122A067403122A8E7919
:10D6D00000E508240B12C86412D31F1232B9740378
:10D6E000122A30AA0CAB0D123C0180077AD37B00C2
:10D6F000124105740802C10925E0F8E433F922EA71
:10D70000241DF582E42274F012242A8A0A8B0B89E4
:10D710000C8C088D099007DE12CB65607B741012AB
:10D720002CAFE0F50D12D6F8E8240EFAE439FB121E
:10D730003B5F8A0E8B0FAE0EAF0FEE4F605A8E829C
:10D740008F8374D4F0A3A3E50AF0A3E50B12BE49BE
:10D75000E50CF0AC08AD09EE2405FAE43FFB1245F8
:10D760002512B21FE50DF07411122CAF12DBA9784F
:10D77000081229FEAC0DEC2CFCE433FDEE240EFA6D
:10D78000E43FFB123B3B7403122A30EEFAEFFB90AE
:10D7900007DE12C5CC12487202C10CF583E0FEA36D
:10D7A000E0FF8E828F8322F0A3E50CC43354E02285
:10D7B00074F612242A74F8122AC4890812D6FF3B80
:10D7C00012D820F98809A3AE82AF83740169704230
:10D7D000EEFCEFFDAA18AB19124525EE2408FE5009
:10D7E000010FAC18AD197A657B0512451FE9602958
:10D7F00074E05509701C8E828F83A3E0FA8E828FAD
:10D8000083A312C0A48E828F83E0F91232D1A908BB
:10D8100080097AD37B001241057900740802C4B5EF
:10D82000F583E02401FEA3E03400FF8E828F83E0C5
:10D83000F8741F582274F612242A74DF122AC4EADC
:10D84000FEEBFF12CB6060508E828F8312D31FAC31
:10D8500018AD1912CD5A1231A57409122CAF12DA73
:10D86000D97003A3E069603012C5C8122841750859
:10D87000FE7509FF7808122A02741C122CAFE0F919
:10D88000740D122CAF12B040740F122CAF12D31FB4
:10D8900012303D7404122A30742102C4B574F71298
:10D8A000242AE9FC7A007B007E00800B12D93FE03D
:10D8B0002AFAA3E03BFB0E904E0212D2605029EEF2
:10D8C00075F016A4F8ADF0EDF912E7BBF460E7745B
:10D8D0000D28F582740E3912CB6360DAEC60CD123C
:10D8E000D93FE4F0A3F080CE7E00800B12D92CE06B
:10D8F0002AFAA3E03BFB0E12D25D502DEE75F01715
:10D90000A4F8ADF0EDF912E9197003A3E0F460E6B4
:10D9100074E028F582740F3912CB6360D9EC60CCC7
:10D9200012D92CE4F0A3F080CD02B13BEE75F017D4
:10D93000A4F8EDF974E028F582740F39F58322EE2E
:10D9400075F016A4F8EDF9740D28F582740E39F50A
:10D95000832274EC12242A890CEAFEEBFF90059DC9
:10D96000E0C3950C503B1232119005CD12DA0490B1
:10D970000537E0F508E4F509F50AF50B9080B07875
:10D9800010122C587808791012233B78081229FAC3
:10D990007A007B0290059EE0F9123CC17404122AC1
:10D9A0003002971C74F612242AEAFEEBFF9005B7AA
:10D9B000801388828983E06E7003A3E06F603688ED
:10D9C000828983A3A312CB6570E87A047B00123BA3
:10D9D000FB8A088B09A808A909E849601888828988
:10D9E0008312DA049005B712D9F8A3A312DA1390C0
:10D9F00005B712C88102C4B812983D888289832273
:10DA00008A828B83EEF0A3EFF022EE241AF582E4F3
:10DA10003FF583EAF0A3EBF02274F412242A7E008F
:10DA20009005B780070E88828983A3A312CB657007
:10DA3000F4EE12DAC5123BFB8A088B09EA4509604D
:10DA40007E7F009005B780218882898312B040EFE5
:10DA500012DAC5E5082AF582E5093BF583ECF0A367
:10DA6000EDF00F88828983A3A312CB6570DA90054D
:10DA70009912DAD97003A3E0697808701C122A029F
:10DA8000EEF50A780A122A067C657D057900900574
:10DA90009912D31F1232B9801A122A02EEF50A78AF
:10DAA0000A122A067C657D05790090059912D31F1C
:10DAB0001232AD7403122A30AA08AB09123C0112CB
:10DAC0002E4502984725E0FAE433FB228E828F83AD
:10DAD000A3A3A3A3A3A3A3A3A312D0E0900544E010
:10DAE0006822C082C08380128A828B83A3A312B86B
:10DAF000989005B712C881123C019005B712AFE3A8
:10DB000070E602C14474F512242A90055112B89FA0
:10DB10009005CD12DB9D12C8817ACD7B057950121C
:10DB200045F79005CD12DBA9801512E35B650870FF
:10DB300004A3E06509600612E4AF123343050A123C
:10DB4000DB925018E50A12E49B7003A3E06F70DAD1
:10DB500074D528F582740F12EFB480E19005CD12D0
:10DB6000B89F9007E012CB6560257A067B00123BD8
:10DB70005FEA4B601A8A828B8374D5F0A3A3E41208
:10DB8000DBB00412DBBF9007E012C5CC1248720272
:10DB9000EEDF904DEEE493F8E50AC3982212DBA184
:10DBA0002212D0E5F99005512212ACCA750A002262
:10DBB00012DBB42212DBB82212AE73A3A3A322128B
:10DBC000DBB4A3EEF0A3EFF022C082C0839005CFB8
:10DBD00074FBF0A37432F09005D174F5F0A37432A5
:10DBE000F09005D37413F0A3743302AA55C082C019
:10DBF00083900544E064FE7003A3E0F4600E90059A
:10DC00003EE0A2E1500612335B12330102C14474BC
:10DC1000F012242A900592E06053F50CE4F50DF51E
:10DC20000EF50F9080A07808122C58780C79081205
:10DC3000233B123B598A088B09A808A909904DE19A
:10DC4000E49358F508A3E49359F509E4F50AF50BB4
:10DC5000780C7908122B8D780C1229FA7A007B0146
:10DC600090059EE0F9123CC77404122A3002C10CE0
:10DC700074EE12242A7E007F008E0A8E0B122E096B
:10DC80008E0D803E850D08AA087B00122E038A089F
:10DC90008B09A808A909E849602688828983A3A37B
:10DCA000A3A3E060046404701788828983A3A3A3FC
:10DCB000A3A3A3A3A3A3A3E0F912336DE960010F0B
:10DCC000050D904E02E493F8E50DC39840B612336B
:10DCD000318A0E8B0F8E0C8023AA087B0012333DF5
:10DCE0008A088B09A808A909E849600EE8240F12E0
:10DCF0009721F912336DE960010E050C850C08C3FC
:10DD0000E508950EE4950F40D0EF2EFE700302DE7D
:10DD1000098E0875090074027808122BC6AA08AB90
:10DD200009123BFB8A0A8B0BEA450B700302DE07E4
:10DD3000750C008E0875090074027808122BC6ACA9
:10DD400008AD0979FF123B47750D00805D850D0810
:10DD5000AA087B00122E038A088B09EA450960484D
:10DD60008A828B83A3A3A3A3E06004640470398A2E
:10DD7000828B83A3A3A3A3A3A3A3A3A3A3E0F912CA
:10DD8000336DE96023050C780A122A02EEFD85083E
:10DD900082850983A3A3A3A3A3A3A3A3A312DEAF96
:10DDA0001233077402122A30050D904E02E493F8E4
:10DDB000E50DC3985006E50CC39F4091750C008596
:10DDC0000C08C3E508950EE4950F503DAA087B00AA
:10DDD00012333D8A088B09EA45096027EA12DE9B67
:10DDE00012DEA9F912336DE96019780A122A02EEDF
:10DDF000FDE508240E12C86412DEAF123307740268
:10DE0000122A30050C80B87E00750E6290053CE049
:10DE1000600CF9122D0DE9F87454C398F50E75F0E5
:10DE200003E50E84F50D94204003750D1F850A0847
:10DE3000850B09750C00E50E6006750C20750E004B
:10DE4000E50DC39E5004AF0D8008EEFFE50CD2E651
:10DE5000F50CAC08AD09AA0CEFF912330DE9F50F7A
:10DE6000E50CA2E6401A1F7800800BE5082404F5B3
:10DE7000085002050908E8C39F40F0EFCEC39EFE9C
:10DE8000E97006E50CA2E650AAE50A450B6007AA70
:10DE90000AAB0B123C01A90F02BE59240FF582E414
:10DEA0002274682508F58274133509F583E022E0B1
:10DEB000FC85088285098312983D2274F212242A77
:10DEC000EAFEEBFF89088C098D0A7C007D00740E48
:10DED000122CAF12D31F8C0B800DEAFCEBFDEA2451
:10DEE00004FA50010B050BE50BC3950A400302DF52
:10DEF000868A828B83E0F47003A3E0F46077EC4DB4
:10DF0000600C8C828D83C3E09EA3E09F50CC8A82FC
:10DF10008B8312E2CAEE98EF9950BFEAF8EBF988CA
:10DF2000828983E0F47003A3E0F46010E82404F82D
:10DF3000500109050BE50BC3950A40E3E8FCE9FD38
:10DF4000E824FCF8E934FFF9888289831297768CFB
:10DF5000828D83E50CF0A3E50D12DF898C828D8321
:10DF6000A3A312E65EE08C828D83A3A3A3F0C3EA91
:10DF700098EB9940C712DA008A828B83A3A3E50944
:10DF800012DBB0E508F002D0F112DF8FA3E022F03F
:10DF900088828983A32274F212242A74FD122AC46F
:10DFA00089088A09ECFEEDFF750A0175F003E9A402
:10DFB0002402C0E07401122CAFD0E012C9CB12329F
:10DFC00041EA4B607812C98D7408F0741F550845FA
:10DFD00009A3F0E82402F8500109750A0080388E80
:10DFE000828F83E088828983F0A3A882A9838E82AE
:10DFF0008F8312C9A18E828F83A3A3E05407C4FC30
:10E000008E828F83A3A3A3E054074C12C9A3EE24EE
:10E0100004FE50010F050AE50AC3950840C18A8233
:10E020008B83A3A374FCF0A374FFF0EA2413F5829E
:10E03000E43BF5837401F0122E2DE9F50A02D0EAD3
:10E0400074F112242A8A0A8B0B7508007AFE7BFF72
:10E050007CFE7DFFE50A12D700350B12CA80F50958
:10E06000741F5509F50CE82402F8500109E509A2CE
:10E07000E7406FE50A2417F582E412E23AFE75F0F4
:10E0800003E50CA424026E7059E50C600B888289AC
:10E0900083E0FEA3E0FBEEFA750D00801DE054075F
:10E0A000F50EA3A882A983EEFC900544E06E7003F0
:10E0B000A3E06F7003850E08050DE50DC3950C50A8
:10E0C0002B88828983E0FEA3E0FCE4CCFDEE2CE407
:10E0D0003DFFE82402F850010988828983E05488D2
:10E0E00060BB7AD37B0012410502E22FE508700B7A
:10E0F000A909123319E9700302E22F12E24C12D37C
:10E100001F122DB58A0C8B0DAE0CAF0DEE4F605A61
:10E110008E828F83A3A3A3A3A3A3A3E4F0904DF1C6
:10E1200093F88E828F83A3A3A3A3A3A3A3A3E0C387
:10E1300098402412E2565001097A027B00122243D1
:10E14000E88E828F83A3A3A3A3A3A3A3A3F0E508D0
:10E15000C39407500205088E828F83A3A3A3A3A3B1
:10E16000A3A3A3A3E508F002E22F7CFF7DFF12E248
:10E170004C12D31F1233258A0C8B0DAE0CAF0DEE53
:10E180004F704F12332B8A0C8B0DAE0CAF0DEE4F30
:10E19000700302E22F7C177D007900123B4712E2E8
:10E1A0004C12CB5612847D8E828F83A3A3A3A3A38C
:10E1B000A3A3A312C9B812B60174AA12E275500142
:10E1C000097A027B0012224312B21FE812E2617444
:10E1D00001F0904DF1E493F8EE240D12BB43C39887
:10E1E000401912E2565001097A027B0012224312B2
:10E1F000E240E508C394075002050812E8C7E508A5
:10E2000012E266E4F0129C6E122D4FE97021850A2D
:10E2100082850B83A3A3A3A3A3A3A3A3E06010E51C
:10E220000A12D30C350B12B628129C6F1245250228
:10E23000A86B7468250AF5827413350BF583E02208
:10E24000EE240DF582E43FF583E8F022E50A12EDB5
:10E250008E350BF58322904DF1E49379002401F87B
:10E2600022F012E8CB22F012E26B22EE240CF582AF
:10E27000E43FF58322F0904DF1E49379002401F816
:10E280002274F712242AE9FE74FE6A700374FF6B8D
:10E29000603474605E6460602DEEA2E5401CA2E60E
:10E2A000900544500DC3E09AA3E09B5019790002F9
:10E2B000B13BC3E09AA3E09B40F390054412E2CA4D
:10E2C000EC98ED9940E7790180E512D0E0C3227423
:10E2D000F712242A7E00800712E4A71233430E129D
:10E2E000D25D40F47E00EE12E2FD129B38888289F6
:10E2F00083E4F00EEEC3940340EC02B13B75F003EF
:10E30000A4F8A9F074B928F8740539F988828983CA
:10E31000A32274F712242A7F0080010F904DEEE4AF
:10E3200093F8EFC398502DEF75F017A4F8A9F012E9
:10E33000E7A76A7003A3E06B70E112E35B6C700304
:10E34000A3E06D600A74FF6C700374FF6D70CC12F3
:10E35000E4AF80047A007B0002B13B12E35F2274D9
:10E36000D528F582740F12E7B62274F612242A7C9F
:10E37000FF7DFF7AFE7BFF123325EA4B703C750868
:10E38000008032E50875F017A4F8A9F074DA28F5D2
:10E3900082740F129724600512E79C701674CB28C4
:10E3A000FE740F39FF8E828F8312D31F123043EE1B
:10E3B000FAEFFB050812E3BD40C902C4B8904DEE68
:10E3C000E493F8E508C39822C082C0837A007B00FA
:10E3D0007D00801012E9117003A3E0F460050AEAE1
:10E3E00070010B0D904DEEE493F8EDC39840E502FB
:10E3F000C14474F412242A8A088B09ECFEEDFF80D4
:10E400000B123343EEFCEFFDAA08AB09123325EAE9
:10E410004B70EE02984774F612242A7D007E00802D
:10E42000020D0E12D25D5018EE12E9127003A3E035
:10E43000F460EF8D08EA65084B70E612E4AF8004E3
:10E440007A007B0002C4B874F712242AEAFEEBFFBC
:10E45000EE4F601A7C177D007900123B478E828F49
:10E460008374FEF0A30412ACEDA314129B3A02B124
:10E470003B74F712242AEAFEEBFF7508008014E5CE
:10E480000812E49B7003A3E06F600612E4AF12333E
:10E4900043050812E3BD40E702B13B75F017A4F84D
:10E4A000A9F012E35F6E22EE75F017A4F8A9F074DC
:10E4B000CB28FA740F39FB2274F412242A8A088BB1
:10E4C00009ECFEEDFF900902E06004640170209009
:10E4D0000551E06E7003A3E06F7014122DB58A0A27
:10E4E0008B0BA80AA90BE8496005E82408801AEEFE
:10E4F000FCEFFDAA08AB091233258A088B09A8088E
:10E50000A909E8496009E8240DFAE439FB80047A96
:10E51000007B0002984774F412242A8A0A8B0BECC1
:10E52000FEEDFF7508007509008034E50912E90168
:10E53000122D4FE96027E50975F017A4F8A9F0122C
:10E54000E7C67004A3E0650B700375080AEEFCEFE4
:10E55000FD12E90812451FE960034308A005099070
:10E560004DEEE493F8E509C3985004E50860BC0259
:10E57000BED974F612242A7E00805C8E08AA087B1D
:10E5800000122E038A088B09A808A909E8496046E9
:10E5900088828983A3A3A3A3E06401603988828968
:10E5A00083A3A3A3A3E06402602CE82407129721AD
:10E5B000FA74012AF0900593E0C39A501988828971
:10E5C00083A3A3A3A3A3A3A3A3A3A3E412E655A396
:10E5D00012E6641230430E904E0212D260409C7ECE
:10E5E000008059EE75F017A4F8AAF0EAF912E919BB
:10E5F0007003A3E0F4604474CB28F8740F39F9E891
:10E60000240C129721F8740128F0900593E0C39828
:10E610005029EE75F017A4F8EAF974CB28F8740FB6
:10E6200039F9E812DE9B39F583E4F0E8240EF5822F
:10E63000E439F583E412E6641230430E12D25D40F1
:10E64000A27B00EB12CF56600214F00BEBC39403D5
:10E6500040F102C4B812E65EA3A3A3A3A32212DF73
:10E660008FA3A32212E66CFAA3E0FB22F088828932
:10E6700083E02274F312242A8A088B09ECFEEDFF52
:10E68000750C007B007C01740D122CAFE0F50AA321
:10E69000E0F50B8010123B59E50CF5F0EA84ABF085
:10E6A000750C007C007D0080010D904DEEE493F828
:10E6B000EDC398504912E9117003A3E0F460EA1227
:10E6C000E7CC7004A3E0650960DF12E7A76E700372
:10E6D000A3E06F60D412E7C67004A3E0650B60C9C5
:10E6E00012E79C60C4C3940750BFEC050C70BAE5F8
:10E6F0000CC39B40B474CB28F582740F80787A00E9
:10E7000080010A904E02E493F8EAC3985070EA75CB
:10E71000F016A4F8A9F012E7D264FE7003A3E0F4A7
:10E7200060E012E7D265087004A3E0650960D312C7
:10E73000E7D26E7003A3E06F60C812E7D2650A707B
:10E7400004A3E0650B60BB740628F582740E129773
:10E750002460AFC3940750AA12E7BB640160A3E032
:10E760006402609EEC050C7099E50CC39B409374A9
:10E77000FD28F582740D39F58312D31F8019E50C3D
:10E780006011EB700E7401650C600302E6957B016D
:10E7900002E6A07AFE7BFF7F050226B974D928F530
:10E7A00082740F12E7B62212E7AB2274CB28F582EF
:10E7B000740F12E7B62239F583E022740128F5823E
:10E7C000740E12E7B62212E7AB650A2212E7AB65B8
:10E7D000082274FD28F582740D12E7B62274F51232
:10E7E000242A8A088B09ECFEEDFF750A00800205D9
:10E7F0000A12DB925022EEFCEFFDE50A12E901124B
:10E80000451FE960EAE50A75F017A4F8A9F074CB92
:10E8100028F582740F12EFB402EEDFE9F87907C32E
:10E82000940D400479018019E8C3940740047903EA
:10E83000800FE8C39403400419198005E870027939
:10E84000000229E274F012242A8A088B098C0A8DAE
:10E850000B890C12332B8A0E8B0FAE0EAF0FEE4FBF
:10E8600060627C177D007900123B478E828F831295
:10E87000EFB78E828F83A3A3A3A3A3A3A3A312D6D0
:10E8800015E50C600712B600E50C800512B60074A1
:10E8900001F09005D112CB656015900598E06401F8
:10E8A000700612E8C7E4800C12E8C77407800512EE
:10E8B000E8C7740112E2755001097A027B00122246
:10E8C0004312E24002C10C12E8CB22EE240EF58284
:10E8D000E43FF5832274F712242A7E00801BEE1297
:10E8E000E9127003A3E0F4600F12E908122D4FE95A
:10E8F000700612E4A71233430E12D25D40E002B15B
:10E900003B75F017A4F8A9F074CD28FA740F39FB01
:10E9100022ED75F017A4F8A9F012E7AB64FE22C04F
:10E9200082C0839005D57485F0A37433F09005D729
:10E93000748BF0A37433F09005D97491F0A3743301
:10E9400002AA5574F712242AEAF8EBF9900514127A
:10E95000E98CCA2406F582E43AF583E0702B8882BC
:10E960008983A3A3A3A3A3A3A3A3A31228419005D0
:10E970001412E991122C8088828983A3E0F9122E67
:10E98000FF7402122A30122E4502B13BE0FAA3E0D6
:10E990002212E98CF5838A8222C082C08390059B73
:10E9A00012EA5CF090059B12CB657005790112327A
:10E9B000CB02C14474F612242A74FC122AC4E9FE64
:10E9C000904DF7E493700874E16E600302EA57EA31
:10E9D0002408F8E43BF98882898312EA5C12EA652C
:10E9E000700E90059BE4F0A3F079011232CB8067A2
:10E9F000900904E06061FA90059B12E2CAEA98E48B
:10EA000099505479001232CB8A088B09AC08AD09B1
:10EA1000ECF8EDF9E875F064A4F8AAF075F064E993
:10EA2000A42AF990059B12D31F12224BE8941AE9ED
:10EA3000940040239007D812CB65601B90059B1271
:10EA4000C87D7402122CAFECF0A3ED12C9CB900775
:10EA5000D812C5CC124872740402C4B5E02401F087
:10EA6000A3E034002212E66CF8A3E0F9E84922C0E2
:10EA700082C08374F8122AC490805AAC18AD1974FD
:10EA80000812295EAC18AD1912451FE96401700423
:10EA9000790080027901028489C082C0839005DBFD
:10EAA000740FF0A3742EF09005DD7415F0A3742E8E
:10EAB000F09005DF74A9F0A37433F09005E174AF12
:10EAC000F0A37433F09005E374B5F0A37433F090C1
:10EAD00005E574BBF0A37433F09005E774C1F0A3AF
:10EAE0007433F074A9443360031233A902C144742F
:10EAF000F412242A74E9122AC48A088B09740412B5
:10EB00002CAF7402F004122A861232418A0A8B0B4F
:10EB1000AE0AAF0BEE4F700302ED3512EDD2700866
:10EB200088828983A37420F0850882850983A3A342
:10EB3000A3A3A3E06401700988828983A3E0D2E6DD
:10EB4000F0850882850983A3A3A3A3A3A3E064019E
:10EB5000700A88828983A3E0D2E7800312ED49120C
:10EB6000EDC37019850882850983A3A312CB656064
:10EB700006EE241612ED6912EDA512C881850882F1
:10EB8000850983A3A3A3A3A3A3A3E0640170031235
:10EB9000ED7A85088285098312D31F12325FE960FE
:10EBA0000312ED7312ED661231BD12CB6BFAA3E0C6
:10EBB000FB8E828F83A3A312DA1312325FE9600304
:10EBC00012C971EE241312BB43700D904DFBE493F8
:10EBD000C0E012CA61D0E0F08E828F83E0A2E750DD
:10EBE0000454038019EE241412BB437012900530B4
:10EBF000E0C0E012ED3FD0E0F0900530E004F0120C
:10EC0000ED5870199008E1E0600D90053BE0700D43
:10EC10008E828F83E07006EE241112C974AC18AD99
:10EC200019EEFAEFFB1231998A088B09EA4509704F
:10EC30000302ED297A217B00123BFB7406122CAFF4
:10EC400012DA137406122CAF12CB65700302ED1D9D
:10EC5000900902E060046401700812B600A3E04469
:10EC600004F07401122A8679501245F17401122CB5
:10EC7000AF12B8987406122CAF12E98CCA2409F5A9
:10EC800082E43AF58312C88190054412B89874154D
:10EC9000122CAF12C8817406122CAF12B88A12ED72
:10ECA00084F07406122CAF12ADBF740212EDBC7466
:10ECB00006122CAF12E99112BC26C0E07406122C89
:10ECC000AF12B88A12ED4FD0E0F0EE240E12ED61D3
:10ECD000C0E07406122CAF12ED94D0E0F07406126E
:10ECE0002CAF12860C12EFB5EE240F12B892740CF2
:10ECF000122CAF12C8818A828B83E0C0E0740E129E
:10ED00002CAFD0E0F07406122A86123115E9F50A0C
:10ED10007406122CAF12D31F123C018003750A1027
:10ED2000AA08AB09123C018003750A10EEFAEFFB4A
:10ED3000123C018003750A10A90A7417029844EE68
:10ED40002414F582E43FF5832212CA65740122245B
:10ED50001EF582E438F58322EE241112B60C64010C
:10ED60002212B5F3E022EE2417F582E43FF5837416
:10ED700001F02212B6094404F02212C9857401F090
:10ED8000A3E4F02212ED8E38F583740222EA240BFC
:10ED9000F582E42212ED982212D0E5C8240CF58207
:10EDA000E438F5832285088285098312D0DEEE12CD
:10EDB000EDB3222418F582E43FF5832212B6421205
:10EDC000D0DF2212EDCAE064012212EDEBA3A3A36F
:10EDD000A32212C85312C9977404F0A3E412EDE7FA
:10EDE000A3A3A3E064012212EDEB22F08508828543
:10EDF0000983A32274F612242A7E00801F7C047DDE
:10EE00000079FF8E088D0974027808122BC6746889
:10EE10002508FA74133509FB123B470E904DFD127D
:10EE2000D26040D902C4B874F512242A74F7122AA9
:10EE3000C4750A00801E850A0875090074027808E6
:10EE4000122BC6746A2508F582741312C86712EE75
:10EE5000CDF0050A904DFD12DB95506D850A0875C1
:10EE6000090074027808122BC612DEA1F47003A305
:10EE7000E0F460DE850A0875090074027808122B38
:10EE8000C6746A2508F5827413350912CB6370A61F
:10EE90007408122CAF7402F0850A0875090078080E
:10EEA000122BC674682508FE74133509FF8E828FF5
:10EEB0008312C87D12EED612463F7C047D0079FF96
:10EEC000EEFAEFFB123B4780897409800FE024FFC4
:10EED000F0A3E034FF2212F04422740D122A307F96
:10EEE000030226B974F012242A74F7122AC4EAFE27
:10EEF000EBFF8C088D09750CFF7408122CAF12F013
:10EF000036124639E9641A700302EFB0750E0080BC
:10EF10000B74FF650C7003850E0C050E904DFDE41F
:10EF200093F8E50EC3985048850E0A750B007402DD
:10EF3000780A122BC612E232F47003A3E0F460D117
:10EF4000850E0A750B007402780A122BC612E23283
:10EF50006E7003A3E06F70C2750F007402780E121A
:10EF60002BC6746A250EF5827413350FF583803035
:10EF7000E493650E702D74FF650C602E850C0A7588
:10EF80000B007402780A122BC67468250AF87413F1
:10EF9000350BF98882898312DA0488828983A3A3D6
:10EFA00012EFB77901740902C10912EED612463F79
:10EFB000790080F139F583E508F0A3E509F02274C2
:10EFC000F412242A74F7122AC4EAFEEBFF74081222
:10EFD0002CAF12F03612463F750A008002050A90E7
:10EFE0004DFD12DB95504C850A08750900740278B6
:10EFF00008122BC612DEA1F47003A3E0F460DE85D4
:10F000000A0875090074027808122BC612DEA16E78
:10F010007003A3E06F70C67C047D0079FF8D0B74D4
:10F0200002780A122BC67468250AFA7413350BFB92
:10F03000123B4702ADAF740212A4BCEEF0A3EFF096
:10F0400012F0442290055112B048AA18AB1922C000
:10F0500082C08374F8122AC485188285198312DA53
:10F06000137402122CAFE4F0A3F07404122CAF74EA
:10F0700001F07405122CAF7401F07406122CAFE489
:10F08000F07407122CAFE412C9CB1233A3028489A7
:10F0900074EE12242A8A088B09ECFEEDFF750C0031
:10F0A000EE65087003EF6509600C123C798A0A8BE3
:10F0B0000BEA450B7006750C0102F14CEEFAEFFB02
:10F0C000123C798A0E8B0FAC0EAD0FEC4D6007EE43
:10F0D000FAEFFB123C8BE4F50EF50F780E122A02C4
:10F0E000AC0AAD0BEEFAEFFB123C737402122A303D
:10F0F000E96059AA0AAB0B123BFB8A0E8B0FEA455B
:10F100000F6046780E122A02780A122A027C007DCD
:10F1100000AA08AB09123C857404122A30E9701D5C
:10F12000780E122A02780A122A027C007D00EEFA7A
:10F13000EFFB123C7F7404122A30E96003750C0166
:10F14000AA0EAB0F123C018003750C10A90C02BE75
:10F150005974F112242A74D2122AC47508008A82C2
:10F160008B83A3A3E0700302F21D14700302F22349
:10F1700014700302F22914700302F22F14700302B8
:10F18000F23514700302F23B14700302F241147062
:10F190000302F42324FE700302F24714700302F406
:10F1A0002324FA700302F27114700302F29524FD15
:10F1B000700302F28314700302F28914700302F2E6
:10F1C0008F24F6700302F24D14700302F253147090
:10F1D0000302F25914700302F25F14700302F26525
:10F1E00014700302F26B24E5700302F29B147003A7
:10F1F00002F2E924F9700302F34514700302F38666
:10F2000014700302F3A714700302F32124FE7003A9
:10F2100002F40C246D700302F41102F42012398BF5
:10F2200002F42312399102F42312399702F42312C3
:10F23000399D02F4231239A302F4231239A902F4EE
:10F24000231239AF02F4231239B502F4231239BB69
:10F2500002F4231239C102F4231239C702F4231233
:10F26000486702F4231239D302F4231239D902F485
:10F2700023EA2403FCE43BFD8A828B83E0FB7A10C3
:10F2800002F4081239E502F4231239DF02F42312E2
:10F2900039EB02F4231239F102F42312F43E12295D
:10F2A000FE7C087D007409122CAFAA82AB83123B4E
:10F2B0003B7403122A307403122A86122D737404CD
:10F2C000122CAFE0C0E07401122CAFD0E0F0740457
:10F2D000122CAFA3E0C0E07402122CAFD0E0F074A7
:10F2E00001122A8E7B0202F3A38A828B83A3A3E0FE
:10F2F000FEEA2403F582E43BF583E0FAA3E0F9EAB1
:10F30000F87404122CAFE8F0A3E9F07403122A8613
:10F31000122D6D7406122CAFAC82AD837B0802F304
:10F32000A312F43E1229FE7C087D007413122A8673
:10F33000123B3B7403122A307410122A861240C901
:10F3400012F42F805E8A828B83A3A3E0F509EA245E
:10F3500003F8E43BF9E8FEE9FF8E828F83A3858200
:10F360000A85830BE0FA8E828F83E0F9122D918E4D
:10F37000828F83EAF0850A82850B83EBF0EEFCEF47
:10F38000FD7B0202F40612F44FE0FA7B00122E031A
:10F39000EAFCEBFD7418122A861239FD7418122A41
:10F3A0008E7B16EEFA80618A828B83A3A3E0F50937
:10F3B000EA2403FEE43BFF0A0A0AFB122D4FE96030
:10F3C00006EEFAEFFB80047A007B008E828F83A327
:10F3D000A3A3A3A3A3A3A3E0FC8E828F83A3A3A3D1
:10F3E000A3A3A3A3A3A3E0F8E4C8F9EC28E439FDA0
:10F3F000122DC1EAFCEBFD7418122A861239FD7435
:10F4000018122A8E7B16AA097967800F1239F780A5
:10F41000127C007D007B007AE0794712380580037A
:10F42000750802A908742E122A307F070226B9E94E
:10F43000851882851983F0AC18AD197B012212F46E
:10F440004FA982AA83890C8A0D750E00780C228A36
:10F45000828B83A3A3E0FE8A828B83A3A3A322745F
:10F46000F012242A74FF122AC4750A0E7E007F004F
:10F47000851882851983E4F0900902E06004640134
:10F48000701CAA18AB19122DD98A088B09AE08AFC7
:10F4900009851882851983E0C333240EF50A850A8D
:10F4A00008AA087B00123BFB8A088B09EA45097011
:10F4B0000302F5648A828B83E412F574780C122AB5
:10F4C00002750E08750F00780E122A027C007D006E
:10F4D0007A017B00123C857404122A30E50C240862
:10F4E000F50C5002050D1231C3850C82850D83EA9F
:10F4F000F0A3EBF0A3740712F5749007A812F57847
:10F50000900902E060046401703E851882851983C9
:10F5100012F578851882851983E06034EEF8EFF9EA
:10F520007C00851882851983E0FAECC39A50218803
:10F5300082898312F57888828983A312F5780CE892
:10F540002402F850DD0980DA850C82850D83E4F011
:10F55000AC08AD09AB0A7A007967123805AA08AB86
:10F5600009123C01EE4F6007EEFAEFFB123C01740A
:10F570000102F89D12F58322E0850C82850D83122D
:10F58000F58322F0A385820C85830D2274F012246A
:10F590002A74FA122AC47A207B00123BFB8A088B59
:10F5A00009AE08AF09EE4F700302F7627C207D00C0
:10F5B00079FF123B478E828F83A385820A85830B56
:10F5C000780A122A027508087509007808122A02BA
:10F5D0007C007D007A017B00123C857404122A3085
:10F5E000E9F5086003750801E50A2408F50A5002E8
:10F5F000050B7402122A7E880C890D780C122A02DF
:10F60000750C04750D00780C122A027C007D007ABE
:10F61000847B00123C857404122A30E96008E508F6
:10F62000D2E1F50880607402122CAF780C122C58CD
:10F630007418780C122A65850A82850B83E50CF014
:10F640007402122CAF780C122C587410780C122AF9
:10F6500065850A82850B83A3E50CF07402122CAF3A
:10F66000780C122C58E50D850A82850B83A3A3F034
:10F670007402122CAF780C122C58850A82850B83E9
:10F68000A3A3A3E50CF0E50A2404F50A5002050B38
:10F69000A818A919880C890D780C122A02750C0279
:10F6A000750D00780C122A027C007D007A837B00A5
:10F6B000123C857404122A30E96008E508D2E2F5AC
:10F6C00008801E851882851983E0850A82850B8350
:10F6D000F0851882851983A3E0850A82850B83A3B0
:10F6E000F0E50A2402F50A5002050B780A122A02F4
:10F6F000750C01780C122A027C007D007A617B0077
:10F70000123C857404122A30E9850A82850B83A392
:10F7100085820A85830B6006E508D2E3F508780A3E
:10F72000122A02750A10750B00780A122A027C0050
:10F730007D007A627B00123C857404122A30E960F5
:10F7400006E508D2E4F5088E828F83E508F0EEFC2A
:10F75000EFFD7B207A017967123805EEFAEFFB1294
:10F760003C01740602F89D74F612242A74FD122AD4
:10F77000C412F8A550010B8A828B83E0FCA3E0F948
:10F78000ECF87401122CAFE8F0A3E9F07401122A2E
:10F790007E880889097808122A027A837B00123C45
:10F7A000798A088B097808122A027C007D007A8306
:10F7B0007B00123C7F7404122A3012F7DE123805E7
:10F7C000740380127B00123C7F7404122A3012F7FB
:10F7D000DE1238057401122A307F020226B9E9854B
:10F7E0001882851983F0AC18AD197B01EEFA7967A0
:10F7F0002274F012242A74FB122AC412F8A55001B4
:10F800000B8A828B83E0F508E4F509F50AF50BA372
:10F81000E0F50CE4F50DF50EF50F7408780C1229DF
:10F82000BD7808790C122B8D8A828B83A3A3E0F517
:10F830000CE4F50D7410780C1229BD7808790C12BF
:10F840002B8D8A828B83A3A3A3E0F50CE4F50E74C1
:10F8500018780C1229BD7808790C122B8D740112BE
:10F860002CAF7808122C497401122A7E8808890965
:10F870007808122A027A847B00123C798A088B0964
:10F880007808122A027C007D007A847B00123C7F7B
:10F890007404122A3012F7DE1238057405122A3069
:10F8A0007F080226B912F908FA2274F612242A7483
:10F8B000FF122AC412F8FC122A027A617B00123C61
:10F8C000798A088B097808122A027C007D007A6107
:10F8D00002F7C474F612242A74FF122AC412F8FC28
:10F8E000122A027A627B00123C798A088B09780816
:10F8F000122A027C007D007A6202F7C412F908F530
:10F9000008E43BF50978082285188285198374017B
:10F91000F08A828B83A3A3E0FEEA24032274F71209
:10F92000242A74FF122AC4EAFCEBFD8C828D83A387
:10F93000A3E0F508851882851983E4F0EC2403FC24
:10F9400050010D8C828D83E0FAA3E0F8E4C8F9EA57
:10F9500028E439FB541FF98C828D83A3A3E0603126
:10F96000740569600A74FF6A700374FF6B700C9011
:10F97000072174FFF0A3F0A3F0A3F0740669600AF6
:10F9800074FF6A700374FF6B703790071774FF8001
:10F990002D740569600A74FF6A700374FF6B700B45
:10F9A000900721E4F0A3F0A3F0A3F0740669600AC5
:10F9B00074FF6A700374FF6B7007900717E4F0A37D
:10F9C000F0AC18AD197B01AA0879671238057401EB
:10F9D000122A307F010226B974F012242A74FC1214
:10F9E0002AC4123CE58A0C8B0D8C0E8D0F9080A0E2
:10F9F0007808122C58780C79081223BB8518828558
:10FA00001983E50CF0850D09E509F5087401122C40
:10FA1000AFE508F0850C08850E0A850F0B74107889
:10FA200008122A657402122CAFE508F07418780CDD
:10FA3000122A657403122CAFE50C12FAEE7B047ADD
:10FA4000097967123805740402F89D02FD3702FD3A
:10FA50003702FD37C082C08374FE122AC412FA89AD
:10FA6000122CAF74FF12FAEE7B027967123805741C
:10FA70000202FD4D02FD37C082C08374FE122AC40B
:10FA800012FA89122CAFE480DC12FD57F0740122C7
:10FA9000C082C08374FA122AC4E580851882851951
:10FAA00083F0E590C0E07401122CAFD0E0F0E5A047
:10FAB000C0E07402122CAFD0E0F0E5FDC0E07403AA
:10FAC000122CAFD0E0F0E5FEC0E07404122CAFD0F1
:10FAD000E0F0E5FFC0E07405122CAFD0E012FAEEC2
:10FAE0007B067A157967123805740602FD4DF0AC75
:10FAF00018AD192274F612242A74FA122AC49080BE
:10FB000069AC18AD19740612295EE5FD8518828569
:10FB10001983F0E5FEC0E07401122CAFD0E0F0E5EF
:10FB2000FFC0E07402122CAFD0E012FCFC7044E87D
:10FB30006008146018146028807875080175090041
:10FB4000E97808122BC6E508F452FD8065750801B6
:10FB5000750900E97808122BC6E508F452FE8052B8
:10FB6000750801750900E97808122BC6E508F452FA
:10FB7000FF803FE860081460171460268034750821
:10FB800001750900E97808122BC6E50842FD8022BC
:10FB9000750801750900E97808122BC6E50842FED0
:10FBA0008010750801750900E97808122BC6E50870
:10FBB00042FFE5FDC0E07403122CAFD0E0F0E5FE9B
:10FBC000C0E07404122CAFD0E0F0E5FFC0E0740593
:10FBD000122CAFD0E012FAEE7B067A147967123855
:10FBE00005740602F7D674F612242A74F7122AC492
:10FBF000908039AC18AD19740912295EE58085181A
:10FC000082851983F0E590C0E07401122CAFD0E03A
:10FC1000F0E5A0C0E07402122CAFD0E0F0E5FDC02A
:10FC2000E07406122CAFD0E0F0E5FEC0E0740712DD
:10FC30002CAFD0E0F0E5FFC0E07408122CAFD0E0AC
:10FC400012FCFC7044E86008146018146028807886
:10FC5000750801750900E97808122BC6E508F45209
:10FC6000808065750801750900E97808122BC6E5E2
:10FC700008F452908052750801750900E97808125D
:10FC80002BC6E508F452A0803FE860081460171402
:10FC900060268034750801750900E97808122BC6C2
:10FCA000E50842808022750801750900E97808128C
:10FCB0002BC6E50842908010750801750900E978A7
:10FCC00008122BC6E50842A0E580C0E07403122CA0
:10FCD000AFD0E0F0E590C0E07404122CAFD0E0F0BB
:10FCE000E5A0C0E07405122CAFD0E012FAEE7B095B
:10FCF0007A167967123805740902F7D6F08A828B72
:10FD000083A3A3A3E0F88A828B83A3A3A3A3E0F930
:10FD10008A828B83A3A3A3A3A3E022C082C083749F
:10FD2000FF122AC48A828B83A3A3A3E0F912306D49
:10FD300012F42F7A11800FC082C08374FF122AC47C
:10FD400012FD5712F43679671238057401122A3001
:10FD5000D083D0820229E28A828B83A3A3E0FA8532
:10FD6000188285198374F52274ED12242A74E9121D
:10FD70002AC4EAFEEBFF8E828F83A3A3E0F50FEE89
:10FD80002403FE50010F7C0E7D0079FF7409122AB6
:10FD900086123B47740B122CAF74FEF0740C122CBD
:10FDA000AF74FFF08E828F83E0F50CA3AE82AF8339
:10FDB000E0F87408122CAFE8F08E828F83A30EAFA8
:10FDC00083740368700DEEFCEFFDAA18AB191245A1
:10FDD000258010E0FAA3E0F9EA851882851983F0FE
:10FDE000A3E9F0EE2408FE50010F8E828F83E0F528
:10FDF0000DA3E0F50EA30E0EAF83605B25E0F50AC0
:10FE0000E433F50BAA0AFB123BFB8A088B098E1020
:10FE10008F1175120078101229FEAC0AAD0B123B3F
:10FE20003B7403122A30E5084509602B7808122A32
:10FE300002AD0EAC0D7402122A86A90C1237817421
:10FE400002122A30EAFCEBFD7409122A86123A03E8
:10FE5000AA08AB09123C017409122A8E7B0EAA0F64
:10FE600079671238057417122A307F0B0226B9748D
:10FE7000F412242AEC4D700C8A828B8374FEF0A35A
:10FE80000402FF0C12FFA98C828D83A3A3A3A3A35A
:10FE900012FF248C828D83A3A3A3A3A3A312FF2804
:10FEA00012FF28A312FF3B12FF3BA312FFA0240B5B
:10FEB000F582E43DF58312FFA0240C12FF9378082D
:10FEC000122C5812FF12122C58E5098A828B8312C9
:10FED000FF18122C5874107808122A6512FF12129B
:10FEE0002C5874187808122A658A828B83E508F0EA
:10FEF000A30AAB83EC2410F8E43DF98882898312CD
:10FF0000FF2488828983A3E08A828B83F07F0402A6
:10FF100026B98A828B83E508F0A30AAB838E828F91
:10FF20008378082212FFE02212FF2C2212FFE48CB9
:10FF3000828D83A3A3A3A3A3A3A32212FF2CA3A315
:10FF40002274F512242AEC4D70158A828B8374FF7B
:10FF5000F0A3F0A314F0A304F0A3F0A3F0802F12F9
:10FF6000FFA9EC240512FF9312FFA02406F508E474
:10FF70003DF509750A0078081229FE8E828F83E00C
:10FF800025E0FCE433FD123B3B7403122A307F036F
:10FF90000226B9F8E43DF9E8FEE9FF8E828F83225C
:10FFA00012FFA42212FFE4EC228C828D83E08A826D
:10FFB0008B83F0A3AA82AB838C828D83A312FFA4D0
:10FFC0002402F8E43DF98882898312FFE08882895F
:10FFD0008312FFDF8C828D83A3A3A312FFDF22A3F2
:10FFE00012FFE422E08A828B83F0A30AAB8322C251
:10FFF000AF75C9AB75C95B80FE0229E2FFFFFFFF49
:020000040001F9
:10000000C082C0837900EA1282053BF583C082C0BA
:100010008390051012D3FFD083D082C3E09CA3E06D
:100020009D500CEA240B12805212803260010902AA
:10003000A37EEA75F00BA4FAA8F075F00BEBA428E8
:10004000FB900512E02AF8A3E03B8882F583E05498
:100050000F22F582E43B12B4F72274F712242A89A6
:100060000812AB90A3E0F9E875F00BA4F8ACF075BA
:10007000F00BE9A42C1283B6E8FEE9FF74016508D1
:1000800060067402650870228A828B831286E2748D
:100090000265087021EA2403FA50010B122D4FE982
:1000A00070148E828F83E4F0800CEA2403FCE43B1E
:1000B0001286D9122D498E828F83E0D2E7F0123E4C
:1000C0000502A80974F412242A12879C79008E82F2
:1000D0008F83E06075890A890B8064E50A75F00BEF
:1000E000A4FAA8F075F00BE50B12803E7049E50A02
:1000F00075F00BA4F8AAF075F00BE50B12833A8E9D
:10010000828F83E085088285098312A1FC128659BB
:10011000EE2403FCE43F1281F8122D4912A9CB1200
:10012000BF281298EAD2E7F0123E05790190051037
:10013000E0F50AA3E0F50B050AE50A7002050B12CB
:1001400085B5E50A9AE50B9B409102AE7E74F512E7
:10015000242AEAFEEBFF750A01740B122CAF1290F1
:10016000A9EC4D6015EC1282053D1287AA790112A7
:100170002D19E508450960758023E50845096044A7
:1001800012820335091287AA1281F9122D4FE964F0
:1001900001701BEEFAEFFB122D1FE9F50A850882AC
:1001A0008509831286517902AA08AB09801112864B
:1001B000DA122D4FE9640170347903EEFAEFFB1285
:1001C0002D1980298E828F83A3E064FE7003A3E043
:1001D000F4700B1286DA122D4FE96401700CEEFAFE
:1001E000EFFB122D1FE9F50A8003750A00028C143B
:1001F000E50A2403FCE4350BFDE5082403FAE435A5
:1002000009FB22E50812C42E2274F712242A900555
:100210001012AAE8EA4B602FEA75F00BA4FAA8F0D6
:1002200075F00BEBA428FBEAFEEBFF123BFB9005FD
:100230001212AAE890051212B4E26012EEFCEFFD71
:100240007900123B478007900512E4F0A3F002A862
:100250000974F612242AE4F508F5097808122A022E
:100260009005101290A475F00BA4FCA8F075F00B8B
:10027000EDA428FD7A237B00123C737402122A300D
:10028000E9FE6003122D37EEF9028B2774F6122473
:100290002A74FF122AC47E007F00803C8518828564
:1002A0001983E4128E13122A027508017509007869
:1002B00008122A02EEFCEFFDEC75F00BA4FCA8F08E
:1002C00075F00BEDA428FD7A237B00123C7F7404AB
:1002D000122A300EEE70010F1283C240BF74010269
:1002E0008B2474F612242A7E007F008039EEF8EF0A
:1002F000F912832E7808122A0275080B7509007806
:1003000008122A02EEFCEFFDEC75F00BA4FC75F070
:100310000BEDA42AFD7A237B00123C857404122A7B
:10032000300EEE70010F1283C240C2028B27E875B7
:10033000F00BA4F8AAF075F00BE9A42AF9900512C5
:10034000E028F508A3E039F5092274F612242A7E84
:10035000007F00804AEEF8EF1283A788828983E04D
:10036000A2E75036C2E7F085820885830978081233
:100370002A0275080B7509007808122A02EEFCEFB4
:10038000FDEC75F00BA4FC75F00BEDA42AFD7A23AF
:100390007B00123C7F7404122A300EEE70010F12A3
:1003A00083C240B1028B27F9E875F00BA4F8AAF0DC
:1003B00075F00BE9A42AF9900512E028F8A3E039BA
:1003C000F92290051012A7F0C3EE98EF9922C0828F
:1003D000C083EC4D600512452580097C087D0079BD
:1003E00000123B4702A37E74F612242A7900EA4BDE
:1003F00060177800EA28F582E412BC3F60047901B6
:10040000780808E8C3940840EB028B2774F712249D
:100410002A74F3122AC4ECFEEDFF85188285198335
:10042000E4F004122CAFEAF0A3EB12A7E2122D6D58
:100430007403122CAFAC82AD83EEFAEFFB122D49A0
:10044000EEFAEFFB122D4F02A80474F712242A745F
:10045000F3122AC4ECFEEDFF851882851983E4F0BF
:10046000EAFCEBFD7403122CAFAA82AB83122D4978
:10047000AA18AB19122D737401122CAF12A2098E97
:10048000828F8312A7D374FE68700374FF696004BF
:1004900079018002790002A80474F712242AEAFE86
:1004A000EBFF122D13E9F508740165087011128530
:1004B00002F4FA88828983E05A4480F0123E0502F1
:1004C000985F74F712242AEAFEEBFF7508008E820B
:1004D0008F83E0602A122D13E9F508740165087016
:1004E0001E128502FA88828983E05A70128E828FEA
:1004F00083E04480FA88828983E04AF0123E050254
:10050000985F12A9CF129A371283A78E828F83E049
:100510002274F412242A8A088B097C007D00EA12D6
:1005200081FB122D49E508128673790085088285C2
:100530000983A3E064FE7003A3E0F460757E007F8E
:10054000008066EEFAEFFB1280326058EEFAEFFBA5
:10055000EA75F00BA4FAA8F075F00BEBA428FB9059
:100560000512E02AF50AA3E03BF50B850882850910
:1005700083A312BC1A850A82850B83A3E06A7003E9
:10058000A3E06B701FE50A2403FAE4350BFB122D80
:100590004FE9640170061281F0122D4912866879C4
:1005A0000112D2330EEE70010F1285B5EE9AEF9B59
:1005B000409102AE7E90051012B4F9C32274F3127A
:1005C000242A8A088B098A828B83128651EA128632
:1005D00073750C00EA1281FB122D4FE96401706AF9
:1005E0007E007F00805FEEF8EFF9E875F00BA4F86D
:1005F000AAF075F00BE9A42AF990051212D2A5E031
:10060000540F603CEEF8EFF9E875F00BA4F8AAF08F
:1006100075F00BE9A42AF9900512E028F50AA3E089
:1006200039F50B1281F012451FE964017012850A39
:1006300082850B83128659128668750C0112D2339B
:100640000EEE70010F1283C2409CA90C7F0502269A
:10065000B9A374FEF0A304F022A312A7F0850882C8
:10066000850983A3129F0E22E50812867DEEF0A372
:10067000EFF02212867D74FEF0A304F02212C43241
:100680003509F5832274F512242AEAFEEBFF8E82E7
:100690008F831286517C007D001286DA122D49EE7E
:1006A000FAEFFB122D13E9F50A7401650A7027129F
:1006B000A7E912832E850882F5831286E21281F95A
:1006C000122D4FE96401700EE5082403FCE435099E
:1006D0001286D9122D49028C14FDEE2403FAE43F50
:1006E000FB22A312BC24129F0E2274F212242A743D
:1006F000E6122AC412879C750C0175080075090062
:10070000750A00750B00851882851983E4F0EE24C4
:1007100003FCE43FFD7403122CAFAA82AB83122DBD
:1007200049AA18AB19122D73E96401701F740B12DA
:100730002CAF1287AC7401122CAF12BC1E7003A335
:10074000E069604AA818A91988088909740D122C53
:10075000AF12A1FBA312A209740E122CAF12A7D3E1
:10076000740D122A86122D6DE964017009740D1240
:100770002A7E880A890B780A122A02AC08AD09EE93
:10078000FAEFFB122D257402122A30E9F50CEEFA6D
:10079000EFFB122D67A90C741A02BB7AEAFEEBFF7D
:1007A00012A9CF74FEF0A304F022F583129A37F950
:1007B00012A9CF129F0E22C082C0837800790080D8
:1007C0000508E87001091285B5E89AE99B5029E807
:1007D000FAE9FBEA75F00BA4FAACF075F00BEBA4A8
:1007E0002CFB900512E02AFCA3E03B8C82F583E011
:1007F000540F70CD79008002790102A37EC082C0BF
:1008000083904E02E49375F016A4FCADF079FF7A64
:10081000FD7B0D123B4702A37E74F612242AEAF8F0
:100820007508007D008012ED12BC31C3994009E0CB
:10083000FAE8C39A400205080D904E02E493FAEDDF
:10084000C39A40E3AA087B00028B2774F012242A83
:1008500074F3122AC48A0C8B0D8C088D09890AEC5A
:1008600045096016AA08AB09122DBB8A0E8B0FAE84
:100870000EAF0FEE4F600302893E7B0080010B122A
:10088000BF1E500F1289E670F574FD28FE740D39F5
:10089000FF80047E007F00EE4F7003028992904D2E
:1008A000E71289B960217403650A60067404650A59
:1008B00070157A047903122D91904E02E493FC9006
:1008C0004DE71289BF5029904DE51289B96028740F
:1008D00001650A60067402650A701C7A02790112C9
:1008E0002D91904E02E493FC904DE51289BF400794
:1008F0007A007B000289B68518828519837401F01D
:10090000122CAFE50CF0A3E50DF0AC08AD097403B3
:10091000122CAFAA82AB83122D49AA18AB19122D43
:100920007F740B122CAF129F078E828F83A3A3A319
:10093000A3A3A3E412D3FBAA0CAB0D1233377800A8
:10094000E50A6007C39405500278048E828F83E520
:100950000CF0A3E50D12C9DFE50AF0E88E828F8363
:10096000A3A3A3A3A312BF2F5001097A027B0012F5
:10097000224312942AA312BB5AA312946EE50A6072
:100980000DC3940350081293F91289D7800312946F
:1009900010F07A047900122D918A08904E02E493A7
:1009A000FAC3E5089AEB940040059014D6E4F012DF
:1009B000320BEEFAEFFB028D721289CFE849221258
:1009C00089CFECC398F8E499F9C3EA98EB9922E44B
:1009D00093F8740193F922F9EE2414F582E43FF5BB
:1009E00083E8F0A3E922EB75F016A4F8A9F01294BD
:1009F00063F42274F212242A74F3122AC48A088B34
:100A000009ECFEEDFF750A00EEFAEFFB122DBB8A32
:100A10000C8B0DA80CA90DE8497003028AB78882D7
:100A20008983E065087004A3E065097003028AB752
:100A300088828983A3A3A3A3E0C394055079888205
:100A4000898312C85F12AC4CE0603488828983A32A
:100A5000A3A3A3E0C394035026904DDDE493FA745E
:100A60000193FB12974C904DDFE493FA740193FBD2
:100A7000E82414F582E439F583EAF0A3EB800DE86D
:100A80002412128ABEF0E82414128ABEF08518825D
:100A90008519837401F0122CAF12C85FF0EEFCEFE1
:100AA000FD7403122CAFAA82AB83122D49AA18AB96
:100AB00019122D7F750A01A90A740D02BB7AF582FD
:100AC000E439F58374FEF0A3042274F612242A128A
:100AD0002DB58A088B09A808A909E84960148882FD
:100AE0008983A3A3A3A3E06009C3940550047901FB
:100AF00080027900803174F612242A122DB58A08FA
:100B00008B09A808A909E849601488828983A3A3EE
:100B1000A3A3E06009C39403500479018002790023
:100B200080057402122A307F020226B974F612245C
:100B30002A122DB58A828B83E5824583600BA3A39D
:100B4000A3A3E0700479018002790080DAC082C03A
:100B500083EAFCEBFD7A007B0002A37BC082C083AA
:100B60007C007D0002A37B74F512242A74F3122A00
:100B7000C4EAFEEBFF8C088D09C3EC94F8ED94FFFA
:100B80004004EE4F606A750A00801974FF650870B2
:100B90000474FF6509600B12CB5C7004A3E0650967
:100BA000603B050A904E02E493F8E50AC398504072
:100BB000E50A1289E760EBEE4F60D0128BFB122C36
:100BC000AF12A7DE122D79E960D87403122CAFACF6
:100BD00082AD83EEFAEFFB12451FE960C5E50A75A9
:100BE000F016A4F8A9F074FD28FA740D39FB8004FE
:100BF0007A007B00740D122A30801B8518828519BB
:100C0000837401F074FF28F582740D39F58312A7FF
:100C1000F0740B22A90A7F030226B974F412242A65
:100C200074F3122AC4750800122DBB8A0A8B0BAE0E
:100C30000AAF0BEE4F601F128C7E128C0E122CAF7F
:100C400012A7DE122D617C167D0079FFEEFAEFFB14
:100C5000123B477508017A047900122D918A0A9097
:100C60004E02E493FAC3E50A9AEB940050099014FB
:100C7000D67401F012320BA908740D02AE7B8518F0
:100C8000828519837401F08E828F83A3A32274F767
:100C900012242AE9FC74FE6A700374FF6B7D0070F5
:100CA00003802C0D128CF05026ED1289E760F412AF
:100CB000D6406A7003A3E06B70E98012ED75F01600
:100CC000A4F8A9F012D6336018E0640360130D1283
:100CD0008CF05015EC60E512945760F2C394055007
:100CE000ED12CDA012BC1780047AFE7BFF02A8098A
:100CF000904E02E493F8EDC39822122DCD02A37E0C
:100D0000C082C083790180F274F012242A8A0A8B8F
:100D10000B7A047901122D918A0C8B0DEA450D6036
:100D200040EA2AFAEB33FB123BFB8A088B09AE0838
:100D3000AF09EE4F60267AFE7BFF122DD374FE6A58
:100D4000700374FF6B601E85088285098312AAE810
:100D5000E5082402F50850E2050980DE750C0080E4
:100D6000047E007F00850A82850B83E50C12AA1C95
:100D70008005740D122A307F080226B9E493F8EC3E
:100D8000C3982274F612242AE4F508F509780812AB
:100D90002A02904E02E493F50874037808122BC6D9
:100DA000129096123C737402122A30E9FE740A6E95
:100DB0006024E4F508F5097808122A02904E02E44E
:100DC0009325E0FCE433FD7A3F7B00123C73740210
:100DD000122A30EE6003122DE502828774F6122487
:100DE0002A74FE122AC4851882851983E4F0A3129E
:100DF0008E13122A027508027509007808122A0259
:100E00007C007D007A227B00123C7F7404122A3021
:100E1000028B22F0A818A919880889097808227479
:100E2000EE12242A74E4122AC48A0E8B0F8C088DC9
:100E300009750C007A227B00123C798A0A8B0B7AA6
:100E40003F7B00123C798A108B11AE10AF11E50A7E
:100E5000450B6017E508650A7004E509650B600B32
:100E6000AC0AAD0B7A227B00123C8B7430122CAF93
:100E7000E0F50AA3E0F50BEE4F6015E50A6E70038E
:100E8000E50B6F600BEEFCEFFD7A3F7B00123C8BB5
:100E9000E4F510F5117810122A02AC08AD097A2297
:100EA0007B00123C737402122A30E9640A70030258
:100EB000908CE4F508F5097808122A02AC0AAD0B0B
:100EC0007A3F7B00123C737402122A30E9640A7084
:100ED0000302908C7404122A7E880889097808120B
:100EE0002A027508027509007808122A027C007D22
:100EF000007A017B03123C857404122A30E96003F6
:100F000002908C851882851983E4F0A3F0FE02908C
:100F1000037406122A7E880889097808122A027545
:100F200008087509007808122A028E0874037808E8
:100F3000122BC6E5082402FCE43509FD7A017B0387
:100F4000123C857404122A30E9600302908C740804
:100F5000122CAFE0F47003A3E0F47003029002746B
:100F600006122A7E880889097808122A027508085C
:100F70007509007808122A027404122CAF1290A985
:100F800074037808122BC6129096123C7F740412D8
:100F90002A30E9600302908C7402122A7E88088944
:100FA000097808122A027508027509007808122AC1
:100FB00002EE25E0FCE433FD7A027B03123C8574EB
:100FC00004122A30E970387402122A7E88088909CE
:100FD0007808122A027508027509007808122A0298
:100FE0007404122CAF1290A42CFCED33FD7A3F7BDD
:100FF00000123C7F7404122A30E9600302908C12C4
:10100000955F0E851882851983C082C083904E0239
:10101000E493F8D083D082C3E098A3E094005021F9
:10102000851882851983C082C0837404122CAF1284
:10103000A209D083D082C3E098A3E0995003028F25
:1010400011A818A919880889097808122A027508B0
:10105000027509007808122A027C007D007A227B42
:1010600000123C7F7404122A30E97020AC0EAD0FE0
:101070007A017B03123C8BE97012742E122CAF1292
:10108000D3FF7A027B03123C8BE96003750C01A944
:101090000C741C02B143E5082402FCE43509FD7A16
:1010A000227B002212D403EC22E0F508A3E0F5092C
:1010B0002274EC12242A74FE122AC4750A008518C0
:1010C00082851983E4F0A3F0904E0293F510F508A1
:1010D00075090074037808122BC6E5082402F50888
:1010E00050020509E51025E0F510E433F5117A22E8
:1010F0007B00123C798A0C8B0DAE0CAF0D7A3F7BD6
:1011000000123C798A0E8B0FA818A919880C890D3A
:10111000780C122A02750C02750D00780C122A0246
:101120007C007D007A227B00123C857404122A30F8
:101130007A017B03123C798A0C8B0D7A027B0312B5
:101140003C798A128B13A812A913E50C450D700A7D
:10115000E5086E7003E5096F7025E849700CE5102D
:10116000650E7004E511650F7015E50C450D607B8B
:10117000EE4F604E85188285198312AAEE60437C7B
:10118000017D037A227B001233C7E9F8880A705B7D
:101190007C027D037A3F7B001233C7E9F8880A702E
:1011A0004AEEFCEFFD7A227B00123C8BE9700EAC1C
:1011B0000EAD0F7A3F7B00123C8BE96011750A017E
:1011C0008029AE0CAF0DE8496004880E890F7810B5
:1011D000122A02780E122A02AC08AD09EEFAEFFBD1
:1011E000122DEB7404122A30E9F50AA90A740212CE
:1011F0002A307F0C0226B974F112242A74D9122ADB
:10120000C47402122CAFE4F0A3F0122DF1E96003D4
:101210000293E87402122A7E880889097808122A43
:10122000027508027509007808122A027C007D0008
:101230007A227B00123C857404122A30E960030292
:1012400093E8904E02E493FA7402122CAF12A209B2
:10125000C3EA98E49950030293E8750A00750B00FD
:10126000750800803E85188285198312BD0312CD52
:101270009312A7D3851882851983129A371289D7BA
:10128000F07A047900122D918A0C904E02E493FAC0
:10129000C3E50C9AEB940040059014D6E4F01232AA
:1012A0000B0508904E0212BB3940030293E874020A
:1012B000122CAF12A209C3E50A98E50B994003026C
:1012C00093E87411122A7E880C890D780C122A0278
:1012D000750C08750D00780C122A0285080C740331
:1012E000780C122BC6E50C2402FCE4350DFD7A22A5
:1012F0007B00123C857404122A30E970A474131226
:101300002CAFE0F47003A3E0F46096050AE50A70E0
:1013100002050B7404122CAF7401F07413122CAF7D
:1013200012A209740F122CAF12A7D37404122A86CA
:10133000122D79E970030292A112D3FC7411122CC0
:10134000AF12BC1A123337E50875F016A4F8A9F0ED
:1013500074FD28FE740D39FF7411122A7E880C89E1
:101360000D750E00780C1229FE7C087D00EEFAEF58
:10137000FB123B3B7403122A3012BF345001097A2E
:10138000027B0012224312942A12946EA818A91903
:10139000880C890D780C122A02750C02750D0078E4
:1013A0000C122A02AC08EC2CFCE433FD7A3F7B00E3
:1013B000123C857404122A30E96003029281851878
:1013C00082851983E0F47003A3E0F4600302926560
:1013D000E508129458600BC3940350061293F90267
:1013E000927D1294100292807402122CAFE0F97474
:1013F00027122A307F070226B9904DDD1289CFEEE1
:1014000012CD97129F0E904DDFE493F87401932252
:10141000EE241212941EF0EE241412941E22F58271
:10142000E43FF58374FEF0A30422E88E828F83A349
:10143000A3A3A3A3A3A3A312944F740112944FA335
:1014400074AAF0EE2410F582E43FF583E4F0221252
:10145000CA02A3A3A3A322ED75F016A4F8A9F01263
:10146000946322740128F582740E12D4EF22A3F043
:1014700012A9CFE4F0EE240CF582E43FF583E4F00A
:10148000A3F0A3F0A3F02274F312242A74FE122A0C
:10149000C4851882851983E4F0A3F0F50C02952029
:1014A000E50C75F016A4F8A9F074FD28F50A740D82
:1014B00039F50B850C82AE82780A122A027508086B
:1014C0007509007808122A028E0874037808122B16
:1014D000C6129096123C7F7404122A30E50A241436
:1014E000F508E4350BF5097808122A02750802752B
:1014F00009007808122A02EE2EFEE433FFEEFCEF1C
:10150000FD7A3F7B00123C7F7404122A30850A82E8
:10151000850B83A3A3A3A3E0F4600312955F050CDE
:10152000904E02E493F8E50CC39850030294A0A8EF
:1015300018A919880889097808122A0275080275FD
:1015400009007808122A027C007D007A227B0012B2
:101550003C7F7404122A307402122A3002864C85B1
:101560001882851983E02401F0A3E03400F022C042
:1015700082C0837D008009EA24FF1AEB34FFFB0D53
:10158000128CF05016129457C3940550F2EA4B7027
:10159000E674FD28FA740D39FB80047A007B0002A2
:1015A000A37E74F712242A74F3122AC47E000296D2
:1015B0003AEF75F017A4F8A9F012D61612BD00750F
:1015C000F016A4FAABF074FD2AF582740D12BF5226
:1015D0007003A3E0696040EF75F017A4F8AAF0EA81
:1015E000F912D61639F58312A2097401122CAFE054
:1015F000687003A3E069601FEF75F017A4F8EAF9BB
:1016000074CD28FC740F39FD7403122CAFAA82AB81
:101610008312451FE96013EF75F017A4F8A9F07461
:10162000CB28FA740F39FB1233430F904DEEE4933D
:10163000F8EFC39850030295B10E904E0212D18577
:10164000501FEE12D639F47003A3E0F460EB128B56
:10165000FB122CAF12A7DE122D79E960DC7F00802F
:10166000CA02A80474F712242A74F3122AC490053B
:10167000E312B4E27003029710750800802BE508AE
:1016800075F016A4F8EAF9741128F582740E12D4D4
:10169000EB64FE7003A3E0F4600D740F28F5827410
:1016A0000E39F58312BB700508904E0212BB3950FB
:1016B0005FE50875F016A4F8AAF0EAF912945F60E5
:1016C000E6C3940350E1740F28F582740E12B4DF60
:1016D00070ACE50875F016A4F8EAF974FD28F87402
:1016E0000D39F9E8FEE9FF1297AE1297A41248727D
:1016F000128C7E128C0E122CAF12A7DE122D79E9FD
:1017000060A57403122CAFAA82AB83122DC78097F9
:1017100002A80474F612242A122DB58A088B09A88F
:1017200008A909E849602088828983A3A3A3A3E0CC
:101730006011C39403500CE82414F582E412BC1722
:1017400012974C790180027900028B27E82412F568
:1017500082E439F583EAF0A3EBF02274F712242A2D
:10176000EAFEEBFF9005DD12B4E260309005E31273
:10177000B4E260289005E712B4E2602012CEE112D4
:101780004872E9701712979F124872E96401700C51
:101790008E828F83A3A312CECE12487202A80912A2
:1017A00097AEA3A312B4F99005E312CED822904DC0
:1017B000DFE493FC740193FD8E828F8322C082C08C
:1017C0008390051974C7F0A37430F090051B74C1A1
:1017D000F0A37430F090051F74BDF0A3742EF002D6
:1017E000A37EC082C08390051D74BBF0A37430F04B
:1017F00002A37E74F712242AEAFEEBFF900553E061
:101800006408601CE0640460178E828F83E05403D8
:101810006401704112B8D2F8129864E06406703521
:101820008E828F83A3A3E064FE7003A3E0F460259F
:101830008E828F83A3A312C4147003A3E06970087F
:10184000EE241512C4096005123187800312318D10
:10185000E9F50880037508C2EEFAEFFB123C01A916
:101860000802A809A3E0F58388822274F412242ACE
:101870008A088B09129A33FAE82AFAE43400FB1238
:101880003BFB8A0A8B0BAE0AAF0BEE4F6055850807
:1018900082850983E0FC7D007900123B478E828FB0
:1018A00083A31286511231C38E828F83A3A3A3A375
:1018B000EAF0A3EB1298EAF8EE28F8E43F1287AFBB
:1018C000850882850983A3E0C0E012BF14D0E0F050
:1018D0001231D512BF0AE9129EEAE0C0E0129EE082
:1018E000D0E0F0EEFAEFFB02AE7EF08508828509CB
:1018F00083E02274F412242A74E8122AC48A088B22
:10190000098C0A8D0BE9FE900553E064046005E044
:101910006408700479C2803CA37808122C49EE90C8
:10192000055A129B76123B478518828519837808E1
:10193000122C497405122CAFEEF07404122CAF7403
:1019400001F07407122CAFE4F0900553740212A753
:10195000E212460F02AE7974F412242A74E8122AB5
:10196000C4EAFEEBFF90051412B4E26003029A2E63
:101970007A077B00123BFB90051412AAE89005142D
:1019800012B4E27003029A2A8E828F83122C8C90FA
:101990000514E0FCA3E0F5838C82122C98EE24045D
:1019A000F50AE43FF50B850A82F583E0C0E0900577
:1019B0001412B4B6A3A3A3D0E0F0EE2405F508E416
:1019C0003FF509850882F583E0C0E090051412B464
:1019D000C4D0E012A7D8C0E0900514129A37C824EA
:1019E00006F582E438F583D0E0129B76123B478EF1
:1019F000828F83122C8C851882851983122C9885EE
:101A00000A82850B83E0C0E07405122CAFD0E0128F
:101A100098EAC0E07404122CAFD0E0F07407122CE6
:101A2000AFE412A7E212460F800679108002790116
:101A300002AE798A828B83E0F8A3E022C082C08361
:101A400090051412B4E2601090051412BC1A123CF6
:101A500001900514E4F0A3F01230F11232E302A376
:101A60007E74F412242A74E8122AC48A0A8B0BECBE
:101A7000FEEDFF89087428122CAFE0FC7429122CAB
:101A8000AFE0FD740F6C7005740F6D60129015411E
:101A9000E064026005ECC39D500579C1029B73743C
:101AA00024122CAF122C8C900554122C98E508901F
:101AB000055AF0EC900558F0EDA3F0742A122CAF03
:101AC000E090055BF074FF650A700474FF650B70AD
:101AD00024901555E0F47003A3E0F4700C123B5908
:101AE000900551EAF0A3EB801290155512CDBDE898
:101AF000F0A3E9800690055112BF28F0EE4F601761
:101B0000EEFAEFFB123397E96401700BEEFCEFFD88
:101B10007A657B05124525900544E4F0A3F0900515
:101B200047F0A3F0900564F0901541E0640270085E
:101B3000900558740FF0A3F09005537405129B762E
:101B4000123B477404122CAFE4F0900554122C8C15
:101B5000851882851983122C9890055AE0C0E0748C
:101B600005122CAFD0E0F07407122CAFE412A7E2FC
:101B700012460F02AE79F07C187D007900AA18ABEE
:101B8000192274F712242AE9900518F07A807B0054
:101B900090059EE0F9123CCD122E5D790002A80955
:101BA000C082C083900518E07003123F49122E5D79
:101BB00002A37E74F012242A900518E09014D570C8
:101BC0000FE060057900123DC99014D5E4F0804A19
:101BD000E064016008900518E0F9123DC99014D541
:101BE0007401F0900518E0F46030E0F50CE4F50DB8
:101BF000F50EF50FF09080A07808122C58780C792B
:101C00000812233B780C1229FA7A807B0090059EFB
:101C1000E0F9123CC17404122A307AD57B14794160
:101C20001245F7028D7774F712242A7CFE7DFF128D
:101C30002E6902A80974F212242AEAFEEBFF8C082E
:101C40008D09890A900553E06408706C122DBB8BD6
:101C50000DEA450D600479C5806074FE6508700466
:101C600074FF6509701C7402550AF9122F8F8A08D7
:101C70008B0974FE6508700474FF6509700479C7E8
:101C80008038E50AA2E1500CA2E350047904800EEA
:101C90007903800AA2E35004790280027901EEFC04
:101CA000EFFDAA08AB09122D978B09EA45096004DC
:101CB000790080067910800279C202BB7D74F4122B
:101CC000242A74E8122AC48A088B098C0A8D0BE92D
:101CD000FE9005537401129B76123B47851882854E
:101CE00019837808122C497405122CAFEEF0740495
:101CF000122CAF7403F07407122CAFE412A7E21297
:101D0000460F02AE79122E7B02A80974F712242A1C
:101D10007C0080F174F012242A74FC122AC4E98534
:101D20001882851983F0EAFEEBFF8C0A12D3FC12AD
:101D300030E58A088B09EA4509700579CA029EDBFD
:101D40008A828B83A3A3A3A3A3A3A3E064FE70034F
:101D5000A3E0F4700579C3029EDB1231C38A0C8BB9
:101D60000DA80CA90D850882850983A3A3A3A3A3AD
:101D7000A3A3E0687003A3E069700579C2029EDB4B
:101D800090055112A209850882850983E0687003D5
:101D9000A3E069601285088285098312A061AA0800
:101DA000AB0979501245F790055112BC1A1233490C
:101DB000850882850983A3A3A3A3A3A3A3A3A3A3A5
:101DC000E00490056412A04D1245257402122CAF58
:101DD0007402F014122A861232418A0C8B0DAE0C5A
:101DE000AF0DEE4F7003029ED112AE027406F0A347
:101DF000A882A98390053E12C04012B8AF1231BD2F
:101E000012AADFEE241312B8B212BF007440F0A37E
:101E1000E4129EEAA3A3A3A3A3129F07129EE0E5E8
:101E20000A12AA1C122E2DE9F50B6003029ED49013
:101E300005537409F0E5082407FEE43509FFEEFABE
:101E4000EFFB794B1245F78E828F8312A0579005D6
:101E500046E0F8851882851983E068600CE09005FB
:101E60004612A7E279E11245F790152E12A20990C9
:101E70001530E0687003A3E069602890051612A78A
:101E8000D390153012BC1A1231ED129EF4780C1258
:101E900029FA7A017B0090059EE0F9123CC1740496
:101EA000122A307A007B0490059EE0F9123CCD1294
:101EB0009EF47402780C1229BD780C1229FA7A006B
:101EC0007B0490059EE0F9123CC17404122A308014
:101ED00003750B10900788E4F0A90B7404028D744D
:101EE000EE2411F582E43FF58322F085088285090E
:101EF00083A3A322901530E0F508A3E085080CF534
:101F00000DE4F50EF50F2212BF4A129F0E22E8F0E3
:101F1000A3E9F02274F612242A74E2122AC4851866
:101F200082851983ECF0A3EDF0EAFEEBFF890890BF
:101F30000553E064046005E06408700579C202A0FE
:101F4000487429122CAFE064FE7003A3E0F470051E
:101F500079C302A0487C197D0079007405122A8695
:101F6000123B47900553740312A7E279501245F7CC
:101F70007429122A86794B1245F7851882851983B0
:101F800012A061E508900546F07429122CAF12A04A
:101F9000577428122CAFE0F50990053E12A04D129F
:101FA000452574CE55094480C0E0741D122CAFD075
:101FB000E0F0900902E060046401700B742B122CB5
:101FC000AFE004900564F0741A122CAF7402F07440
:101FD00029122CAF12A2097412122CAFE8F0A3E957
:101FE00012A202741B122CAF12A7D37410122CAFC2
:101FF000E508F0740D122CAFE4F0900559740FF061
:102000007A597B0579541245F7900558740FF07A88
:10201000587B0579471245F7900558E0C3940F5057
:102020001F7410122CAFE0C0E07402122CAFD0E08D
:10203000F07404122CAF7401F004122A8612461BAD
:102040007405122A861245FD741E028B24F0EEFCE4
:10205000EFFD7A657B052212A7F0900547129F0ECF
:102060002212CDC1129F0E2274F712242AEB900582
:102070005BF01230D302A80974F712242A74E91213
:102080002AC4EAFEEBFF7508008E828F83A3A3A308
:10209000E0C0E07406122CAFD0E0128C86E0C0E005
:1020A0007408122CAFD0E0F07409122CAF74011236
:1020B000A1FC12B4E2600D8E828F8312BC1A122D25
:1020C0004FE970357407122CAFE4F01231BD74047F
:1020D000122CAF12AAE8900553E06404700E12317E
:1020E000C97402122CAFEAF0A3EB80557402122CD3
:1020F000AF74FDF0A374FF8048900902E0600764AC
:1021000001600302A18DAC18AD198E828F8312BCC1
:102110001A122D5B8E828F83A3A3A3A3E070307469
:1021200007122CAF740112A2027402122CAF12A774
:10213000D38E828F8312A2097404122CAFE8F0A30D
:10214000E9F07402122A86123229E9F508803E125B
:10215000A203740A122CAF12A7D37414122CAF125C
:102160008C84A3E0C0E07415122CAFD0E0F074169C
:10217000122CAF12A1FB12D3FF740C122CAFAA8247
:10218000AB83124525740A122A86123DE1A9087410
:102190001702A80674F712242A74F8122AC4EAFE59
:1021A000EBFF7900900553E064086005E06404707B
:1021B0004585188285198374FDF0A374FFF01231F0
:1021C000BD7402122CAF12AAE87405122CAF12A132
:1021D000FBA3E0C0E07404122CAFD0E012A1FCE03D
:1021E000C0E07406122CAFD0E0F07407122CAFE4FC
:1021F00012A7E2123229740802A806E4F08E828F38
:102200008322F085188285198312A7F02274F112B7
:10221000242AECFEEDFF7C008C0BE92479602B2452
:10222000FC700302A2AD24F3601324FC601514605B
:102230003A14600302A31990055302A33890054194
:1022400002A338123331EA02A339750BC112333DB0
:102250008A0C8B0D8B09EA4509700302A33E750EAB
:1022600000780C1229FE7C1702A306750BC9900991
:1022700002E060076401600302A33E783B79117AB3
:1022800000801788828983E064FE7003A3E0F46015
:10229000010CE82407F85001090A904DEBE493FB88
:1022A000EAC39B40DEEC8E828F83F08067750BC99A
:1022B000900902E060076401600302A33E750BC150
:1022C00075083B7509117800800C0CE5082407F5AA
:1022D000085002050908904DEB12C8C350608508EC
:1022E00082850983E064FE7003A3E0F460DD8C0C5A
:1022F000EA650C4B70D485080C85090D750E0078C5
:102300000C1229FE7C077D00EEFAEFFB123B3B74BA
:1023100003122A30750B008025747F29C3941E4058
:1023200005750BC98018743029F8E43405F9E824E0
:102330007FF582E934FFF583E08E828F83F0A90B6D
:102340000293F4C082C083900525745FF0A3742FBC
:10235000F09005CB7489F0A37432F0900529749540
:10236000F0A3742FF090052B745FF0A3742FF090FE
:10237000052D749BF0A3742FF08003122DC1D08320
:10238000D0820229E274F412242A74F9122AC48A2F
:10239000088B098C0A8D0B851882851983780812A1
:1023A0002C497404122CAFE9F07405122CAFE4F040
:1023B0007406122CAFE412A7E2122E3F740702AE8D
:1023C0007B74F512242A8A088B098A828B8312D2A5
:1023D00036EE4F700302A5799004E412B4E2601562
:1023E0008A828B83A3A3E0F9EEFAEFFB9004E51257
:1023F00098651248728E828F83A3A3A3A3A3A3A37D
:10240000A3A3E06402600302A4E28E828F83A3A3ED
:10241000A3A3A3A3E05402700302A5068508828546
:102420000983A3A3E064E9700302A50685088285F9
:102430000983A3A3E064CD700302A5068508828505
:102440000983A3A3E064F0700302A5068E828F8344
:10245000A3A3A3A3A3A3A3A3A3A3E07016901545CE
:10246000E0048E828F83A3A3A3A3A3A3A3A3A3A308
:10247000F0801012A58A12325FE970077A307B0172
:10248000124105850882850983A3A3E0701F750AA0
:102490000080097A367B01124105050A850882858C
:1024A0000983A3A3A3E0F8E50AC39840E68E828FD0
:1024B00083A3A3A3A3A3A3A3A312C9F6A3A3A3A324
:1024C0007404F090154612BF44E812A57C123CD368
:1024D000EA4B4C4D700C7A207B0090059EE0F9127F
:1024E0003BA18E828F83A3A3A3A3A3A3A3A3A3E053
:1024F000640260128E828F83A3A3A3A3A3A3A3A3CA
:10250000A3E0640670738E828F83A3A3A3A3A3A307
:10251000E0A2E05064850882850983A3A3E0F9EE78
:10252000FAEFFB12471D8E828F83A3A3A3A3A3A35D
:10253000E054FEF012A58A12325FE985088285090F
:1025400083A3A3702AE070237A2F7B011241057EBA
:1025500000850882850983A3A3A3E0F8EEC3985001
:10256000187A367B011241050E80E67A318005E04B
:1025700070077A2D7B01124105028C16F0A3E9F059
:102580007A207B0090059EE0F9228E828F8312CE06
:10259000D812B4F92274EC12242A74DB122AC4EA89
:1025A000FEEBFF8C108D11750E007405122A8E1231
:1025B0002CE37412122CAFE070087415122CAFE0EB
:1025C00060207405122CAFE0A2E6501B8E828F8330
:1025D000A3A3A3A3A3A3A3A3A312BC1A12325FE9CC
:1025E00060057A3502A6DE7405122CAFE0540C6447
:1025F000047005750D018003750D00E0A2E55030F3
:10260000750E01E50DA2E040271231C38A088B093F
:10261000A808A90912B8D2687003A3E06960117410
:1026200005122A8E12C423124741E9600302A6DC78
:102630007405122CAFE0A2E650227406122CAFE013
:10264000540370187405122CAFE0540C640C600C29
:10265000E0540C64086005750C018003750C00746F
:1026600005122CAFE05403F8740268700E74051262
:102670002A8E12C423122CF502A7C8740168704177
:10268000E50CA2E0500B7405122A8E12C423122C02
:10269000E97405122A7E7403122CAFE8F0A3E91244
:1026A000A7E8851882851983E8F0A3E912A7D8C0A6
:1026B000E07402122CAFD0E012A7E212484902A740
:1026C000C8E8600302A7C890053BE0640170178E5C
:1026D000828F83A3A3A3A3A3A3E0700A7A347B0110
:1026E00012410502A7C87424122CAF740212A7E885
:1026F000741C122CAF12A7D3E50CA2E0500B74058A
:10270000122A8E12C423122CE97439122CAF7808C5
:10271000122C58E50DA2E0EE5072240F12C409C02D
:10272000E07417122CAFD0E0F09004E612B4E2701F
:102730000302A7C81231C38A128B13A812A91374FB
:102740001C122CAFE0687003A3E069707B7808125C
:1027500029FAE50EF5087808122A068E828F83A3DF
:10276000A3A3A3E0F5087808122A067810122A021B
:10277000A90C740D122A8E7424122A869004E61273
:10278000BC8C1248727408122A30803C12C407F5BF
:102790000C780C122A0678081229FAE50EF508784A
:1027A00008122A067810122A02900551122841EECA
:1027B000241212C409F97426122A8E740F122A8662
:1027C000124711740A122A3074250291EFA3A3A3B1
:1027D000A3A3A3E8129F0F2212C9FEA3E022E8F0F0
:1027E000A3E9F0AA18AB1922F012A9CF12A7F02280
:1027F00012A7F422E0F8A3E0F92274F712242A12B7
:102800003DA58005740D122A307F010226B974F7A8
:1028100012242A123DB180F174F712242A123DBD10
:1028200080E7C082C083123DB702A37E74F71224F2
:102830002A123DC380D374F712242A7409122CAFD4
:10284000E0F5087808122A06123DD5740180B7C059
